:100000000063002029300100AD5F0200FD2F0100D8
:10001000FD2F0100FD2F0100FD2F01000000000059
:100020000000000000000000000000009D2A010008
:10003000FD2F010000000000492A010069C30100F2
:10004000552B010031850200552B0100552B010075
:10005000552B0100552B0100552B0100552B01009C
:10006000F9840200552B0100552B01001785020071
:10007000552B0100552B0100552B0100552B01007C
:10008000552B0100552B0100552B0100552B01006C
:10009000552B0100552B0100552B0100552B01005C
:1000A000552B0100552B0100552B0100552B01004C
:1000B000552B0100552B0100552B0100552B01003C
:1000C000552B0100552B0100552B0100552B01002C
:1000D000552B0100552B0100552B0100552B01001C
:1000E000552B0100552B0100552B0100552B01000C
:1000F000552B0100552B0100552B0100552B0100FC
:1001000053B94AB9002908BF00281CBF4FF0FF317E
:100110004FF0FF3000F06CB9ADF1080C6DE904CE82
:1001200000F006F8DDF804E0DDE9022304B07047D2
:100130002DE9F047089E0D4604468E46002B40F000
:1001400082808A42174646D9B2FA82F24AB1C2F197
:10015000200105FA02F320FA01F1974041EA030E6B
:1001600094404FEA1748230CBEFBF8FCB9B208FBD9
:100170001CEE43EA0E430CFB01F098420AD9FB182F
:100180000CF1FF3580F01681984240F21381ACF1FA
:10019000020C3B441B1AA4B2B3FBF8F008FB10336B
:1001A00044EA034400FB01F1A14209D93C1900F1E2
:1001B000FF3380F00181A14240F2FE8002383C44CE
:1001C000641A40EA0C4000211EB1D4400023C6E965
:1001D0000043BDE8F08702B9FFDEB2FA82F2002ADE
:1001E0004FD1CB1B4FEA174E1FFA87F80121B3FB03
:1001F000FEFC250C0EFB1C3345EA034508FB0CF303
:10020000AB4207D97D190CF1FF3002D2AB4200F2AC
:10021000E7808446ED1AA3B2B5FBFEF00EFB105545
:1002200043EA054408FB00F8A04507D93C1900F152
:10023000FF3302D2A04500F2D7801846A4EB080491
:1002400040EA0C40C0E78B4208D9002E00F0AF8096
:100250000021C6E900050846BDE8F087B3FA83F13E
:1002600000294BD1AB4202D3824200F2B780841AFC
:1002700065EB030301209E46002EAAD0C6E9004E7E
:10028000A7E7C2F1200C01FA02F3974020FA0CF024
:100290004FEA174E21FA0CFC1843BCFBFEF1050C8B
:1002A0000EFB11CC1FFA87F845EA0C4501FB08F359
:1002B000AB4204FA02F409D97D1901F1FF3C80F048
:1002C0008B80AB4240F2888002393D44EB1A85B204
:1002D000B3FBFEF00EFB103345EA034500FB08F3C9
:1002E000AB4207D97D1900F1FF3C71D2AB426FD907
:1002F00002383D44EB1A40EA014178E7C1F1200C95
:100300008B4022FA0CF71F4320FA0CF405FA01F394
:100310004FEA174E25FA0CF51C43230CB5FBFEF9EA
:100320001FFA87F80EFB195543EA054509FB08FA41
:10033000AA4502FA01F200FA01F308D97D1909F180
:10034000FF3047D2AA4545D9A9F102093D44A5EBA2
:100350000A05A4B2B5FBFEF00EFB105544EA0544B5
:1003600000FB08F8A04507D93C1900F1FF352DD254
:10037000A0452BD902383C4440EA0940A4EB0804CC
:10038000A0FB02894C45C6464D4619D316D05EB136
:10039000B3EB0E0264EB050404FA0CFCCA404CEA11
:1003A0000202CC40C6E900240021BDE8F0873146B6
:1003B00030460EE7AC46EDE6184601E74345E6D287
:1003C000B8EB020E69EB07050138E0E72846D3E7F2
:1003D00060468FE78146BAE7614677E708464BE714
:1003E000ACF1020C3D4415E702383C4426E700BF5F
:1003F000704700BFF8B515460A4A1C4656682EB12C
:1004000001B02A46B446BDE8F040604700208DF8B0
:10041000000068460BF0AEF99DF80000281A207025
:100420000020F8BD00000020002819D003781349EF
:10043000134A13B1012B0ED011E00379012B00D028
:100440006BB943790BB1012B09D18368643B8B42B3
:1004500005D2C0680EE00379012B02D00BB1002059
:10046000704743790BB1012BF9D1C368643B8B42D0
:10047000F5D280689042F2D8012070473D86010095
:10048000FF1FA10710B5054C206810B18047002060
:100490002060BDE8104001F0DBBF00000800002034
:1004A0002DE9F0410E46050004D000F045F807465E
:1004B00000240AE06FF01500BDE8F081204600F04E
:1004C00041F8807838B1641CE4B2BC42F6D300BF76
:1004D0006FF00B00F0E72746FF2CF9D0204600F024
:1004E00031F804460BF0E1FA27712146074801F084
:1004F00087FFE070202805D00120A560A07037702C
:100500000020D9E76FF02200D6E700001BB80000FA
:1005100010B5820702D06FF00D0010BD054A1170B2
:10052000506028B101EBC1018A0000210BF043FDAE
:10053000002010BD0C00002001480078704700002A
:100540000C00002005490A78904201D30020704732
:10055000496800EBC00001EB800070470C000020F0
:1005600070B50546202A27D019481A4C00EB831C89
:100570000CEB420004EB8303202922D00CEB410159
:1005800040784C784870204601460CEB410091427F
:1005900005704078F8D193F82220202A1ABF0CEB7E
:1005A0004202547083F8214020220CEB410C8CF85D
:1005B000012083F8221070BD40F27E21702003F0EC
:1005C00069F993F82040407883F82000DBE70000C9
:1005D0000C0E00208C0E00202DE9FF4F85B0154633
:1005E0000C4602F0F5F8284420F07F400290216884
:1005F000081A0002C11700EB11600012002800F376
:10060000D580AC48089FAC4E00EB8700039090F873
:1006100020502020E9460DF104088DF8000006F571
:10062000407A202D18BF0AEB871B25D005EB45002B
:1006300006EBC0002268C168511A0902CA1701EB13
:1006400012610830091217D4618971B1418961B909
:1006500000F0BAFD02F0BCF82168081A0002C117C8
:1006600000EB11600012332806DB0BEB450089F824
:1006700000504578202DD9D199F8000088F8000065
:10068000A146202D1CBF8D4800EB871B00F00E817A
:1006900005EB450106EBC10AD9F80420DAF8081089
:1006A0004846891A0902CA1701EB12610AF10807C4
:1006B000091215D47989002900F0F88041890029B0
:1006C00040F0F48000F080FD02F082F83968081AEA
:1006D0000002C11700EB11600012332880F2E6809F
:1006E00088F800509AF8141099F80C00814206D945
:1006F0000BEB45004578202DCAD100F0D7B89DF806
:10070000040000EB400006EBC005688AEF68002893
:1007100043D16089E8B3A8680BF065FA698A2A7C3E
:10072000674B1144491C4218984204D940F20961B0
:10073000702003F0AFF86348814204DD40F20A61A3
:10074000702003F0A7F86048814204DA40F20B61A0
:10075000702003F09FF85D489042DCBF02F5F7027D
:10076000A2F1F85205DD002ABCBFA2F5F70202F1A2
:10077000F852104602F02CF820F07F41781A00025F
:10078000C21700EB126000123328B8BF01F133002A
:1007900000E002E0B8BF20F07F470298381A00025C
:1007A000C11700EB11600012002803DD09B0002022
:1007B000BDE8F08FD4E90010401A384427F07F419B
:1007C00020F07F40C4E900100398DDF820806F46D8
:1007D00090F8205020200DF1040A8DF80000202D03
:1007E0001CBF364800EB881925D000BF05EB45003B
:1007F00006EBC0002268C168511A0902CA1701EB52
:1008000012610830091216D4618971B1418961B948
:1008100000F0DAFC01F0DCFF2168081A0002C117C1
:1008200000EB11600012332805DB09EB45003D7039
:100830004578202DDAD138788AF800002746202D17
:100840001CBF1E4800EB881B30D005EB450106EBB2
:10085000C1097968D9F808203846511A0902CA171F
:1008600001EB126109F10808091212D4B8F80A1054
:10087000E1B14189D1B900F0A7FC01F0A9FFD8F896
:100880000010081A0002C11700EB11600012332893
:100890000CDA8AF8005099F81400397B88427FF608
:1008A0002EAF0BEB45004578202DCED109B00120AD
:1008B000BDE8F08F8C0E00200C0B00200C0E0020E9
:1008C000FF7F841E0020A10700E05EF80080841EE8
:1008D0002DE9F05F04463C480E4600EB86003B4F96
:1008E00090F82050202098469246107007F54079E5
:1008F000202D18BF09EB861B28D000BF05EB450053
:1009000007EBC00000F10801C0682268101A00025D
:10091000C21700EB1260001218D4608978B14889C0
:1009200068B9084600F050FC01F052FF2168081A2F
:100930000002C11700EB11600012332806DB0BEB3D
:1009400045008AF800504578202DD7D19AF800004C
:1009500088F80000202D18BF09EB861A30D005EB6F
:10096000450107EBC1096168D9F808202046511AF2
:100970000902CA1701EB126109F10806091210D425
:100980007189E9B14189D9B900F01EFC01F020FF5D
:100990003168081A0002C11700EB116000123328F9
:1009A0000EDA88F8005099F81400217B884202D8AA
:1009B0000020BDE8F09F0AEB45004578202DCED100
:1009C0000120BDE8F09F00008C0E00200C0B0020E1
:1009D0002DE9F74F4FF0000898B016460D46C34674
:1009E00002F06EF90446012D18BF022D05D040F625
:1009F00094114FF0700002F04DFFFD490120086096
:100A0000FC498968086000200C90401E0E90FA494D
:100A100006EB460001EBC00308330FAF0FCB87E8AE
:100A20000F000FA800F0D0FB0D90F348BDF84690E2
:100A3000B0F89C03ADF84C00B9F1000F14BF4FF0B3
:100A4000010A4FF0000A0F981490BAF1000F09D074
:100A5000EA4890F82C0028B902F0B8FE002808BF38
:100A6000012700D00027E64800221592007816469C
:100A7000012818BF032840D1E148B0F80280A8EB54
:100A800009001590C84538D90D9B6FEA0801DFF8B9
:100A900074E358180DF10C0C17AA734504D940F2F1
:100AA0000961702002F0F6FED74B994204DD40F256
:100AB0000A61702002F0EEFED44B994204DA40F253
:100AC0000B61702002F0E6FED1498142DCBF00F5E7
:100AD000F700A0F1F85005DD0028BCBFA0F5F70035
:100AE00000F1F850614601F08FFE03980F9920F055
:100AF0007F400390081A20F07F42002F18BF322653
:100B000004D19DF84C00002818BF0226B4F1807F64
:100B100008D00F98001B0002C11700EB11600012F3
:100B2000012802DA042118980BE047B1B34890F885
:100B30002D0020B19DF84C00061C18BF022620464F
:100B40000121B9F1000F02D0159B1E2B02DA9DF88E
:100B50004C3013B14FF0010B491E8B19A8499DF879
:100B60004DE0097815910F99891A21F07F4CACEB73
:100B700000010902CE1701EB16610912994218DB38
:100B8000002A18BFCDF83CC00F9E0597002701F042
:100B900091FF301A0002C11700EB116000123E28CD
:100BA0003FDA012D20D0701E059920F07F4019B347
:100BB0002DE082B1BEF1000F04BF159903290AD0C0
:100BC00027B99DF84C10002918BF9B1E00228DF8F4
:100BD0004C209046C7E707BB9DF84C10E9B10021B7
:100BE0008DF84C109B1EBEE7B4F1807F20D140F6FB
:100BF0000D11702002F04EFEB4F1807F07D0211A53
:100C00000902CA1701EB12610912042903DD044627
:100C100001F056FF0CE000290ADD1BB00020BDE802
:100C2000F08F701E20F07F44204601F049FF5746A8
:100C3000B4F1807F28D00F98DDF840C0001B8BF006
:100C40000103744A20F07F40ACEB040C2CF07F4C85
:100C5000834298BFB0F5800FDFD26245DDD32046D6
:100C60000AF0C1FF67490D9A4B1C161AB6EB930F99
:100C700024BFA0EB020CBCEB930F10D3B14208D2FF
:100C8000081A1044461C0AE040F62C21702002F09D
:100C900001FE61452CD2891A0844401C464257483F
:100CA000807F50B3284645464FF0000BD8460128B8
:100CB00005D0022002F04CF9012002F049F9A945C3
:100CC0002CD2A6EB05014FF001034FF003024FF0C9
:100CD000020002F075F8002808BF4FF00108B9F1D2
:100CE000000F35D00123A6EB09010322184623E0AB
:100CF00040F60C31702002F0CDFDC14534BF4046B6
:100D00004846BBF1000F14BF00211E210844B04229
:100D1000C8DB40F63F21702002F0BCFD10D9012352
:100D2000A6EB09010322184602F04AF828B37DB168
:100D3000711B01230322022002F042F8E8B107E010
:100D400055EA090004D040F67711702002F0A2FDA8
:100D5000012303223146002002F032F868B1012558
:100D6000B8F1000F03D014980F908DF84CB0DFF855
:100D7000A880BAF1000F0ED109E0022002F0E8F8D5
:100D8000012002F0E5F81BB00020BDE8F08F1B4801
:100D900090F82D0000B14FB3DFF860A09AF82C0056
:100DA00018B102F0BDFB8AF82CB007B3A4F13200F1
:100DB00020F07F414FF40020C8F8000000230322F8
:100DC000052001F0FDFF68B34FF08044052002F0DC
:100DD0009FF91249C1F81005C1F814451049E012F5
:100DE0000860064C94F82D00F0B35BE01BE01FE0B8
:100DF00008050040140000200C0B00208C0E002081
:100E000016000020FF7F841E0020A10700E05EF88E
:100E10000080841EFFFF3F0008F5014098F001406C
:100E200004F5014035E0DFF8B8A09AF82C0058B37B
:100E30002B4C94F82D0050B14FF40020C8F800005E
:100E4000052002F085F802F0D3FB84F82DB00CAC3D
:100E5000244894E80E10C0F88013C0F88423C0F82A
:100E60008833C0F88CC300E018E010AC94E80E1092
:100E7000C0F89013C0F89423C0F89833C0F89CC30E
:100E80001BB00120BDE8F08F02F066FB8AF82C5001
:100E90008BE740F23E31702002F0FCFC02F09AFB3E
:100EA00084F82D50A6EB0900A0F11901002904DCFB
:100EB00040F66921702002F0EDFC03220123104668
:100EC00001F07EFF38B108488068C0F800B00748DC
:100ED000C0F800B0BBE740F67421702002F0DAFCE5
:100EE0008C0E00200C0B0020140000200805004090
:100EF0002DE9F043064683B008789073CF7A577394
:100F0000887A10730889144650810D460A785F4923
:100F100099464FEA810C4B42ACF101085AB1C043EB
:100F2000D5F8048004F1080288423DDD40F20A61F0
:100F3000702002F0AFFCEE686D686FEA000904F102
:100F4000080206EB0900464504D940F20961702009
:100F500002F0A0FC8945E9DC994528DB8445DCBF2B
:100F600000F5F700A0F1F85005DD0028BCBFA0F5A2
:100F7000F70000F1F850214601F046FC206820F00F
:100F80007F417019401C2160002F08BF7A3003D0C8
:100F9000012F08BF44302DD101F01AFC20F07F4012
:100FA000606003B0BDE8F0830146984204DA40F285
:100FB0000B61702002F06EFC8445DCBFA1F1F4509F
:100FC000A0F5902005DD0028BCBF01F1F45000F52C
:100FD0009020214601F018FC2068002F20F07F416E
:100FE00008F10100216008BF7A3008D0012F08BF46
:100FF000443004D040F2B161702002F04BFC01F0AB
:10100000E7FB20F07F416160608901AA694601F039
:10101000FBFB1F4890F82F10202923D00069401DAA
:1010200020F07F40D4E90021891A2060084420F094
:101030007F4060604B4632462146E868FFF7CCFAB5
:1010400000281CBF03B0BDE8F083D4E90010401AAB
:10105000304426F07F4120F07F40C4E9001003B007
:10106000BDE8F083608906F1090720B102F0AEFB0C
:10107000002808BF3237074841780098814284BF72
:10108000081A074427F07F40CCE700000020A107A2
:101090008C0E00201600002010B5154C94F82F007F
:1010A000202818BF10BD94F82E2004EB820090F881
:1010B0002010202917D0DFF83CC00CEB821303EB83
:1010C00041035B7880F82030012380F8233084F8D6
:1010D0002B3084F82F10022000F0B0F8002084F8A4
:1010E0002A00A07710BD40F28B31702002F0D2FBB5
:1010F0008C0E00200C0E00202DE9F05FDFF8B88088
:1011000098F82E5008EB850090F82140202C08BF5D
:10111000BDE8F09FDFF8A4B0DFF8A4A0AAF54079FD
:101120000AEB8517072617F8140001280ED00428AB
:1011300008BF02260AD005280CBF0326062805D0C2
:1011400040F6D9014FF0700002F0A4FBBBF1000F94
:1011500018BFAFF30080EFF3108072B607EB4401C5
:101160004A7808EB850181F8212091F82220A242DB
:1011700004BF202281F82220B8B12A46214601204E
:1011800000F05CF804EB440109EBC10059F8312090
:1011900040683146904798F82E5008EB850090F84B
:1011A0002140202CBCD1BDE8F09F0648002818BF84
:1011B000AFF3008062B6E0E78C0E00200000000074
:1011C0000C0E00200000000010B5044600680AF074
:1011D0000AFD02466089217A144B0844411C5018CC
:1011E0009A4204D940F20961702002F053FB104A80
:1011F000914204DD40F20A61702002F04BFB0D4A7F
:10120000914204DA40F20B61702002F043FB0A497C
:101210008142DEBF00F5F700A0F1F85010BD0028B4
:10122000BCBFA0F5F70000F1F85010BDFF7F841E91
:101230000020A10700E05EF80080841EDFF854C0A3
:1012400010B500230CEB821C07281ED2DFE800F04B
:10125000050505050404040001230CF81100002B0A
:1012600008BF10BD0C4800EB820292F82200202833
:101270000EBF82F821100CEB4000417020200CEBD7
:101280004103587082F8221010BD4FF41571702080
:1012900002F000FB0C0E00208C0E00202DE9F34F15
:1012A00083B05C48049900EB8100019090F82040E5
:1012B00003982546012818BF022805D04FF42B615A
:1012C0004FF0700002F0E6FA0027202D4AD0514876
:1012D00000910026807F002808BF022601F0EAFB6B
:1012E000DFF838A104EB44010AEBC101DFF82891D3
:1012F0008A68C968121A091A22F07F4221F07F41D8
:10130000964298BFB2F5800F01D2894528D2444A4F
:10131000009902EB811B22460BEB42014C78202CFA
:1013200016D004EB44010AEBC10CDCF80880DCF8B1
:101330000CC0A8EB000828F07F48ACEB000121F0BE
:101340007F41464598BFB8F5800FE4D28945E2D386
:10135000202A05D020210420009BFFF701F9044634
:10136000AC4215D12F48002818BFAFF3008001F020
:10137000A1FB284C94F8301020290DD0E168821C84
:10138000511A0902CA1701EB12610912002903DD83
:1013900005B00020BDE8F08F202D0DD02A4603991E
:1013A000FFF716FB58B3019880F8237084F830508B
:1013B00005B00120BDE8F08F94F82C0018B102F0C0
:1013C000AFF884F82C7094F82D0050B116494FF402
:1013D00000200860052001F0BBFD02F009F984F847
:1013E0002D70042001F0B4FD01F01AFE202084F8D5
:1013F00030000E48806807600D480760D8E72A462D
:1014000020210420049BFFF7ABF805B00020BDE8C5
:10141000F08F00008C0E0020FFFF3F000C0B00201F
:101420000C0E00200000000008F501401400002010
:1014300008050040064910B591F82F20202A1CBF4E
:10144000887710BD40F2EA31702002F023FA0000E4
:101450008C0E00202DE9F04F5B4E814685B096F84A
:101460002F008A4620284DD096F82F0006F10C0454
:1014700000EB4000A6F5607808EBC00720208DF84F
:10148000000096F82E0003AA06EB800001A990F850
:101490002050306902903068484401F0B5F9F8688E
:1014A00001994A4A0844A9F1640191422FD8B968C8
:1014B000411A21F07F41B1F5800F28D220F07F4002
:1014C0006060304684F80CA090F82E00EA46202D8B
:1014D0001CBF3F4901EB801B3CD005EB450008EBEE
:1014E000C0076068BA682146101A0002C21700EBF4
:1014F000126007F1080600121BD4708950B34889A6
:1015000048B127E040F67B31702002F0C3F905B006
:101510000120BDE8F08F2046FFF756FE01F058F994
:101520003168081A0002C11700EB1160001233285D
:1015300010DA8AF80050397D207B814205D8029864
:10154000606005B00220BDE8F08F0BEB45004578E8
:10155000202DC2D1052001F0FBFC1B4C4FF0FF30C9
:10156000A06094F82E309DF800202021202A13BF7F
:10157000052004EB830090F82000FEF7F1FF94F8BB
:101580002E20134901EB821194F82F2001EB420128
:101590004870206848442060012084F82B00607E59
:1015A000012805D12069401E20F07F4001F022FB78
:1015B0009DF80000202803D00648407802F03AFA4F
:1015C00005B00020BDE8F08F8C0E00209C1FA10705
:1015D0000C0E002014000020064810B590F82F10C3
:1015E00020291CBF007E10BD40F67431702002F02F
:1015F00051F900008C0E00200246144B10B508442F
:101600009A4204D940F20961702002F043F9104A6D
:10161000914204DD40F20A61702002F03BF90D4A6C
:10162000914204DA40F20B61702002F033F90A496A
:101630008142DEBF00F5F700A0F1F85010BD002890
:10164000BCBFA0F5F70000F1F85010BDFF7F841E6D
:101650000020A10700E05EF80080841E104A0B1AEB
:1016600002F1010CB3EB9C0F3CBF1846704710B55C
:10167000441AB4EB9C0F3CBF184610BD9A4203D2EB
:10168000101A0844401C10BDA24204D2511A08444A
:10169000401C404210BD40F60C31702002F0FAF8B8
:1016A000FF7F841E074991F83020824204BF4868BA
:1016B000704700EB4000044901EBC0000830FFF721
:1016C00083BD00008C0E00200C0B00200E4910B5CD
:1016D00091F82F00202812D091F82F00A1F5607208
:1016E00000EB400002EBC00091F82F10406801EBC6
:1016F000410152F83120BDE810400421104740F666
:10170000BC01702002F0C6F88C0E0020F8B56D4DBB
:101710006D49012605F56074082873D2DFE800F0F2
:1017200004679DAFCD44B4B994F82C0018B901F00A
:1017300013FF84F82C60E08A10B102F047F888B1FA
:10174000FFF7AAFC84F82960A168B1F1FF3F05D03A
:1017500001230322052001F033FB40B1607E012804
:1017600010D109E04FF40761702002F093F840F6C1
:101770007501702002F08EF82069401E20F07F4035
:1017800001F038FA94F82F0094F82F1000EB400085
:1017900005EBC000406801EB410155F8312001B074
:1017A0000121BDE8F0401047FFF776FC4FF0FF3015
:1017B000A06094F829008DF800009DF8000088B121
:1017C00094F82F0094F82F1000EB400005EBC000B8
:1017D000406801EB410155F8312001B00621BDE818
:1017E000F040104740F68601702002F053F8FFF7F2
:1017F00053FC84F8286001F0E9FF20B194F82C0034
:1018000030B109E059E040F69601702002F042F84C
:1018100001F0A2FE84F82C6094F82D0058B12B49F9
:101820004FF400200860052001F092FB01F0E0FE7B
:10183000002084F82D0094F82F0094F82F1000EB6E
:10184000400005EBC000406801EB410155F8312034
:1018500001B00021BDE8F040104701F02BFCE08A08
:1018600010B101F0B3FF28B119480078032808BF70
:101870006677F8BD40F6A101702002F00BF815481C
:10188000066088680660F8BD0878BDE8F84002F098
:10189000D1B8FFF701FC94F82F0094F82F1000EB5B
:1018A000400005EBC000406801EB410155F83120D4
:1018B00001B00521BDE8F040104740F6B4017020AA
:1018C00001F0E8FF0C0B00201400002008F5014097
:1018D0001600002008050040034810B540780AF0C3
:1018E00082F980B210BD0000160000202DE9F34FF0
:1018F0008246DC488BB00068DB4DC005C00D0ED0C1
:10190000103840B20028B8BF00F00F0000F1E0200E
:10191000ACBF90F8000490F8140D40090DD00C985D
:101920004FF0000B0078002818BF012818D040F2B3
:101930004F714FF0700001F0ADFF95F82F004FF0A0
:10194000010B202807D00C98007848B140F24B7169
:10195000702001F09FFF4FF4E961702001F09AFFC1
:10196000C24C24B1002140F25270AFF30080C04954
:101970000AEB4A0001EBC0004FF00108009024B1CF
:10198000002140F25A70AFF30080B8F1000F09D087
:1019900095F82E604FF0000985F82B90BBF1000FF1
:1019A00007D032E0B348002818BFAFF3008062B61A
:1019B000EEE73746012020EA0706AF48402200EB59
:1019C000871100EB86100AF07CFA24B1002140F266
:1019D000CD50AFF3008005EB870105EB8600096A67
:1019E000016224B1002140F2D150AFF3008024B154
:1019F000002140F26470AFF3008095F82B008DF861
:101A000004009DF804000028B9D124B1002140F25F
:101A10006E70AFF3008001F04DF88046334606AAA1
:101A20000C99FFF765FA24B1002140F27570AFF30D
:101A30000080914906A801EB861717F81A100129B2
:101A400018BF02293CD10699079BA1EB08018B4ADC
:101A500021F07F41A3EB080323F07F43022971D3D8
:101A6000B1F5800F6ED29A426CD34FF0010901ABF1
:101A700005AA3146FEF72CFF00286BD09DF8141004
:101A80009DF8042033468A4268D00520FEF768FDA1
:101A900007EB4A0148709DF81400202803BF05EBAE
:101AA000860080F820A080F8239007EB400018BF44
:101AB00080F801A0324651465FF00300FFF7BEFBFD
:101AC00005EB860090F823008DF804009DF8047063
:101AD00024B1002140F27C70AFF3008068480028F8
:101AE00018BFAFF30080EFF3108872B624B1002165
:101AF00040F28270AFF3008095F82B008DF804005F
:101B00009DF8040000287FF43AAF24B1002140F290
:101B10008A70AFF300800DF1180E00989EE80E1049
:101B200000F10800B9F1000F80E80E1044D024B194
:101B3000002140F29770AFF30080BBF1000F2CD171
:101B400016E0FFE7324651460420FFF777FB4FF0DF
:101B50000109B5E7324651460420AFE7202919BFF5
:101B600007EB4100407805EB860090F820008FE7F6
:101B70009FB195F82F0020280FD124B1002140F209
:101B80009C70AFF3008031460220FFF787FB20B93D
:101B90000C980078F0B301284CD024B1002140F219
:101BA000B970AFF30080BBF1000F18BF01204AD01D
:101BB00085F82B004FF0010924B1002140F2CA70D2
:101BC000AFF30080B8F1000F45D024B1002140F2FE
:101BD000CE70AFF30080B9F1000F11D095F82E0050
:101BE00005EB800090F82100202809D024B10021C5
:101BF00040F2D570AFF300802248407801F01AFF20
:101C000024B1002140F2DA70AFF300800DB04846F5
:101C1000BDE8F08FFFE724B1002140F2A470AFF3DC
:101C2000008095F82E2051460420FFF707FB4FF067
:101C30000109C1E7002C3FF4A2AE002140F2AF70D1
:101C4000AFF300809BE695F82E10012020EA0101F9
:101C500085F82E10ACE70748002818BFAFF30080C6
:101C600062B6B2E704ED00E08C0E00200000000038
:101C70000C0B0020000000000C0E0020FFFF3F00B6
:101C800000000000140000202DE9F14FA5488CB0A1
:101C90000068C005C00D11D0103840B20028B8BF90
:101CA00000F00F0000F1E020ACBF90F8000490F8C5
:101CB000140D400908BF4FF0010901D04FF0000991
:101CC0000C98007800284FF000001CBF0DB0BDE854
:101CD000F08FDFF854A2954D954C4FF0000B0B9010
:101CE00025B100214FF4CB60AFF3008094F82E6053
:101CF00084F82BB04FF0000825B1002140F25D6060
:101D0000AFF30080B9F1000F1DD13746012020EA62
:101D100007068848402200EB871100EB86100AF086
:101D2000D0F825B1002140F2CD50AFF3008004EB94
:101D3000870104EB8600096A016225B1002140F2A7
:101D4000D150AFF3008025B1002140F26560AFF3C0
:101D5000008000F0AFFE074633466A460C99FFF755
:101D6000C7F825B1002140F26B60AFF3008094F812
:101D70002F00202814D020690099091A0902CA17D7
:101D800001EB126109120BD5DDE90021891A20F05F
:101D90007F42084420F07F40CDE900204FF0010849
:101DA0004DB1002140F27560AFF30080002140F298
:101DB0007B60AFF3008000980199C01BC91B20F025
:101DC0007F4021F07F41B0F5800F05D28A4503D3D3
:101DD000B9F1000F0CD103E0B9F1000F38D094E055
:101DE00033463A4669465448FEF7F6FB48EA00088F
:101DF000B8F1000F22D0009809F0F5FEBDF80A10E6
:101E00009DF808204D4B1144491C4218984241D876
:101E1000494881425ADC404281425FDB581C904273
:101E2000DCBF02F5F702A2F1F85205DD002ABCBFC3
:101E3000A2F5F70202F1F8520C98C26001200B9053
:101E4000002D62D0002140F28E60AFF300805CE094
:101E5000BDF80A0008AA07A900F0D6FC94F82F00E4
:101E600020281CD02069401D20F07F40DDE90021A2
:101E7000891A014421F07F41CDE9000109F0B3FE48
:101E8000BDF80A109DF808202C4B11444A1C8118FB
:101E9000984218D940F20961702001F0FBFCBDF8AE
:101EA0000A0007F1090620B101F090FC002808BFE4
:101EB0003236234841780798814284BF081A064485
:101EC00026F07F40D2E71C48824204DD40F20A61DE
:101ED000702001F0DFFC1B48824204DA40F20B6103
:101EE000702001F0D7FC18488842DCBF01F5F701EB
:101EF000A1F1F85105DD0029BCBFA1F5F70101F101
:101F0000F8510C98C16001200B9094F82B008DF8CB
:101F100010009DF8100000287FF4E2AE0B980DB081
:101F2000BDE8F08F04ED00E0FFFF3F00000000007F
:101F30008C0E00200C0E00200020A107FF7F841EC5
:101F40001600002000E05EF80080841E2DE9F14FAD
:101F5000884D8CB095F82E00002009900120864C09
:101F60004FF00009A5F180078046089024B10021B8
:101F700040F2E970AFF300800898002837D000BF26
:101F800085F82B9024B1002140F2EE70AFF3008071
:101F900095F82EA0402228EA0A0607EB861007EBE8
:101FA0008A11834609F08DFF24B1002140F2CD5003
:101FB000AFF3008005EB860005EB8A010090096A0B
:101FC000016224B1002140F2D150AFF3008095F8B6
:101FD0002B008DF808009DF8080078B1002C1CBF7C
:101FE000002140F2F470C1D0AFF30080BEE7634837
:101FF000002818BFAFF3008062B6C1E724B100210A
:102000004FF4FF60AFF300800C981BF8100003281A
:1020100072D1DDF800A0CDF818A00C999AF8200034
:10202000884214BF4FF0000B4FF0010B0AF1200C57
:102030008646202207EB861303E0024603EB4200AC
:102040004078884202D020280AD0F6E7202807D01E
:10205000864507D103EB4E0040788CF8000007E07E
:1020600048460CE003EB400003EB42014078487027
:1020700024B1002140F23750AFF30080404610EA0F
:102080000B0F18BF8AF82380002852D024B10021FA
:1020900040F2FD70AFF30080324601200C99FFF74B
:1020A000CDF8069890F823008DF808009DF808A058
:1020B00024B1002140F60800AFF30080304800282A
:1020C00018BFAFF30080EFF3108072B6089024B110
:1020D000002140F60D00AFF3008095F82B008DF83D
:1020E00008009DF8080040B1002C1CBF002140F6FC
:1020F00011003FF43BAF77E71BE0BAF1000F08D0C7
:1021000095F82F00202804D131460220FFF7C6F8A9
:1021100008B324B1002140F62500AFF3008095F804
:102120002E0028EA000085F82E0085F82B8001207B
:10213000099024B1002140F62E00AFF300800898EA
:1021400088B124B1002140F63200AFF30080099835
:102150000DB0BDE8F08F002CF1D000214FF40260EB
:10216000AFF30080E6E70548002818BFAFF3008012
:1021700062B6E6E78C0E00200000000000000000C0
:1021800000000000202824BF0020704700EB400022
:10219000034B43F8301003EBC0004260012070474E
:1021A0000C0B002010B5202811D20E4991F82E30CA
:1021B000A1F1800202EB831C1CF810303BB191F8B6
:1021C0002E3002EB831212F81020012A01D00020D9
:1021D00010BD91F82E2001460020FFF72FF80120B6
:1021E00010BD00008C0E00202DE9F84F804E804677
:1021F00096F82E00A6F1800707EB801010F8180063
:10220000002868D096F82E907A4D25B1002140F62E
:10221000C130AFF3008007EB891414F818000128CF
:1022200018D0C0B204281CBF0528062858D02DB1EC
:102230004FF0000140F6CD30AFF3008001F050FCCC
:1022400025B1002140F6D130AFF3008014F818001A
:102250000128E6D1012425B1002140F6D830AFF3A2
:102260000080002C42D0002086F82B0025B10021F0
:1022700040F6DD30AFF3008096F82EB0012020EA62
:102280000B0907EB8B1107EB8910402209F019FEAF
:1022900025B1002140F2CD50AFF3008006EB8B005A
:1022A00006EB890A006ACAF8200025B1002140F235
:1022B000D150AFF3008096F82B008DF800009DF808
:1022C0000000D0B1002D1CBF002140F6E330C2D089
:1022D000AFF30080BFE740F6B831702001F0DAFAC2
:1022E0004A4641460120FEF7A9FFA9E742480028D7
:1022F00018BFAFF3008062B6B5E725B1002140F604
:10230000E730AFF300809AF821200AF1210114464A
:102310004FF0200B07EB89100AF1220A03E0A346D5
:1023200000EB4B035C78444502D0202C2BD0F6E721
:10233000202C28D0A24204D100EB42004078087043
:1023400005E000EB440100EB4B0049784170BAF125
:10235000000F11D025B1002140F22F50AFF30080C3
:102360009AF80000A04207D125B1002140F2325076
:10237000AFF300808AF800B05DB1002140F2375021
:10238000AFF3008000E025B1002140F6EB30AFF361
:1023900000801A48002818BFAFF30080EFF31084C4
:1023A00072B696F82B008DF800009DF8000038B149
:1023B000002D1CBF002140F6F1303FF44CAF87E701
:1023C00086F82E90012086F82B0054B1002D08BF0E
:1023D000BDE8F88F002140F6FE30AFF30080BDE885
:1023E000F88F0548002818BFAFF3008062B6EDE70C
:1023F0008C0E002000000000000000000000000023
:1024000070B50D46064601F0CFF90F4890F82E2022
:102410000024803800EB821010F8141029B1611CE0
:10242000CCB2202CF8D3202070BD084804EB440126
:1024300040F8316000EBC100214645600120FEF705
:10244000FDFE204670BD00008C0E00200C0B00200D
:102450002DE9F04F83B000F02DFB054600F0E0FDC4
:10246000674CA068B0F1FF3F1CBF4FF0FF30A06089
:10247000A07FDFF890B1A8B9D4E90301081A0002DF
:10248000C11700EB116000124FF40C7109F0D8FB7A
:1024900021690844281A0002C11700EB11600012DC
:1024A000C00F13D0607E28B394F829008DF8000087
:1024B0009DF80000F0B100F009FC00BF94F82A007C
:1024C000F0B140F24741702001F0E4F994F82F0098
:1024D00094F82F1000EB40000BEBC000406801EBBC
:1024E00041015BF83120082190474FF4866170204C
:1024F00001F0D0F9E81C20F07F4000F0E1FADDE7C0
:102500004FF0010A84F82AA094F82F00202824D044
:1025100094F82F80202084F82F0084F830000026C3
:1025200084F8286084F829603748266000780228FB
:1025300016BF032801200020207794F82E7004EBAA
:10254000870999F82000202831D000EB40000BEBE0
:10255000C000817D012905D029E040F24A41702068
:1025600001F098F9AB4600F10805408A01AA6946D6
:1025700000F04AF994F82F00202804D02069401D6B
:1025800020F07F400BE068890BF1090B28B101F0C6
:102590001DF9002808BF0BF1320B2BF07F40D5E965
:1025A0000021891A2860084420F07F40686039467D
:1025B0000120FEF773FE0028F9D0144800EB8710C5
:1025C00010F81800022804D13A4641460620FEF7CA
:1025D00035FE84F82BA099F82100202803D00C4860
:1025E000407801F027FA207F002804BF03B0BDE83F
:1025F000F08F00F05FFD2677667703B0BDE8F08FBF
:102600008C0E00200C0B0020160000200C0E002069
:102610001400002010B5324C82B094F82F102029FD
:1026200008D0A168B1F1FF3F09D040F6E921702040
:1026300001F030F940F6E821702001F02BF96268D2
:102640000146284B50189A4204D940F20961702083
:1026500001F020F9244A914204DD40F20A61702021
:1026600001F018F9214A914204DA40F20B6170201E
:1026700001F010F91E498142DCBF00F5F700A0F11E
:10268000F85005DD0028BCBFA0F5F70000F1F850B8
:1026900001AA694600F0B8F89DF804000F288CBF25
:1026A000012000200099084420F07F41A16094F8A7
:1026B00029008DF800009DF80000002804BF02B03A
:1026C00010BD01230322052000F07AFB00281CBF67
:1026D00002B010BD40F6F121702001F0DBF80000DF
:1026E0008C0E0020FF7F841E0020A10700E05EF812
:1026F0000080841E70B51E4C202184F8201084F8C0
:10270000211084F82210002084F8230084F82E0081
:1027100084F82F10421EA2602060A07784F8280061
:1027200084F829002077607784F83010114984F804
:102730002C0084F82D00087048704880A4F18201B4
:102740001022887001F8040F521EFAD10A4D01269A
:1027500084F82A60FF202870084801F04DF968705D
:1027600001F0A8F9A86000F0EDFC84F8316070BDBC
:102770008C0E00201600002014000020F91000002C
:1027800070B504461546084609F02DFA0F4A011B9C
:10279000531CB1EB930F24BFA4EB000CBCEB930FC5
:1027A0000BD38A4203D2111B0844411C05E0624549
:1027B00007D2101A2044401C414201F10F00281A90
:1027C00070BD40F60C31702001F064F8FF7F841E6C
:1027D000410B48F2376251430A0C094B510202FB8C
:1027E00003020848504300F586306E30400D5B42CE
:1027F00010FB03F3B2EB532F88BF491C084470470A
:10280000F7C2FFFF6F0C0100430B48F2376C03FB6C
:102810000CF330B41B0CDFF844C05C0203FB0C0368
:102820000F4858434FEA505C04EB0C0043F6095440
:102830001CFB04F404F5807C43F60855A3EB5C2CE8
:102840002C440CF0FF0CB3EB542F84BF4FF0000C62
:10285000401C086082F800C030BC7047F7C2FFFF20
:102860006F0C01002DE9F041384CD4F80403DFF877
:10287000E08010F4803F4FF400664FF0E0274FF007
:1028800000051CBFD4F84001002817D0C4F84051FF
:10289000C7F880622F480068D8F80010A0EB01004C
:1028A00020F07F40022802D3B0F5800F06D34FF40A
:1028B0008030C4F808030420FEF728FFD4F804038E
:1028C00010F4003F1CBFD4F84401002817D0C4F80E
:1028D0004451C7F8806220480068D8F80010A0EB87
:1028E000010020F07F40022802D3B0F5800F06D30C
:1028F0004FF40030C4F808030520FEF707FFD4F8B2
:10290000040310F4802F1ABFD4F848010028BDE852
:10291000F081C4F84851C7F8806210480068D8F8C0
:102920000010A0EB010020F07F40022804D3B0F596
:10293000800F38BFBDE8F0814FF48020C4F8080351
:10294000BDE8F0410620FEF7E1BE000000B0004007
:1029500004B5004040B5004044B5004048B50040D3
:102960002DE9F0413A4D287804286CD0E81C01226A
:10297000017859B1012908BF6A7002D0697800292D
:102980005CD002210170407800F0E2FA314CD4F8BA
:1029900004034FF0000810F4002F4FF480764FF03E
:1029A000E0271CBFD4F84C01002808D04FF00300EA
:1029B00000F0CEFAC7F880620320FEF7A7FED4F835
:1029C000040310F4802F1CBFD4F84801002808D05D
:1029D0004FF0020000F0BCFAC7F880620220FEF758
:1029E00095FED4F8040310F4003F1CBFD4F8440152
:1029F000002808D04FF0010000F0AAFAC7F8806262
:102A00000120FEF783FED4F8040310F4803F1ABFC0
:102A1000D4F840010028BDE8F0814FF0000000F03C
:102A200097FAC7F8806204202870C5F80880C4F8B7
:102A30000082BDE8F0410020FEF768BE4FF45A71F5
:102A40006C2000F027FFBDE8F0410720FEF75EBED6
:102A50002000002000800040012213024FF0E021FE
:102A60000020C1F8803101F5C071BFF34F8FBFF373
:102A70006F8FC1F800310C494A60431EC1F808331A
:102A80000A4B1860C1F840011B1D1860C1F84401D1
:102A90001B1D1860C1F848011B1D1860C1F84C01CE
:102AA0000A6103494870704700800040408500403B
:102AB00020000020014800687047000004B5004075
:102AC0002DE9F05F414E0446F71E96F800C0F86805
:102AD000BCF1010F04BFA042BDE8F09F4FF04041A0
:102AE0003B4A11603B496FF48023C1F808333A4AEE
:102AF0004FF00005BCF1000F57D06FF4A023C1F8D0
:102B000048331560C1F84451D1F848214FF0E0290D
:102B10004FF00108002A04BF4FF40062C9F8802278
:102B20004FF48033C1F80833C1F84833C1F840513D
:102B30002A4AD2F800A0A4EB0A0A2AF07F4BBBF184
:102B4000020F3CD34FF0020ABBF5800F37D2C1F819
:102B50004045C1F84433BCF1000F05D01168411A5B
:102B600021F07F410229F9D3C7F808803D70FFF7B3
:102B700073FF1B480560001DC0F800A01949042020
:102B800008601949C1F80C80BA68C1F800228101B7
:102B9000C9F88012C9F80011144A41071160FC609D
:102BA000707086F80080BDE8F09FC1F84833104B84
:102BB0001D60C1F840511560C1F84451A4E7C1F847
:102BC000405540F2F1116C2000F064FE230000201B
:102BD00008F5014000B0004044B5004004B5004095
:102BE00004850040108500400080004004F501404D
:102BF00040B500402DE9F0412B4CE168814214BF03
:102C000001220022DFF8A4C09CF80070022F02D03D
:102C1000002A38D003E0002A08BFBDE8F0816278BE
:102C200082B3234B4FF080421A60224B9513C3F8B6
:102C30000853C3F848530026C3F840611E4AD2F82F
:102C40000080A0EB080828F07F48B8F1020F24D3D9
:102C5000B8F5800F21D2C3F84005C3F844532FB113
:102C60001368CB1A23F07F43022BF9D3134B0221B5
:102C70004A071A60E06004208CF801008CF800100C
:102C8000BDE8F08104E040F2FF116C2000F002FE8C
:102C900040F203216C2000F0FDFDC3F8406540F2D6
:102CA0000F216C2000F0F6FD200000202300002002
:102CB00008F5014000B0004004B5004004F50140B3
:102CC0000148C06870470000200000202DE9F04155
:102CD00033486FF48024C0F80843DFF8C8C0324A94
:102CE00000219CF8003063B16FF4A024C0F8484381
:102CF0001160C0F8441100BFD0F84801012280B92A
:102D000009E0C0F84843294C2160C0F84011116027
:102D1000C0F84411F0E74FF0E0244FF40060C4F82D
:102D20008002022B04D040F21B216C2000F0B2FD87
:102D30001F4E30681F4CC01C20F07F40E3681E4DC2
:102D400098420BD03768DF1B27F07F47042F05D34D
:102D5000B7F5800F02D2FFF7B3FE1BE03068181AF8
:102D600020F07F40022813D3B0F5800F10D2134B10
:102D70004FF080401860A26021706A60EA604000F5
:102D8000191F086004208CF801008CF8002001E075
:102D9000A2602170A068C5F80002BDE8F0810000C3
:102DA00000B000402300002044B5004040B5004082
:102DB00004B50040200000200080004008F50140DC
:102DC0002DE9F047DFF874C101274FF000089CF8A7
:102DD00000509CF801C007287ED2DFE800F0040410
:102DE00004046A6A6A00564CE668B6F1807F04BF44
:102DF0006478002C02D0022D05D03CE040F24E2138
:102E00006C2000F047FD4FEA8C0404F18046ACF1E1
:102E100004042406A40D04F1804906F5004609F5D2
:102E200030490024012D02D0022D11D020E0BCF148
:102E3000040F05D2D6F840A1BAF1000F18D104E072
:102E4000D9F840A1BAF1000F12D14FF000440FE0C1
:102E5000BCF1040F05D2D6F840A1BAF1000F07D19A
:102E600004E0D9F840A1BAF1000F01D144F0804448
:102E700014F0804FD5D1334C00F1100C07FA0CFC44
:102E8000C4F808C38000204452B10764D0F84065FC
:102E90008D1B25F07F45AA4298BFB5F5800F43D220
:102EA000C0F84015012B08BFC4F804C30120BDE8D9
:102EB000F08735B1844504D140F271216C2000F0D7
:102EC000E9FC001FC0B2012B0CBF01240024032821
:102ED00006D340F24B1100E02BE06C2000F0DAFC4E
:102EE000DFF864C000F1100307FA03F3CCF80833ED
:102EF000CCF8483380006044C0F840814AB1134D9B
:102F00002E688D1B25F07F45AA4298BFB5F5800F2E
:102F10000AD2C0F84015002C18BFCCF80433CCF806
:102F200044330120BDE8F087C0F840850020BDE8AB
:102F3000F08740F276216C2000F0ACFC23000020EA
:102F4000200000200080004000B0004004B5004098
:102F5000F8B50127002407284CD2DFE800F004046C
:102F6000040416161600264A00F1100107FA01F1B2
:102F7000C2F8081381001144C1F84045C1F840412E
:102F8000204951F820000090F8BD1F4D011FCEB21E
:102F9000297879B16A7882420CD11C4A4FF04040BE
:102FA0001060012908BFFFF757FD2C7018494FF03A
:102FB0008070C86006F1100007FA00F11548C0F8EB
:102FC0000813C0F84813B00000F1804000F530400D
:102FD000D0F84015104A1268891A21F07F41022961
:102FE00024BFC0F84045C0F840410C4850F82600C6
:102FF0000090F8BD40F2EF216C2000F04BFC000087
:1030000000800040408100402300002008F501407E
:103010002000002000B0004004B5004040B1004056
:103020001E496FF48023C1F808331D481D4A90F8EB
:1030300000C00020BCF1000F0AD06FF4A023C1F83B
:1030400048331060C1F84401D1F8481181B909E052
:10305000C1F84833144B1860C1F840011060C1F842
:103060004401F1E74FF0E0224FF40061C2F8801212
:103070000E494FF0FF32C1F808230D4A1060C1F825
:103080004001121D1060C1F84401121D1060C1F80A
:103090004801121D1060C1F84C01704700B000409B
:1030A0002300002044B5004040B5004000800040AF
:1030B00040850040084890F902000028B8BF7047DA
:1030C00000F01F01012202FA01F14009800000F125
:1030D000E020C0F8001270472000002010B507283B
:1030E0000DD2DFE800F004040404060606000649D9
:1030F00002E0001F0549C0B201EB800010BD40F2A4
:103100009A216C2000F0C6FB4081004040B1004095
:1031100010B507280DD2DFE800F004040404060609
:103120000600064902E0001F0549C0B201EB80001D
:1031300010BD40F29A216C2000F0ACFB40810040B1
:1031400040B1004070B51948002404210470C01E2D
:1031500001708905C160FFF77FFC01254FF0E02C6D
:10316000EB02CCF88031BFF34F8FBFF36F8FCCF8F9
:1031700080320F4A556095600E4801680029FCD1E5
:10318000481EC2F80803C2F848030B480460C2F89E
:103190004041001D0460C2F84441001D0460C2F8B3
:1031A0004841CCF80031156070BD000023000020BC
:1031B00000B0004004B5004040B500402DE9F041AA
:1031C000164C607A002827D04FF480718D05284670
:1031D00008F05AFD80464FF48271284608F054FDED
:1031E00000260746B8F1000F09D00120C5F80803F2
:1031F000207920B12671E06908B18047E66137B1D6
:10320000C5F804610220C5F8080300F08BFA4046B7
:10321000BDE8F04100F05AB8BDE8F0813000002070
:1032200010B508F0DBFD30B908F0F9FD18B908F069
:103230002CFE002802D002490220086010BD0000C8
:10324000340C004070B500F087F900F0BFFA094C6B
:103250004FF0804530B1FFF7E3FF012028610420E3
:10326000A07204E00320A0720120C5F8040300202E
:10327000E07170BD3000002070B5134CA079F0B142
:10328000012803D0E179401E814218DA00F09EFA4D
:10329000054600F06FFBA179012902D9E179491CAB
:1032A000E1710DB1616900E02169411A022902DA78
:1032B00011F1020F07DC0DB1606100E02061BDE893
:1032C0007040FFF7BFBF70BD300000202DE9F04710
:1032D00006464FF080454FF48671284608F0D4FC2E
:1032E00080464FF48871284608F0CEFC274C824671
:1032F000277804F1080008F03BFD10B14FF4D571B8
:1033000016E04FF0010946B1A07A032805D1042048
:10331000A072FFF785FFC5F810900026B8F1000FE6
:1033200018D0C5F80C61A07A042804D04FF4DE71DF
:103330006D2000F0AFFA08F051FD28B908F06FFDDC
:1033400010B908F0A2FD08B1114806600220A07271
:1033500000F0E6F8BAF1000F08D0C5F81061A07AC5
:10336000022801D1FFF788FFC5F814903FB12670FD
:10337000A07A022801D1FFF765FF00F0D1F8BDE87F
:10338000F0470248083008F00ABD00003000002075
:10339000340C00402DE9F0475C4C4FF00008064625
:1033A000C4F81880437882780078E072637101274E
:1033B000A271BD0784F80780052824D2DFE800F059
:1033C0000F03051F2100A76109E000F0C5F80121E6
:1033D000284608F05EFC0028F9D00220A06108F021
:1033E00084FCB0B100F00CFA217E01F003018842A8
:1033F0000FD1B07950B10220C5F804036AE0444807
:10340000ECE74448EAE74FF44C7149E000F0CCF9AE
:1034100060E0EF604FF4827AC5F80481A069C5F8D6
:10342000180508F0C7FC40B908F0CEFC28B908F030
:10343000E2FC10B908F0F3FC38B14FF08051364887
:10344000D1F84412C1F34231016008F0B3FC40B935
:1034500008F0BAFC28B908F0CEFC10B908F0DFFC7F
:1034600010B12D4810300760AF600220C5F804038A
:10347000B07978BBD5F8040310F0020F0ED0DFF856
:103480009C90D9F80010C94341F30017D9F80010F7
:1034900041F01001C9F800107F1C07E040F2F12153
:1034A0006D2000F0F7F900BF00F01AFB51462846E6
:1034B00008F0EAFB0028F7D000F076F92FB9D9F828
:1034C000001021F01001C9F800100220C5F808030F
:1034D000C5F80481A07970B1307860B900F076F950
:1034E000064600F047FA6FF0004216B1C4E9042026
:1034F00001E0C4E904020121284608F0CAFB08B132
:1035000000F05EF984F80A80BDE8F0873000002002
:1035100001000200010003003C05004010ED00E046
:1035200010B5EFF3108472B60A48417829B141789A
:10353000491E4170417829B108E040F20D116D201B
:1035400000F0A8F9807808B900F04EF9002C00D1FD
:1035500062B610BD3000002010B5EFF3108472B6D3
:1035600006484178491C41704078012801D108F093
:10357000A7FB002C00D162B610BD00003000002077
:10358000054810B5C17821B100210171C170FFF764
:10359000C7FF002010BD00003000002070B50C4CAB
:1035A000E17861B90125E570E061FFF7D5FF00F032
:1035B0000DF930B1E06910B180470020E0610020D2
:1035C00070BD4FF080402571C0F80453F7E700004C
:1035D00030000020EFF3108072B604498A78521C44
:1035E0008A70002800D162B67047000030000020C9
:1035F00010B5EFF3108472B60A48817829B181784A
:10360000491E8170417829B108E040F225116D20F2
:1036100000F040F9807808B900F0E6F8002C00D1FD
:1036200062B610BD300000202DE9F04104006FF0BB
:1036300015003CD02178042939D80029617838D088
:10364000002934D1A178002931D1002008F0E7FA0F
:10365000002008F0D7FA4FF080484FF0FF31C8F84B
:1036600008130026C8F80061C8F80461C8F80C61A6
:10367000C8F81061144F7E70A088B88108F017FB5D
:10368000012508B1FD707D700121404608F001FB65
:1036900008B100F095F82046FFF77CFE7D7200200F
:1036A00008F0B0FA4FF0E0213046C1F80051BDE813
:1036B000F0810029FBD02029F9D8A1782129F6D85A
:1036C0000129C2D1F3E700003000002001488089C1
:1036D000704700003000002010B50D4808F048FB8E
:1036E0000B49083948B1012008704FF0E021C1F8BA
:1036F0000002BDE81040FFF72FBF887A022801D1F1
:10370000FFF7A0FDBDE81040014808F048BB0000ED
:10371000380000200248807A002800D0012070473D
:1037200030000020F8B51F4DE87A00280FD1287E20
:1037300000F0030008F0C9FA002808D0EFF3108168
:1037400072B6FFF7E7FF18B1002900D162B6F8BDE5
:103750000126AE7201B962B618204FF08044C4F859
:103760000803A6614FF42070ADF80000BDF800001A
:10377000411EADF80010F9D20027C4F80C71C4F84E
:1037800010710848083008F006FB2F70FFF75AFD4B
:103790006661687900F07F00C4F838051820C4F825
:1037A0000403F8BD3000002010B5044C207E00F06A
:1037B000030008F08AFA0028F8D010BD300000207D
:1037C0000149012008707047880200204FF08040B6
:1037D000D0F8000118B903480078002800D0012073
:1037E00070470000880200204FF0804001214160B6
:1037F0000021C0F8001101480170704788020020C4
:103800000248006800F00300704700001C040040FC
:1038100010B531B1012907D040F2023105A000F006
:103820000FF8D0F8140401E0D0F8080400F001000B
:1038300010BD00006E72665F636C6F636B2E680074
:10384000024A526802B11047FEE700005000002013
:10385000064810B50021016001210160084608F00A
:103860005BFABDE81040012008F049BAFC1F004097
:10387000074810B501214160891EC0F808130C20CB
:1038800008F04AFABDE810400C2008F038BA0000F1
:1038900000C00040FEB5104A5568E5B1002203465D
:1038A0006E460A2403E0B0FBF4F0521CD2B20028AA
:1038B000F9D1B0540AE000BFB3FBF4F004FB1030C0
:1038C000B3FBF4F3521ED2B23030B054002AF3D11D
:1038D0003046A847FEBDFEE75000002070B5174CEB
:1038E00006460D46607810B14FF0FF3070BD06B946
:1038F000134E62602570FFF7ABFFFFF7B9FF30464C
:10390000FFF792FE0600F1D1FEF7F4FEFFF70AFF83
:1039100008F0D0F8284608F0F2F90120002D09DB64
:1039200005F01F0100FA01F16A09920002F1E0229C
:10393000C2F800116070304670BD000050000020D9
:103940003ABD000001484078704700005000002058
:10395000074890F90000002809DB00F01F02012150
:1039600091404009800000F1E020C0F8001270474B
:10397000500000202DE9F04101264FF0E0223103F4
:103980004FF000084046C2F88011BFF34F8FBFF3DD
:103990006F8F164CC4F800010C2008F0DCF9144DB0
:1039A0002868C04340F30017286840F010002860E2
:1039B000C4F8046326607F1C02E000BF00F090F8AA
:1039C000D4F800010028F9D01FB9286820F01000B1
:1039D0002860084805686660C4F80863C4F8008178
:1039E0000C2008F0B8F92846BDE8F08100C000407E
:1039F00010ED00E008C5004010B5024605200C4956
:103A000004E000BF01EBC0031B7933B1401EC0B21C
:103A1000F8D24B216920FFF73DFF41F8302001EB40
:103A2000C00100224A718A7101220A7110BD000092
:103A3000C00E002010B5052801D35A2106E00A491E
:103A400001EBC0000179012903D05B216920FFF758
:103A500021FF41798279491CC9B28A4200D0417163
:103A6000BDE81040FFF774BFC00E002070B50525FB
:103A70000E4E0F4C16E0217806EBC1000279012AA8
:103A800008D1427983799A4204D04279827156F8FA
:103A9000310080472078401CC0B22070052801D337
:103AA000002020706D1EEDB2E5D270BDC00E00206A
:103AB0008902002000B508F07DF940B908F084F9CA
:103AC00028B908F098F910B908F0A9F908B1024826
:103AD00000BD024800BD00000C05004000E70140A9
:103AE00010B508F09CF930B3EFF31080C8B1002195
:103AF00072B6124802680368C2F3001243F0100362
:103B000003604FF0E023D3F80042D3F804321C43A3
:103B100000D040BF20BF00BF00BF00BF00BF12B138
:103B200005E00121E4E7026822F0100202600029AA
:103B300000D062B610BD20BF10BD000010ED00E047
:103B40008FC00000ABC0000099C00000A5C00000FD
:103B500093C000008DC000008BC00000B1C0000009
:103B60009FC0000085C000007DC0000081C0000033
:103B700077C0000001480068006800475800002036
:103B8000014800680069004758000020014A126897
:103B9000926810475800002001480068C06800473C
:103BA00058000020014A126852681047580000204F
:103BB00001490968096A084758000020014800784F
:103BC000704700008A0200201FB5174C207A022897
:103BD00000D202208DF80100E079032800D20320F2
:103BE0008DF80000A079ADF804006079ADF802000E
:103BF000684606F05BF908B1802110E0E0680290A9
:103C000002A806F069F908B1842108E007480068B5
:103C1000039003A80BF0ADFA002803D088210320FD
:103C200000F0E0F81FBD0000E80E0020CC3E0000D0
:103C300010B528B11422044908F043F9002010BD42
:103C40006FF0150010BD0000E83E000070B56FF089
:103C50002C0378BB274C607808B1981170BD01B374
:103C60006FF015053AB324480B293DD2DFE801F087
:103C70003C06090C10131A2416272D001178017028
:103C800027E01178417024E01168C0F8051020E0A9
:103C90001168C1601DE0117881701AE0117849B98E
:103CA000C17016E0E17811B1117802291CD31178A6
:103CB00001740EE005E017E01188418209E01178F7
:103CC00009B1184670BD017103E0117802290BD3C8
:103CD000017501220849002008F0ECF9B0F5803F99
:103CE00004DB6FF00B0070BD284670BD0121A17090
:103CF00070BD00005C000020E80E002070B50C468E
:103D0000050019D0C4B100F023F9C0B12846FFF76F
:103D100073FE0C4D00220C492870204608F0CAF9A9
:103D20000BF091FE0021287806F030FBFFF74CFFE6
:103D300001206870002070BD6FF0150070BD4FF05D
:103D4000FF3070BD5C000020E80E002030B587B069
:103D500005000CD0FFF7F6FD4FF0FF3420B1FFF760
:103D6000B5FCB0F5FA7F05D9204607B030BD6FF03D
:103D70001500FAE7154C1648656000F0F9F90020C7
:103D80006070A070E07001461822684608F013F9D0
:103D900018221049684608F094F8182269460E481F
:103DA00008F08FF8EFF3108472B60C486FF00C0136
:103DB00000F0ACFD0A4800F06DFE18B1962103201A
:103DC00000F010F804B962B60020CEE75C000020D5
:103DD000C93B0000D03E0000E80E002000C00040BB
:103DE0007D3F00000EB572B6154A5568D5B1002268
:103DF00003466E460A2403E0B0FBF4F0521CD2B234
:103E00000028F9D1B05409E0B3FBF4F004FB103002
:103E1000B3FBF4F3521ED2B23030B054002AF3D1C7
:103E20003046A847BFF34F8F06480168064A01F4A1
:103E3000E06111430160BFF34F8F00BFFDE7000059
:103E40005C0000200CED00E00400FA05064810B507
:103E500081784078014302D04FF0FF3010BD06F06A
:103E6000B5FA002010BD00005C000020064810B527
:103E700081784078014302D04FF0FF3010BD06F04A
:103E800043F8002010BD00005C000020064810B57B
:103E900081784078014302D04FF0FF3010BD0BF025
:103EA00038FB002010BD00005C000020064810B563
:103EB00081784078014302D04FF0FF3010BD06F00A
:103EC00097FA002010BD00005C00002001000000F7
:103ED00001010100001B1B03020000004C1D00003B
:103EE00003001F0000000000DFC04ED61F7C6609E3
:103EF0000AF52BA098F2436462C5A62A054A10B5BC
:103F0000526812B1BDE81040104783210420FFF72A
:103F100069FF0000000F0020054A10B5126812B1B9
:103F2000BDE8104010477D210420FFF75BFF000033
:103F3000000F0020054A10B5926812B1BDE810408C
:103F4000104789210420FFF74DFF0000000F0020DB
:103F50000548016829B1416819B1806808B101209C
:103F60007047002070470000000F002002490DC874
:103F700081E80D0000207047000F0020F8B5124CBA
:103F80000026256811E00098022802D003280CD1F1
:103F900006E0206810B10020266005E028210CE032
:103FA000206868B101202660A847684600F044FDFB
:103FB0000028E8D0052805D035210420FFF712FF9E
:103FC0002D21FAE7F8BD0000640000207CB51F4CED
:103FD0000546207840B1A278611C2846921C07F063
:103FE00070FF0020207021E0194805F0C5FF00286F
:103FF0001DD0174C2078112804D10A213E2008F04A
:10400000FEF818B12078082805D009E010492846A4
:1040100008F0FDFA0AE005213E2008F0F0F838B17A
:104020000B49284608F049F9002800D001207CBD42
:10403000A088ADF8000001A9684608F002FC00283D
:10404000F5D09A210820FFF7CDFE00009E10002039
:104050009C0F002070B50A7882703AB3012A25D8E7
:104060001323037000230AE001EB430400EB430534
:10407000A678EE706488240A5B1C2C71DBB2934234
:10408000F2D300230BE000BF01EB430500EB430438
:104090002E796671AD882D0A5B1CA571DBB2934247
:1040A000F2D3012101EB8200C0B270BD002070BDCF
:1040B00001210C4A40280CD2202803D8401E814000
:1040C000106802E0213881405068014207D1002089
:1040D0007047FF2803D0403881409068F5E7012001
:1040E00070470000680000200121401E8140044804
:1040F000C068014201D001207047002070470000D5
:104100006800002001490068C8607047680000200E
:1041100004490268406842F48C220A60024A104353
:104120004860704768000020F807400201490068B5
:10413000886070476800002005484FF0FF3101603B
:10414000C90C4160002181601F21C16070470000DF
:104150006800002010B5FFF7EFFF0BF04EF90446A2
:104160000248006800B18047204610BD780000205A
:10417000014908607047000078000020022101809A
:10418000418000210171DF21417144F6C061C1808D
:104190000149816000207047D61F7C663EB5044609
:1041A000694608F0ACFE70B140F25A2108E000BF49
:1041B000BDF80400214600F0ABF820B140F25F21C9
:1041C0001720FFF70FFE684600F052F80028EFD0E6
:1041D0003EBD000010B5022804D34FF4D67117205D
:1041E000FFF700FE0149085C10BD00000C0F002025
:1041F000F8B50500009510D00026087849780446E7
:10420000A14200D90C46EA1C22F00302AA4206D0C1
:1042100040F279111720FFF7E5FD0126EDE7134F76
:10422000387079703146684600F0EEF800210B4690
:104230000098C01C20F0030000906EB907EB8102CB
:10424000D060002006E000BFD2F80CC04CF820304F
:10425000401CC0B2A042F7D30098491C00EB840078
:10426000C9B200900229E3D3401BF8BD0C0F002017
:1042700070B5044608F0B7FF08B1102070BD25786E
:1042800000F0FEF802460C48618800EB85000EE065
:10429000C36853F8213043B14A1C6280A180C068D2
:1042A00050F82100A060002070BD491C89B29142E5
:1042B000EED36180052070BD0C0F00202DE9F04188
:1042C00021B1012902D00020BDE8F0810F4C002768
:1042D0003B464FF6FF7604EB810514F801C00AE077
:1042E000DC19D5F80CE0A4B25EF824E0BEF1000FB2
:1042F00004D05B1C9BB29C45F2D834460480204617
:10430000B442E0D0BDE8F04100F034B80C0F00201A
:104310002DE9F0410646A0F57F400C4643F2020726
:10432000FF3820D0022C02D30720BDE8F0813046B0
:1043300000F05AF8050016D00C48294650F8242001
:10434000304690470A48002100EB8407F86840F89F
:104350002610204600F08AF802462946786808F0C0
:10436000ADFD0020E1E73846DFE70000A044000093
:104370000C0F00202DE9F04190460D46074608F04D
:10438000CFFD48B1164800EB8506F06850F82700CD
:1043900028B14FF49D7115E040F2391112E07068B8
:1043A00000281AD0284600F061F80146706808F02D
:1043B00037FD040010D0F068022D40F8274004D3E8
:1043C00040F245111720FFF70DFD064842462146F1
:1043D00050F82530384698472046BDE8F081000067
:1043E0000C0F00209844000070B50C46054608F0FC
:1043F00097FD002805D0034800EB8400C06850F802
:10440000250070BD0C0F00202DE9F843164E88469C
:10441000054600242868C01C20F0030028602046C0
:1044200000F024F8315D4843B8F1000F01D00022BC
:1044300000E02A680146009232B100274FEA0D00E1
:1044400008F01BFD1FB106E001270020F8E706EB8E
:104450008401009A4A602968641C0844E4B2286018
:10446000022CD7D3BDE8F8830C0F0020034931F8A4
:1044700010004FF6FC71C01C0840704794440000C7
:10448000034908784978884200D2084670470000FE
:104490000C0F00201802D40035CF000035CF0000EB
:1044A000DDE9000055DE00002DE9FF4F264C804677
:1044B00081B020689A46934658B1027A424503D9A2
:1044C000416851F8280040B143F2020005B0BDE850
:1044D000F08FA5211820FFF785FC1946029808F0F7
:1044E00041FD86B258460E9908F033FD85B2701929
:1044F000001D87B22068A1463946006808F090FC8C
:1045000004001FD0678025802946201D0E9D074688
:104510005A460123009508F0E3FB208831463844D1
:104520000123029ACDF800A008F0DAFB2088C11917
:10453000384608F006FCD9F800004168002041F830
:104540002840C3E70420C1E77C00002070B5144C6C
:1045500023688BB1197A814212D95A6852F8201017
:1045600071B1002542F820504A88186808F0A6FC6E
:10457000216800200A7A0CE0C8211820FFF732FCDD
:1045800043F2020070BD4B6853F8203033B9401C31
:10459000C0B28242F7D8086808F085FC002070BDE0
:1045A0007C0000202DE9F0410D46040090464FF0BC
:1045B000000609D00027E01C20F00300A04205D02F
:1045C00086211820FFF70EFC0127F4E7CDB1114634
:1045D000002008F052FC0C3000EB85068FB90A4F22
:1045E00004F10C00AA003C602572606000EB8500BD
:1045F00020600021606807F0DEFC4146386808F062
:104600003CFC3046BDE8F0817C00002070B5084DD0
:10461000286800280AD0002404E02046FFF796FF0F
:10462000641CE4B22868007AA042F6D870BD00008D
:104630007C000020094910B502460968002049B1F4
:104640000B7A934205D9496851F82210002900D00D
:10465000081D10BDEE211820FFF7C4FB7C000020D0
:104660000A4910B502460968002059B10B7A9342F5
:1046700007D9496851F82210002902D031F8040BFB
:10468000084410BDFC211820FFF7ACFB7C00002083
:1046900070B51E4B456804460022A1B10120607030
:1046A000588881085FF0000004EB400304EB8006AB
:1046B0001A83198400FB015373602318401C1A7578
:1046C0000428F1D370BD62705FF0000004EB40017C
:1046D0000A830A8404EB80014A602118401C0A7591
:1046E0000428F3D35888B0F5FF7F01D2460800E0D4
:1046F000FF2608F0AAFC656020842918A160668462
:10470000E560A0842161E68470BD00008000002087
:104710002DE9F04170B100251144CCB2244EC11CEA
:10472000002721F003013470814205D04E21092079
:10473000FFF758FB0125EFE71F2B04D84FF6FF7159
:1047400001EA830109E05900FF2B0BD903F1FF02B5
:10475000B2EB430F00D2114689B2C91C21F003030A
:1047600035B107E07C22B2EB430FF5D37C21F3E7B0
:104770007060738004EB840107EBC102002176684E
:104780004FF0010C0DE04DB901EB810700EB020E7B
:1047900006F837C006EBC707C7F804E0491C1A44FF
:1047A000C9B2A142EFD3D21D22F00700BDE8F081CB
:1047B0008000002070B5104A00205168127814E083
:1047C00000EB800311F833306BB100EB800011EB8C
:1047D000C0040CD00025A57001212046FFF758FF2A
:1047E0002570204670BD401CC0B29042E8D3A9217C
:1047F0000920FFF7F7FA000080000020044810B5F8
:104800004088840808F021FC844200D3204610BD73
:1048100080000020094910B507480860084B1120A6
:1048200003EBC0040022C4F81025C4F81425401C72
:10483000C0B21428F4D310BD0000FEFF08F50140FB
:1048400000F0014070B520240021012320FA01F27C
:10485000D20720D04AB2002A10DB00BF4FEA52161E
:104860004FEA860602F01F0506F1E02603FA05F579
:10487000C6F88051BFF34F8FBFF36F8F0BDB02F091
:104880001F054FEA52124FEA820202F1E02203FAB8
:1048900005F5C2F8805201F10101A142D6D370BDE5
:1048A00070B542004FF0000101D5144A1160C0F309
:1048B0008032C0F3C0339A4203D066211B20FFF739
:1048C00091FA10F4404F14D00D4A01205060831E1D
:1048D000C2F808330B4A9060C2F80012C2F80833DD
:1048E000094C2160251D28609060C2F808332160C2
:1048F0002860BDE87040FFF78DBF000004E501406F
:1049000000E0004000F0004000F5004070B50A4CA7
:104910000D462060FFF7C4FF2068FFF793FF00F00B
:1049200077F8FFF777FF08F053FC284600F0AAF865
:10493000BDE8704000F0C2B8880000202DE9FC5F9F
:104940002F4E83463068019001272E4807F010FA59
:10495000DFF8B08020B9002708F1010007F01FFA46
:10496000294C00254FF0030901206060C4F8005174
:10497000C4F80451C6F800B02060DFF890A017E03A
:10498000DAF80000C00613D50E2008F012FCEFF391
:104990001080009072B6C4F80493D4F8000120B9D6
:1049A000D4F8040108B9FFF79BF8009800B962B683
:1049B000D4F8000118B9D4F804010028E0D0D4F8E4
:1049C00004010028D0D137B10198306008F101000E
:1049D00007F0CEF911E008F1010007F0C9F900284D
:1049E000BAD1C4F80893C4F80451C4F800510E2099
:1049F00008F0DFFB034807F0D2F90020BDE8FC9F78
:104A000004E500408B02002000E0004010ED00E0D3
:104A100010B5084807F0BFF908B1242106E00548A1
:104A2000401C07F0B8F9002803D028211D20FFF70B
:104A3000D9F910BD8B02002070B511490A68EAB19E
:104A400000231D4601244A68521C4A60092A00D3EB
:104A50004D600E7904FA06F20E6816420BD0EFF3A1
:104A6000108372B60C6894430C6003B962B649684F
:104A70000160002070BD5B1C092BE4D3052070BDD4
:104A80008C00002002480021016041607047000056
:104A90008C00002010B5084C617809B10F2010BDC2
:104AA000FEF7AAFF2070FF2801D0002010BD76215C
:104AB0001F20FFF797F90000940000200149002013
:104AC00048707047940000200648074A818C52883D
:104AD000914204D190F8220008B1002070470120D3
:104AE00070470000A0110020780200200149488092
:104AF00070470000780200200848094A818C5288DB
:104B0000914209D14FF6FF71818410F8221F19B12B
:104B1000002101700120704700207047A011002083
:104B200078020020074810F8221F012907D0012130
:104B300001700548034900888884012070470020DF
:104B400070470000A0110020780200200649074BA2
:104B50008A8C5B889A4205D191F8222012B10160BB
:104B60000120704700207047A0110020780200202B
:104B700009498A8CA2F57F43FF3B02D000210160E6
:104B800007E091F822200449012A02D001600120A7
:104B90007047002070470000A011002001490880E4
:104BA00070470000780200200549002081F82200AB
:104BB0004FF6FF70888403490880488070470000E2
:104BC000A01100207802002005498A8C824205D17C
:104BD000002081F822004FF6FF70888470470000A3
:104BE000A01100200A4A10B1012807D00EE0507829
:104BF00060B1D2F802000860D08804E0107828B1D3
:104C00009068086090898880012070470020704774
:104C10008D020020084A012338B1012804D1137005
:104C20000868906088889081704753700868C2F85F
:104C300002008888D08070478D020020064910B19C
:104C4000012802D005E0487800E0087808B101208A
:104C500070470020704700008D0200200149487411
:104C600070470000FA0A00200148C0787047000031
:104C7000B00000200148007970470000B00000201B
:104C800078B513494A7C0AB30A7C8DF80020009A53
:104C900000929DF80020CAB1002301F110021A24ED
:104CA000A1F152050E7C8DF80060009E00969DF8E3
:104CB00000604EB1137043700470D5F85A604660BE
:104CC000D5F85E608660EDE7012078BD002078BDF4
:104CD000FA0A002010B5044600F05CF918B1BD21B5
:104CE0002720FFF77FF80348012108F039FE02482A
:104CF000C46210BDD80A0020B00000200149012084
:104D000088717047B00000202DE9F047624D089C83
:104D10002E78002E6BD1002A69D0002B67D0002C92
:104D200065D005F11406C5E90E0186E81C000027D0
:104D3000AF716F71EF70AF702F71AF81EF8100F0C5
:104D400061F9064600F058F9044606F04BF805F004
:104D5000F3FC94F96E0006F0CFF804F1180006F0A9
:104D6000A5F9206906F098F996F8230006F0B8F93D
:104D700005F13800406890F8740108B105F08CFF27
:104D800094F86B10012005F0B7FE00287CD0434852
:104D900005F02EFF2088FFF763FC28632088FFF7CB
:104DA00049FC06F160016863DFF8F49091E80E10A9
:104DB00009F1080888E80E10316FC9F82110716FE9
:104DC000C9F8251000F090F90146208FBA4608F086
:104DD0005FFBA18E814200D208462872A84694F853
:104DE0006B10E08FF77CA58F082904D102E04FF407
:104DF0008A714DE0042108F04BFB0FB9001D80B211
:104E0000854200D22846C5B288F80950F17C09B124
:104E1000042200E000222A44D2B288F80720B4F825
:104E20005400001D904202D240F29F1130E05746DC
:104E3000A1B11B48012108300176D6E91612C0E95C
:104E4000041294F86B0008F029FA154903462A4623
:104E50000831012005F0BAFC05F0EEFC012000F05D
:104E600073FB10480068032810D00B280ED048466A
:104E700040F8527F47600A48B1885230418021880B
:104E8000018096F823100171BDE8F08740F2C71148
:104E90002720FEF7A7FF0000B00000204C570000BD
:104EA000A80A0020501500402DE9F047054600F003
:104EB000A9F8334E0446706A47780DB1012D03D12D
:104EC000716B07F074F9707070784FF000084FF054
:104ED000010950B101281AD0022834D0032848D043
:104EE00040F214412720FEF77DFF012D32D000F063
:104EF000E7F839460122706B07F07CFD28E000BF1F
:104F000084F8088031E000BF84F808902DE0012D7E
:104F100008D000F0D5F839460022706B07F06AFD22
:104F2000022D0BD0D4E91601401C41F10001C4E967
:104F30001601207A012803D084F80890BDE8F08794
:104F400084F80880FAE7012D04D0706B07F063FF46
:104F5000022DF3D0D4E91601401C41F10001C4E94F
:104F60001601207A0128CFD1CAE7BDE8F04704F046
:104F700003BF012DE2D0706B07F04DFFF5E7000095
:104F8000B00000200248C089C0F3802070470000B4
:104F9000B00000200448007808B10C207047034995
:104FA0000020487470470000B0000020FA0A00207A
:104FB0000C4810B5017849B100F138010078022899
:104FC00008D040F2E3112720FEF70CFFBDE81040A7
:104FD00000F0D8B94868D0F80801BDE8104005F0E5
:104FE0000FBE0000B0000020024A93890343938162
:104FF00052691047B0000020014840687047000027
:10500000E80000200148406870307047E800002048
:10501000014A002152691047B000002070B5FFF727
:10502000F1FF0446FFF7E8FF0546214608F0B3FA12
:1050300095F82610012914D1002812D00948426899
:105040002888A2F8F601607A82F8F801A07A82F83E
:10505000F90102F5FA7201201070BDE8704004F009
:105060008BBE70BDE800002070B50546012918D838
:10507000124CA1698847A0B1607990B9E5B904F1F3
:1050800010000178C80605D4E06A0078C00601D493
:10509000012000E00020A26A2AB962891AB1C9067B
:1050A00001D4012070BDA1898A0703D5226AD27874
:1050B000022A01D00843F4D1002070BDB0000020C6
:1050C00010B5084CA06A38B16289616AD21C06F03A
:1050D000F8FEA06A606210BD40F25A412720FEF738
:1050E00081FE0000B000002010B5FFF785FF0446E8
:1050F000FFF788FF0146427B1548242A0ED0897BA2
:1051000024290BD01F2A0DD0202A0BD022290FD002
:1051100094F86A00042800D1082010BD406890F877
:1051200096110EE0222903D0406890F8B00105E006
:10513000416891F8B00191F86310084008F0A4F8B4
:10514000014694F86A00BDE8104008F0B5B80000C8
:10515000E80000202DE9F84388460746FFF752FF94
:10516000574C002605468DF800602078022804D0B0
:1051700040F2B9412720FEF735FEA07B400606D459
:105180004020FFF745FFE08940F04000E081E87CE7
:10519000C7B305F081FB05F065FB68B9E87C58B141
:1051A000606A417841B10078297AC0F3C000884232
:1051B00002D10120A07063E0606A4178618121B171
:1051C000606B07F0F5FDA06200E0A662E08940F4A4
:1051D0008070E081606AE9790078C0F380008842DD
:1051E00005D000F063F9E08940F48060E081606AF6
:1051F000297A0078C0F3C00088420ED1684600F0DA
:1052000017F90AE0FFE708B105F040FBE078401C21
:10521000E070E08940F40070E081A87C98B1FFF76D
:10522000EBFE28490E76D5E91423C1E9042390F852
:105230006A0008F033F80346FB222249002005F0FB
:10524000C5FA05F0F9FA1F4D4A35B8F1000F04D13F
:10525000E1780120FFF708FFB0B105F0FBFE9DF8F3
:10526000000010B10020FFF71FFE37B1E67068792B
:10527000401C6871FFF7D2FE02E0A879401CA871BB
:1052800000F080F8BDE8F8839DF8000010B101201F
:10529000FFF70AFE002000F095F99DF8000010B11C
:1052A0000220FFF701FE37B1E6706879401C687193
:1052B000FFF7B4FEE6E7A879401CA871E2E700001A
:1052C000B0000020B00A00202DE9F0410F468046D2
:1052D000FFF798FE294D04462878012804D040F2B3
:1052E00069412720FEF77EFD61780020012629B163
:1052F000607000210420FFF777FEE670296A0878C5
:10530000C043800709D1A07988BB0220FFF76CFE5B
:10531000286A0078C043800729D0286A407810B1F5
:105320000220A07100E0A671E07CA0B1FFF764FE4E
:1053300013496D7A0E76D4E91623C1E9042390F857
:105340006B0007F0ABFF03462A460D49012005F02C
:105350003DFA05F071FA37EA080704D00021084643
:10536000FFF782FE28B1BDE8F04100F00BB8032042
:10537000D7E7BDE8F041002000F0E6B8B00000201B
:10538000B00A002010B505F023FB05F0D5F90D4C4F
:10539000E089FFF73DFEE2696179A07890470A480D
:1053A000407C58B10848523850F8521F816041681B
:1053B000C16005480121017404F0DEFC002020706A
:1053C00010BD0000B0000020FA0A0020084810B507
:1053D0000078022804D040F217212720FEF702FDB2
:1053E00004490120C871BDE81040FFF7CBBF0000A1
:1053F000B0000020FA0A002030B40C4B42B9DA7930
:10540000FF2A05D190F86B2090F86A40A2420BD099
:1054100031B1DA7990F86B1030BC104605F04EBE11
:10542000FF2290F86A10F7E730BC7047B000002008
:1054300070B50646FFF7E6FD1B4A04460125516A92
:10544000087800F0030001280CD002280AD00328B5
:1054500021D16570D08940F40060D0810120FFF730
:10546000C3FD18E04878B0B1D18941F40061D18121
:10547000916A002909D0FB2808D8907920B1BDE8AD
:1054800070402020FFF7C4BD357070BD507940F0EA
:105490001000507170BD207A012801D0257270BDB6
:1054A0000020207270BD0000B000002070B5FFF732
:1054B000A9FD0446807900282ED002280DD11C4871
:1054C000006B07F070FA40B3D4E91401401C41F1BD
:1054D0000001C4E9140104F04FFC0025A571E07837
:1054E00020B1E57000211020FFF77EFDA07870B19B
:1054F000A570FFF701FB98B100210820FFF774FDAC
:10550000D4E91401401C41F10001C4E91401E0791F
:1055100001280AD00120E07170BD40F2AF3101E0F6
:1055200040F2C7312720FEF75DFCE57170BD000039
:10553000B000002003480078002801D0FFF722BF08
:1055400070470000B00000202DE9F0410646FFF74B
:1055500053FD8046FFF756FD174C05463246E06A7C
:10556000606201214046FFF747FFE87C002780B1D9
:10557000124805F0C7FC124801210176D5E9161240
:10558000C0E904120D49606A05F0A8F805F0BAF800
:1055900004E0606A05F0B6FC05F0CEF816B93846AE
:1055A00005F052FB002198F86A20084605F034FD0A
:1055B00002202070BDE8F081B0000020A809002082
:1055C000B00A00202DE9FC470446FFF71BFD054605
:1055D000FFF712FD0646DFF8689122460021FFF72B
:1055E0000BFFA87901274FF00008A9F1200440B172
:1055F00001281FD0022830D003283CD04FF42D7151
:1056000058E0207A5021ADF8040088534846FFF74F
:105610009DFA28B18020216AFFF7E6FCAF702EE0EA
:105620006A4601A9206B07F051FE206210B195F87F
:10563000431011B14348206221E09DF8001031B9B8
:10564000A0F8008080F80280012108F089F9BDF8F7
:105650000410206A08F048F911E0B6F85000ADF8DF
:1056600004006A4601A9206B07F030FE206230B9C1
:1056700040F2A5211EE04846FFF768FAC0B1206A53
:105680000823017821F008010170EA7903EAC202D7
:10569000114321F0040101702A7A042303EA8202F3
:1056A000114321F010010170C943890705D007E0BB
:1056B00040F2AE212720FEF795FBC07802280FD0DC
:1056C000206B07F098FA08B101210AE0206A0078FF
:1056D000C043800704D0FFF7F7F980F0010100E034
:1056E0000021206A027842EA01110170A97C99B177
:1056F000417889B1144805F005FC1248283880F833
:105700001880D5E91412C0E904120F48216A04F088
:10571000E5FF05F02FF803E005F0F4FB05F00CF8C9
:1057200096F86B200121002005F076FC2771206A95
:10573000018821828078A0742770BDE8FC87000072
:10574000D0000020D80A0020A8090020CD53000076
:1057500055510000C95200003555000000487047FF
:105760009913002004498A78824203D9084490F8AA
:105770004301704700207047C611002004498A7811
:10578000824203D901EB001083307047002070473C
:10579000C6110020054A01EB410102EB41010268FC
:1057A000C1F80B218088A1F80F017047C6110020B5
:1057B0002DE9F0410E46074615460621304607F012
:1057C00074FF0D4C60B1002004E02118401C81F8EA
:1057D0003B51C0B2A1788142F7D80120BDE8F081E9
:1057E0003146384607F081FD082803D0204480F870
:1057F0003B51F2E70020F1E7C611002004498A7806
:10580000824203D901EB0010C01C70470020704792
:10581000C611002010B540F2D3120021084806F04E
:10582000CAFB0822FF21074806F0C5FB05480021F6
:10583000001F017041704FF46171418010BD000084
:10584000C611002080020020014908707047000046
:105850007C02002001480078704700007C02002094
:105860000B4B10B59C7884420FD9184490F8030173
:1058700003EBC00090F853310B70D0F85411116055
:10588000B0F858019080012010BD002010BD00002C
:10589000C611002007498A78824209D9084490F845
:1058A000030101EBC00090F85A0100F001007047BD
:1058B00000207047C61100202DE9F0479846914618
:1058C0000C46054600F036F90646102806D000F0D2
:1058D00001F9102802D01220BDE8F087184FB878DF
:1058E00008282AD2102E05D100222146284600F091
:1058F00005F90646BC781022601CB87007EB041549
:10590000E81C494607F03AFE05F1830010224146A3
:1059100007F034FE1021404607F0C7FE3C4410213A
:1059200084F84301484604F5967407F0BEFEE0771C
:1059300004F8296C0020E073CEE70720CCE70000D4
:10594000C6110020064810B58078401E44B204E01D
:10595000E0B200F037F9641E64B2002CF8DA10BD32
:10596000C611002001484088704700007C020020DA
:1059700038B14AF2B811884203D80349488001205F
:1059800070470020704700007C02002005498A789B
:10599000824203D9084490F83B0108B100207047C7
:1059A00001207047C611002070B50D46064600F074
:1059B000C1F8104C102807D004EBC00191F85A111F
:1059C000C90701D0012070BD6178082910D21028C4
:1059D00008D004EBC000012180F85A116078401C07
:1059E0006070EFE701222946304600F087F8F5E7BE
:1059F000002070BDC611002070B50B4D2878401EE8
:105A000044B20AE005EBC40090F85A01C00702D086
:105A1000E0B200F01FF9641E64B2002CF2DA034910
:105A20000020487070BD0000C61100207C020020DC
:105A30002DE9F04100242546184E29E006EBC50764
:105A400097F85A01C00721D0284600F043F80346D2
:105A5000FFF7D4FE01460020102B09D0F21892F86F
:105A60003BC1BCF1010F02D092F84B2102B10120E1
:105A7000401E01420AD10A4807F5AA710355204683
:105A8000641C97F85321E4B205F0E6FB6D1CEDB2FF
:105A90003078A842D2D8BDE8F0810000C6110020BD
:105AA000800200200246094810B500780B4658B124
:105AB0000748817841B10BB1C01C01E00448833034
:105AC00004F02EFD012010BD002010BD7C0200203E
:105AD000C6110020084910B5034600208A7806E068
:105AE0000C1894F803419C4204D0401CC0B282427E
:105AF000F6D8102010BD0000C611002070B50C4B68
:105B000004461878451C1D70102803D34621282010
:105B1000FEF768F903EBC0030D68C3F85451898898
:105B2000A3F8581183F8534183F85A2170BD00003F
:105B3000C61100202DE9F0410F46064600240D4D08
:105B40000FE000BF05EBC40090F85311B14206D13D
:105B50000622394600F5AA7006F0A1F938B1641C96
:105B6000E4B22878A042EDD81020BDE8F0812046AC
:105B7000FBE70000C611002070B50546FFF7AAFF3D
:105B800010281CD10E4C2078401EC0B22070A842B4
:105B900015D004EBC00204EBC50102F58070D2F809
:105BA0005321C1F85321D0F85700C1F8570120788C
:105BB000FFF790FF102802D0204480F8035170BDF9
:105BC000C61100202DE9F047214C0646A719A07800
:105BD000401EC5B2A57097F80381AE422AD004EBEF
:105BE000051A04EB06190AF1030109F1030010225A
:105BF00006F067F90AF1830109F18300102206F02B
:105C000060F9601905EB450290F8031187F803115C
:105C100006EB460104EB420204EB4101D2F80B31E2
:105C2000C1F80B31B2F80F21A1F80F2190F83B0118
:105C300087F83B0104EBC80090F85A01C00704D173
:105C40004046BDE8F047FFF797BFBDE8F08700008A
:105C5000C611002005494A78521E4A7001EBC00166
:105C6000002281F85A21FFF787BF0000C6110020EB
:105C70002DE9F047044600F170054FF0010971B1BC
:105C800004F186077E1E012921D0022946D003296E
:105C90001BD139463046BDE8F04707F036BD4FF41A
:105CA0000672002106F087F904F010FC44F62B116F
:105CB000084085F8159085F84C00000A85F84D00DD
:105CC000FE2085F87C007F206872BDE8F0874FF0E9
:105CD0000008A4F80E8184F80381E16814480A469C
:105CE0000844B0FBF1F0C4F89C0040F6B830A4F8CA
:105CF000A000E38A284600F01DF83946304607F038
:105D000004FD06F0A8F818B1206900F039FB10B1C5
:105D100084F87481D9E784F87491D6E7C168B4F83F
:105D2000A231D4F89C212846BDE8F04700F002B823
:105D30007FC3C90130B500248486048F134D4C43C2
:105D4000B4FBF2F4048742F210746343B3FBF2F342
:105D50005B1C9BB203FB02F4C386AC4201D95B1E01
:105D6000C3860B4B40F27124B3FBF2F35B1C8387B9
:105D7000038E634302EB03135B1EB3FBF2F3C362B8
:105D8000836A4B43B3FBF2F1816230BD0048E80106
:105D9000005A620270B581EA11418BB2C57A83EA7A
:105DA00002010022CCB2090A94FAA4F491FAA1F1FA
:105DB000240E090E44EA012101EB0111521C194481
:105DC000D2B289B2032AEDD359402522B1FBF2F3B6
:105DD00002FB131200EBD20302F007065B780124EA
:105DE00004FA06F6334201D0104670BD4D43290C2B
:105DF000491CC9B200228518AB798B4212D395F8A1
:105E00000150002304FA03F6354201D0491EC9B2FD
:105E100021B15B1CDBB2082BF4D305E003EBC2001D
:105E2000C0B270BDC91AC9B2521CD2B2052AE2D39F
:105E300040F20D114620FDF7D5FF000070B590F837
:105E4000222090F82130012403FB01212522B1FBFF
:105E5000F2F302FB131100EBD10280F8221001F0E3
:105E60000703927D04FA03F31A4203D080F823104B
:105E7000002070BD90F82020B1FBF2F302FB13115B
:105E8000491CC9B20023C518EA7E8A4211D395F88D
:105E90001650002204FA02F6354201D0491EC9B25A
:105EA00021B1521CD2B2082AF4D304E002EBC301A0
:105EB000DCE7891AC9B25B1CDBB2052BE3D31F20D8
:105EC00070BD0000417841B1C078192803D2044A5E
:105ED000105C884201D1012070470020704700000B
:105EE000A0FC00000CB50BA2D2E90012CDE9001213
:105EF0000179407901F0070269461DF80220012A64
:105F000004D800F00700085C012801D900200CBD6E
:105F100001200CBD000101020102020310B50122A3
:105F2000C170192902D2064A525C06E0FF2904D04A
:105F300040F2D5312A20FDF755FF427010BD000018
:105F4000A0FC00002DE9F0475FEA000906D0214DD2
:105F500005F11000697B824619B10BE040F29331E4
:105F600005E0002107F0D1FD20B140F296312B2051
:105F7000FDF738FF2E8A0020FEF72CF9164FDFF8C8
:105F80005C800446386858B1288AA04208D3001BB8
:105F9000C0B2012106F0A9FF48B149463A6804E0C1
:105FA000D8F800201AB1288A4946904768B90021DC
:105FB000504607F0AAFD10B9288AB042E2D108483D
:105FC000016829B14846884710B10120BDE8F08733
:105FD0000020FBE7200F00202C02002030020020D0
:105FE0003802002070B505000C462ED01848026813
:105FF0005AB32846904740B32078112802D014287D
:1060000003D020E02079F0B10AE0207920B12846C1
:1060100007F084FF20B116E00E490020487312E01B
:10602000E4880021204606F060FF60B1008807F098
:10603000DFF800212046FEF76BF920B14FF49A718A
:106040002B20FDF7CFFE012070BD002070BD0000A9
:1060500028020020200F00202DE9F34F87B00C46C6
:1060600002A9079807F084F900287DD1DFF8209174
:106070004FF0010A8046039890F8700000280CD079
:10608000D9F8002062B121460798904740B12046D8
:1060900000F01AF90028EED1012009B0BDE8F08F18
:1060A000039D95F83401703550B995F824008DF8AA
:1060B0000400019801909DF8040008B1012000E05F
:1060C0000020834695F84500C0B195F8460080074A
:1060D00014D584F8018084F800A084F8048007991E
:1060E000A4F8051095F84710E171B5F84810218122
:1060F000B5F84A10618185F84580C8E70798FEF732
:10610000AFFA07000DD006F009FD060015D084F89F
:1061100001800D2020700798E080268184F804A07B
:1061200007E040F23A212DE0002138460A4606F009
:106130000BFE761EB6B2F7D2A9E70798FEF77AFAF9
:10614000F0B1BBF1000F20D006F01DFC60B1079844
:1061500007F04EF800210798FEF7DAF884F801807E
:106160000A214046217000E00FE084F8048007997E
:10617000A4F8051095F82510E1712435287086E7FC
:106180004FF416712B20FDF72DFE002085E700004F
:10619000340200202DE9F041124C07460E46E07D06
:1061A00010B1208B002812D00E480E30804607F028
:1061B00056FCA8B9E589E0893246394607F05EFC0D
:1061C00038B1E07D10B1208B401E20830120BDE856
:1061D000F081404607F043FC10B9E089A842EAD1BB
:1061E0000020F4E7200F002010B5017919B1012932
:1061F00006D0002010BD428883680088022103E099
:10620000428883680088012100F008F810B902492B
:1062100001200870012010BD200F00202DE9FF474C
:106220008A4699461546044601A907F0A1F8E0BB45
:10623000029F4FF0000870378DB12046FEF710FA2C
:1062400004000FD0294606F0A8FC060003D01D4824
:106250008088A84208D2002004B0BDE8F087012061
:10626000387529E089212AE02046314603AA06F044
:106270008DFC0398A0F8008080F80280397D09B178
:106280004FF0020A514607F06BFB314603262046C9
:106290004A462B46009606F05FFB2046294606F04C
:1062A00019FC58B1444601A800E005E007F0DAFB0C
:1062B0000298A0F8FA403C750120CDE79F212B20E1
:1062C000FDF790FD200F002010B52C4986B08A7D87
:1062D0000178D30701D1192904D018291ED0122919
:1062E00045D049E08088ADF8000002A907F040F8E9
:1062F00008B1582135E0039810F8661F8DF8021098
:1063000041788DF803104088ADF8040002216846FA
:1063100009F09AF840B340F24D1122E091072BD4D6
:10632000848803A9204608F0AEFE10B14FF4AA718C
:1063300017E0ADF80040BDF81200ADF80200BDF85E
:106340001400ADF80400BDF80E00ADF80600BDF86D
:106350001000ADF80800684608F013FF20B140F2C5
:106360005D112B20FDF73EFD012006B010BD510749
:1063700002D4807BC007F7D00020F6E7200F002072
:10638000F0B56FF01F02010C02EA90261F25A1F55F
:10639000AA4054380DD0A1F5AA40553809D0A1F52E
:1063A0002850AA3805D0A1F52A40AA3801D00120EA
:1063B00000E00020002213464FEA020482EA0107AF
:1063C000FF431F437F1C0FD006F00107520842EA2B
:1063D000C73205F001075B0876086D08641C43EAC4
:1063E000C733162CEAD3F0BD0020F0BD70B50446CB
:1063F000007C00B302281ED05FF0010004F14901C7
:1064000084F848000D46C0B1E07DF0B1D4F8110029
:10641000C4F84900B4F81500A4F84D00207C07F03A
:10642000E0FC20760820607694F84800294607F0C2
:10643000C4FCA8B90EE00020E0E70020FEF7D2FB84
:106440000028EBD140F2AA4101E040F2AE412D20FC
:10645000FDF7C8FC94F84800294607F0B7FC00B1E6
:106460000120A076207E10B9A078400706D594F8C8
:106470004F0004F1500106F038FF607600252564D6
:1064800005F0AAFB60640021204607F0C9FD84F8EE
:106490005650A078400708D5207E002805D0204619
:1064A000BDE87040002100F0FFBD70BD08B590F858
:1064B00094208DF80020009A00929DF80030002270
:1064C00063B14A7017230B7050F8953F4B604368D7
:1064D0008B60037A0B7300F8012C3BE090F88E3050
:1064E0008DF80030009B00939DF8003043B14A7056
:1064F00005230B70D0F890304B6080F88E2029E097
:1065000090F864308DF80030009B00939DF80030C7
:106510001BB100BF07F05BFD1CE090F886308DF8E2
:106520000030009B00939DF80030ABB190F86430D0
:106530008DF80030009B00939DF80030002BE9D1CE
:106540004A7014230B7050F8883F4B6083880B818E
:1065500000F8022C012008BD002008BD30B50C4613
:106560008DB005460146202202A805F0AAFC0AA823
:1065700007F003FEA07A8DF8180020788DF8080047
:10658000B4F80100ADF800009DF8000000F0010132
:10659000C0F3400241EA4201C0F3800241EA8201B5
:1065A000C0F3C00241EAC201C0F3001241EA021185
:1065B000C0F3401241EA4211C0F3801041EA80105A
:1065C000ADF80A00207D012806D0022804D040F250
:1065D00075210620FDF706FC8DF80C00617A0AA8EB
:1065E00007F0B2FD207D0121022802D1607D401C10
:1065F000C1B2A07E401CC2B20AA807F06CFDBDF873
:106600000A00000701D5002020E00AA807F075FD68
:10661000BDF80A10282200F0EDFD40F2712100F2D1
:10662000D520B0FBF1F04843D4F8021040F27123BA
:106630000A0A40F271214A43D4F80510090A594365
:10664000904201D8049204E0884201D8049000E00E
:106650000491A07C8DF81700207E012800D0002036
:106660008DF81400E86A06F0FEFCE86A06F09EFD6C
:10667000202202A9284605F024FC0A982862BDF8C9
:106680002C00A884E07A68B102280BD05FF00100EA
:1066900085F84F00E0682865208AA5F854000DB001
:1066A000002030BD0020F3E70A4A10B50021117028
:1066B000094C606000F022F810B140F22A3104E089
:1066C000A068002804D140F22D312D20FDF78AFB6F
:1066D00010BD00003C0F0020F000002002490148DE
:1066E00088607047DC710000F000002002490860FB
:1066F0008968096808470000F0000020084810B5C4
:10670000007810B10C24204610BD00241822214628
:10671000034805F050FC04F037F903F019FFF2E7E5
:106720003C0F0020044910B50978012901D100F07F
:1067300083FB002010BD00003C0F002002490148EF
:1067400008607047856F0000FC0000202DE9F041D3
:106750000F00044623D004F12000054607F0F6FCA4
:10676000B0B9A078C0F3C00050B3284607F0C5FC0C
:106770000646284607F0EAFC301AC0B207F03BFD97
:1067800001463548426811444160284607F0FCFC48
:10679000284607F0BEFC0146204607F07DFC2F4D41
:1067A00094F8566000216868018007F08BFC6088CF
:1067B000132813D009DC102836D0122809D131E073
:1067C0002046BDE8F04100F037BB15280FD01D284A
:1067D0000DD040F271612D20FDF704FB00216868A7
:1067E00007F0F6F80121686807F06CFC20E0012151
:1067F000686807F0EDF80121686807F063FC36B1BE
:1068000004F15701686807F0FEF8012106E004F181
:106810005001686807F0F7F894F84F10686807F0BF
:10682000F8F805E0062100E00221686807F0D0F8DA
:10683000204600F0AFFC60881D2806D0152804D043
:10684000A28E216B686807F0B3F839462046BDE890
:10685000F04100F0E7B900003C0F0020F0000020FC
:106860002DE9F0412E4D07462878022805D02878DA
:10687000032802D04FF4506129E02A4C2068017BA4
:1068800009B107F014FC60684FF00008027802F0CC
:106890000F0657B3216801F1490391F84810B1EB95
:1068A000D21F22D106221946093005F0F8FAE0B9C4
:1068B0004146606807F06CF8B8B12A782068314624
:1068C000022A07D02A78032A04D040F6D9412D2085
:1068D000FDF788FAA2682B7852696FF0070606EB7D
:1068E0008303D2589047064600E00126A87B18B1E2
:1068F00004F04AF803F02CFE002E0FD0206807F0B9
:1069000090FC30B104F064F8A0688068BDE8F04104
:1069100000472068BDE8F04100F08EBABDE8F08184
:106920003C0F0020F000002010B5032902D00529FB
:106930000AD102E000F07EFB03E00449096809B1D6
:10694000884708B1002010BD012010BDFC000020C8
:10695000094A0300106801D000F06EBA002909D07E
:106960009168064A096912786FF00F0303EB8202FF
:106970008958084770470000F00000203C0F0020B5
:1069800070B504464088102819D0104DA87B20B15E
:1069900003F0FEFD402004F007F80D48406804F0C5
:1069A000B1FAA078400704D400212279084604F007
:1069B00033FB002004F048F90220287070BD204607
:1069C000BDE870400121FFF7C1BE00003C0F002070
:1069D000F000002010B5124C206800F025F8206867
:1069E00007F01FFC002820680BD00E490A78022A05
:1069F0000BD00A78032A08D040F607412D20FDF776
:106A0000F1F9BDE8104000F017BAA2680978D26821
:106A10006FF0070303EB81015158BDE810400847B0
:106A2000F00000203C0F002010B5017B09B107F0F9
:106A30003EFB0548807B002805D003F0A5FFBDE89C
:106A4000104003F085BD10BD3C0F00202DE9F0473C
:106A5000594D044688B02878F0BB2078FF283CD0F8
:106A60000026AE816E606E70AE7084F86160534B2C
:106A7000DFF84C810FCB8DE80F00D8F80800406894
:106A80000390684604F0B4F804F0ACF904F00CFC90
:106A900003F07AFF03F05CFD4A4804F0FDFA474832
:106AA000001F04F003FB04F12000074607F06CFB15
:106AB000384607F02EFB0146204607F0EDFA94F920
:106AC0000E0004F019FA2179002004F015F8A860EE
:106AD00038B1A07E68B907E0FFE70C2008B0BDE838
:106AE000F0870120287064E0207E10B9A07840076C
:106AF0002BD505F071F882465146606CFAF7AEFD71
:106B0000DFF8C490074690FBF9F109FB1170414290
:106B10005046FAF771FD606497FBF9F0216C084468
:106B20002064FEF71FFF216C88420ED8C4E9106A6A
:106B30000121204607F074FAA078400705D5207E91
:106B400018B10121204600F0AFFA04F13001E06AEB
:106B500006F0FBFA04F13801E06A06F0F9FAFEF7F4
:106B600067FFD8F80400C01C06F0B2FBA873A07839
:106B7000C0071ED004A9002006F0C1F920B140F6DC
:106B8000CE112D20FDF72EF9FF20E8730CE00698BA
:106B9000E169814208D08178E973D0F80310296156
:106BA000B0F80700A88204E004A8FDF761FB002804
:106BB000EDD0002092E700003C0F0020BC710000E7
:106BC000F0000020D6BE898E40420F0010B504466A
:106BD000FFF73CFF002808D104480078012803D0C3
:106BE00000212046FFF7B2FD002010BD3C0F002021
:106BF0000A4810B50A490468087800280DD00878BA
:106C0000022802D00878032802D12046FFF70CFFA3
:106C10002046BDE8104000F00FB910BDF000002084
:106C20003C0F00202DE9F041044627480D464068FE
:106C300004F068F9254E0420307025B360881028D0
:106C40002AD004F120008046B56807F056FA0746BE
:106C5000404607F07BFA381A401EC0B261882822ED
:106C600000F0E8FA0544A078C0F3C00030B17068C5
:106C7000054407F0C4FA2844C4F8B0002279294634
:106C8000002004F04DF96088132813D009DC102887
:106C900017D0122809D10DE02179002003F0E0FE81
:106CA000F1E7152806D01D2804D040F68E512D207E
:106CB000FDF798F82279BDE8F0410121002004F0A9
:106CC000ABB9BDE8F0810000F00000203C0F0020CF
:106CD00010B5044600780B4684F89500FF2910D0C3
:106CE00004F19702511E1846FEF7BAFD30B194F830
:106CF000960040F0020084F8960011E040F6C5715D
:106D000020E0124840680178C1F3801184F89610A1
:106D1000D0F80310C4F89710B0F80700A4F89B004F
:106D200094F926007F280BD084F89D007F2084F8FA
:106D300026007E340120A075BDE8104003F01CB889
:106D40004FF464612D20FDF74DF80000F0000020A5
:106D50002DE9F04790460E460446032904D094F8E6
:106D6000600008B1012000E00020814603F02AFE07
:106D70000546032E03D00127052E05D008E0A07894
:106D80000227C0F3400001E0A078C00700284AD0E5
:106D9000B9F1000F46D12648807B40B106F09BFA3E
:106DA00088F80000FF2802D0FEF774FD0543214E4D
:106DB00094F84F2070680178C1F38011914206D198
:106DC000062204F15001C01C05F069F830B1002022
:106DD00098F80010FF2907D0A8B901E00120F7E7D3
:106DE000607E88420FD008E038B1716811F8030B5B
:106DF000C0F3801007F0D2F828B10020A17849072D
:106E000003D590B90EE00120F8E775B9E07B08B131
:106E1000B84207D1716811F8030BC0F3801007F076
:106E2000BDF810B10020BDE8F0870120FBE70000AD
:106E30003C0F0020F000002070B50446806A134D1E
:106E4000401CA062A87B002620B103F09DFD03F04A
:106E50007FFBAE732E7094F8610008B101210FE042
:106E6000607B60B1A16A884209D80121204607F001
:106E7000EDF9A078BDE87040C00702F07DBF0021A9
:106E80002046BDE8704007F0E1B900003C0F00204B
:106E90002DE9F843044690F8640017460D468DF836
:106EA0000000009800909DF8000010B140F63B41B2
:106EB00054E084F866302888A4F86800002B5DD17F
:106EC000E86806F066FAA4F87E00A88AA4F88000B4
:106ED000E88AA4F8820095F8750184F88400217E80
:106EE00004F14908002629B194F84800414606F00B
:106EF0006DFF40B994F8620070B194F848004146C3
:106F000006F05BFF40B1D4F84900C4F87200B4F851
:106F10004D00A4F8760003E0C4F87260A4F876602F
:106F20001748FF2F40680178C1F3801184F86B1077
:106F300050F8031F15D0A1678088A4F87C0004F1E5
:106F40006C02511E3846FEF78BFC28B114F86B0F0B
:106F500040F0020020700AE040F65C412D20FCF772
:106F600041FF44F86C1F8088A080E6602682288854
:106F7000FDF760FBBDE8F84305F09EBEBDE8F88371
:106F8000F00000202DE9F8430446FF208DF80000B2
:106F900001266A4605212046FFF7DAFEF0B3234DAD
:106FA000234FB0466868FA7B4FF000090178C1F3BF
:106FB0008011914206D1062207F11001C01C04F095
:106FC0006EFF58B36A68E069127810F8851FC2F343
:106FD00040121140017001222046E16900F092F850
:106FE00000239DF800202046E169FFF751FF84F857
:106FF000648002F0C1FE87F800900521E06900F08E
:107000001DFA6868E169D0F8032041F8032FB0F851
:1070100007208A800078C0F3801000E002E0E16978
:10702000887000E000263046BDE8F883F0000020BC
:107030003C0F00207CB50446FF208DF800000125A0
:107040006A4603212046FFF783FE28B3207B68B100
:1070500094F894008DF80400019801909DF80400C4
:1070600020B99DF800102046FFF732FE0C4E00219B
:1070700070680180042106F0ABFC204600F08AF81D
:10708000A28FA16B706806F0DAFC06490520087033
:10709000706803F037FF00E0002528467CBD000043
:1070A000F00000203C0F002070B504460E46407EE4
:1070B000FEF7A4FB050019D0102106F0F6FA00280F
:1070C00014D1012084F8560004F1570132460C46D1
:1070D000284606F0A2F82146054C606806F093FCAD
:1070E0006068BDE87040012106F093BC70BD0000EF
:1070F000F0000020024801210068FFF727BB0000D4
:10710000F00000202DE9F041214E80460C467068C9
:10711000154650F80F1F2161818821838179A1765E
:10712000408906F032F90746E06070683946807D94
:1071300006F0B6FAA08370683946B0F8170006F07A
:10714000ABFA2062706830F81B1FA1824188E1828F
:107150004168C4F88610017A84F88A10417A01F0F7
:107160001F0184F89110407A400984F8750104F1F8
:10717000620005724572012181720021363806F0E5
:107180009DFD98F80E0084F86E00BDE8F0810000C7
:10719000F000002070B5074D044600F14901686811
:1071A00006F03EFC94F848106868BDE8704006F0B0
:1071B0003DBC0000F000002055555500D569000089
:1071C00061680000516900000000000029690000AA
:1071D00081690000C3DF0000C9DF0000CD6B000043
:1071E000F16B0000F5700000D8710000D071000054
:1071F000CC71000010B5421E022A01D9CA2109E053
:10720000401E102909D012290CD013290AD01529A3
:1072100005D0D8212F20FCF7E5FD054904E00449FD
:10722000891D01E00249891F31F8100010BD0000DE
:1072300016E20000421E10B5D2B2012A03D91D2960
:1072400001D0EE210DE0132913D004DC10290BD05E
:10725000122904D10DE0152908D01D290ED04FF4B4
:1072600081712F20FCF7BEFD074804E00648083076
:1072700001E00548001D30F8120010BD40F25A31FF
:1072800010FB01F010BD000004E200002DE9F04108
:10729000044690F8B40015460F4600285BD12146FD
:1072A0004348FBF7ADF80646202854D0342200218D
:1072B00004F1A00004F07FFE84F8A0600126C4F869
:1072C000A47084F8B4605FB1012107F59270FCF7F7
:1072D00031FE97F8240100F00700401C87F82401D4
:1072E000204607F078F9A4F8C000032084F8C20013
:1072F00084F8C360002704F8B87FFAF7EDFA218913
:10730000B83C884200D8084600F2BF601FFA80F8F7
:10731000204606F003FE08B308F07BFB00F5CD60C5
:1073200081B2284604F08CFC2844C4F8BC00A43484
:1073300004F052FC4146FAF75FF9206204F8037C3E
:107340002671012006F057FF00F58470281AA76205
:10735000A060A43C17E00C20BDE8F081204607F0B7
:107360008DF844F8BC0F04F81B6C04F035FC06469D
:10737000002007F0DCF900EB08013046FAF73CF991
:107380002561A060BC3C04F1B80194F8A00007F0AE
:1073900020F938B1A4F8C8700021204606F0E0FDBD
:1073A0000020D9E74FF4F9713020FCF71BFD0000F5
:1073B000AD7A000003480021017001228270417003
:1073C00006F084BF000100200149087070470000EA
:1073D0000001002005494FF47A72B1FBF2F110B5BB
:1073E00001F5237106F083FC80B210BD7D520100CF
:1073F0002DE9F041104CD4E9015703F08DFC06460D
:10740000207828B132463946284605F0C8FF05469F
:107410006068854205D0E168281A0844E060FBF7FF
:10742000F9F86560AE4201D8607810B10020BDE87F
:10743000F0810120FBE700000001002070B5224C24
:10744000054606293CD2DFE801F0050B030E0F25A7
:10745000002100E001212846BDE8704000F0ECB8B2
:10746000032085F8340170BD03F08AFCC5F8700173
:1074700095F86B0008F066FBD5F87011081A616882
:1074800001446160A1680844A0602846BDE87040DE
:1074900007F032B803F040FC01460022A06907F073
:1074A000FCF8A0690949D0F8A42090F8A000FAF7E8
:1074B00069FE0028D7D140F261713020FCF792FCC0
:1074C0004FF4EF61F9E700000001002059E70000E8
:1074D00010B50C2804D340F203310620FCF782FCDF
:1074E000014931F8100010BD52E90000FEB5184CFA
:1074F000012060704FF6FF750BE0002105F0F5FCF0
:10750000060010D096F86801FAF76EFE304607F0D4
:10751000B7F86946002005F0F2FC80B14FF487719E
:107520003020FCF75FFC4FF49771F9E7029830B117
:1075300090F8341119B10088A842DED104E0684601
:10754000FCF796FE0028F1D000206070FEBD000020
:10755000000100202DE9F047044636481E469046BB
:1075600080788946002568B3FCF7D4F850B3B4F8A6
:107570002001022826D394F83401022822D094F85E
:107580004A01F8B994F87501FFF7A2FF00F5C86049
:1075900081B2318094F834010027012815D0E068C9
:1075A00004F04EFBB4F80E2180B24244A2EB090174
:1075B000D4F83C21C4F83C01821A01FB0275012079
:1075C00084F84A012846BDE8F08794F88100032832
:1075D0002CD00121002005F09CFF216A4718D4F827
:1075E0002C013188D03404F02BFBA26D216E821A5D
:1075F00001FB0255A0653188384604F021FBA16EDD
:10760000A066411A0D44318854F8C40C04F018FBEC
:10761000E28F4244A2EB0901226E891AE26E491EF2
:10762000821A01FB0255E066D03CC8E7D4F82C0171
:10763000D3E700000001002038B5002504460129E9
:1076400002D11148407878B1042084F8340100BF99
:1076500006F04BFFA4F86651B4F87400A4F8460194
:1076600004F59574E57738BD0095B4F8FC10012356
:107670000022204600F00AF80028E9D040F2D46148
:107680003020FCF7AFFB0000000100202DE9FF4F88
:10769000044685B090F86B009A46CDE900300F465D
:1076A00008F0B7F9054694F87501FFF711FF284473
:1076B000ADF8080094F87E000D2804D00020039057
:1076C000079810B12EE00120F9E794F8340103285F
:1076D00028D1039830B3B4F89401B84222D1D4F839
:1076E0003C01C4F82801E068C4F82C01B4F8660134
:1076F000B4F80E110844C4F83001204607F03FF9F1
:10770000D4F898012062B4F89601A083D4F89C01C3
:10771000E060B4F8A001A082B4F8A201E0820220E7
:1077200084F83401B4F8740004F5A675381A0FFA19
:1077300080F9B4F86401381A0FFA80F8B8F1000F34
:1077400006DAD4F85C01C4F860010120C846009054
:1077500002AB4A4641462046FFF7FCFE049094F8EF
:107760003401DFF844B340B101287DD0022852D063
:1077700003287AD040F2575192E10121002005F010
:10778000C8FE0646206ABDF80810304404F058FAD6
:10779000C4F83801BDF80810E06804F051FAC4F8E4
:1077A0003C0101A9684603F01BFADDE90012D4F898
:1077B0006001FAF7E5FF8146204606F088FE94F85E
:1077C0006B00D4F86C8108F0CBF94AF2A131014486
:1077D0004FF47A70B1FBF0F0216AD4F838213144CB
:1077E000081A811A41442039A1EB09065000A18BE7
:1077F0006030014494F86B0006F0D9FE2230CBF8DB
:107800001000D4F86C015946301AB0F5D87F59D21F
:107810004FF49E6144E1D4F82C11206A0844BDF86D
:10782000081004F00DFAC4F83801BDF80810E0683B
:1078300004F006FAC4F83C01204606F048FEB4F80D
:107840000E0110BBBAF1000F1FD094F86B804046B8
:1078500008F086F94AF2A13101444FF47A70B1FB85
:10786000F0F0D4F8381101E02DE049E00844226A34
:10787000D4F82C1111440E1A404608F063F9D4F8DC
:107880007011081A0644203E06E0216AD4F82C0143
:107890000844D4F83811461AD4F83021D4F8281105
:1078A000D4F8380101FB02004000A18B6030014494
:1078B00094F86B0006F07BFECBF8100001205946CF
:1078C00084F8340162E0D4F83C11E068B4F80E2189
:1078D000461A02EB0900D4F83021D4F828C1801AE6
:1078E000D4F83831401E0CFB023200FB012040006E
:1078F000A18B6030014406FB08F694F86B0040E071
:10790000E068D4F83C1100FB08F008FB110694F87D
:107910007D00242803D094F87E00242809D1B4F8EF
:107920009401381A00B2002803DB94F8970100B1E3
:1079300001900098D8B1B4F80E01C0B9D4F8700124
:1079400000287CD094F86B0008F00AF94AF2A131C3
:1079500001444FF47A70B1FBF0F0361A94F86B00E2
:1079600008F0F0F8D4F87011081A0644203EB4F874
:107970000E1101EB0900D4F83C114843410060317D
:10798000019806F014FE5946CBF8100004980969D6
:10799000331AD4F83C61E068801BA0F23E20CBF89B
:1079A0001400814200D80846C4F80801002028705D
:1079B000642028811946D4F86001F9F71DFEE860BB
:1079C00004F12C0006F064F9D4F80811084468604A
:1079D000E868C4F86001A4F864710120A872B4F8E2
:1079E000F810C91B09B2002901DD0321A97203990E
:1079F00031B3BAF1000F26D0B4F8202192B3B4F815
:107A0000221100BFA4F8221194F82431491C4B43E1
:107A1000934218D2A97A491E002914DDA872B4F83D
:107A200022010121401CA4F8220104F59270FCF708
:107A300065FA94F8240100F00700401C01E012E010
:107A400014E084F8240194F86801294606F0C1FD89
:107A500020B3079880F0010084F84801002009B0A5
:107A6000BDE8F08F18E040F2425119E0BAF1000F82
:107A7000C2D194F834010028E5D0D4F83C11E06874
:107A8000411A284605F057FD0004000CDBD012997E
:107A900001B108800120E2E70021B3E740F2A251E2
:107AA0003020FCF79FF900000001002070B540B1C4
:107AB00009294AD2DFE801F007173D3D39492B413A
:107AC0004500D3213EE0224904468861FEF70EFEC0
:107AD00010B140F27F2135E0D4F8BC00BDE8704021
:107AE000F738FAF797BD054606F018FAA8B9284600
:107AF00006F0C4FC0446D5F8BC00A0420BD2201A04
:107B00000421F9F7A7FC30B12846C5F8BC40BDE810
:107B1000704006F0D8B9C5F8BC402846FEF702FE12
:107B2000002814D040F2B3210CE0BDE8704003F00F
:107B3000DDBABDE8704006F03DBCBDE8704006F01F
:107B400094BCF5213020FCF74DF9F921FAE770BD1E
:107B50000001002070B50446F9F7BEFE642801D983
:107B6000054600E0642594F86B00282106F020FC0F
:107B70002844D4F83C1100F50E700E1894F86B00F0
:107B8000282106F015FC00F527722046E16A06F070
:107B90001EF8054632462046E16806F018F8074907
:107BA0008542886000D228464860D4F85001A0F28F
:107BB0006510C860BDE87040FAF72CBD00010020D8
:107BC00006480549016506494165074805490165BB
:107BD00006494165704700002191000030010020F6
:107BE000FD91000059980000940100208998000040
:107BF000F8B50D460746002105F077F9041E4FD071
:107C000094F8700000284BD094F8B8018DF800006B
:107C1000009800909DF800000026D8B16E700720F3
:107C200028700BE084F8B861A684D4F8BA016860C3
:107C3000D4F8BE01A860B4F8C201A88194F8B801D4
:107C40008DF80000009800909DF800000028E9D110
:107C50002E710BE194F8C401A0B394F8C4010B2871
:107C600016D00C2804D040F6E9213120FCF7BAF8F0
:107C70002088FCF7DFFC074604F0FDFF78B96E7042
:107C80000C20287094F8C60128712088E88013E041
:107C90002088FCF7CFFC074604F0EDFF08B1002078
:107CA000F8BD6E700B20287094F8C60128712088EA
:107CB000E88094F8CA01287284F8C461384604F058
:107CC000F5FFD3E0FFE794F8FA018DF80000009883
:107CD00000909DF8000030B16E700E202870AF80CB
:107CE00084F8FA61C2E094F8CC018DF800000098A5
:107CF00000909DF8000098B16E70082028702088D0
:107D0000A880D4F8D011C5F80610D4F8D411C5F85D
:107D10000A10B4F8D801E88104F5E6742670A5E0ED
:107D200094F8F4018DF80000009800909DF8000090
:107D3000A0B16E701620287005E000BF84F8F461D1
:107D4000D4F8F601686094F8F4018DF8000000980A
:107D500000909DF800000028F0D187E094F80A0216
:107D60008DF80000009800909DF8000070B16E70D2
:107D700006202870D4F80C026860D4F81002A860BD
:107D8000D4F81402E86004F503743AE094F8DA01D8
:107D90008DF80000009800909DF80000D0B16E7042
:107DA000122028700BE000BF84F8DA61D4F8DC01FF
:107DB0006860D4F8E001A860D4F8E401E86094F8C1
:107DC000DA018DF80000009800909DF8000000286E
:107DD000EAD14BE094F8E8018DF80000009800909B
:107DE0009DF8000080B16E7018202870D4F8EA0168
:107DF0006860D4F8EE01A860B4F8F201A88104F537
:107E0000F57404F8026C31E094F8FC018DF8000080
:107E1000009800909DF8000038B119202870D4F81F
:107E2000FE01686084F8FC6120E094F802028DF89D
:107E30000000009800909DF8000000283FF430AF4B
:107E40006E701320287007E084F80262D4F80402F0
:107E50006860B4F80802288194F802028DF80000E6
:107E6000009800909DF800000028EDD10120F8BD99
:107E70001B481A4981601B4941601B4901601B492D
:107E800081621B49C1621B49C1601B4981611B4959
:107E900001631B4901621B49C1641B4981641B4981
:107EA00041641B4941631B49C1611C481A498160F7
:107EB0001B49C1611B4941621B49C1621B490161E8
:107EC0001B4941611B49416441631B4981611B4955
:107ED00001631B4981641B49C1647047AD95000073
:107EE00030010020E98E0000458F0000C59200009F
:107EF00009930000F18F000085950000C9960000ED
:107F00009D900000999200006D9200004595000040
:107F100075950000E1950000419A00009401002051
:107F2000699A00002998000001990000FD9700005F
:107F3000A999000085990000CD990000C19A000020
:107F4000B9980000E998000006480549816506498E
:107F500001660748054981650649C165704700000B
:107F60002993000030010020019400002D990000A9
:107F7000940100205D9900002DE9F84301267C4C16
:107F8000002566F30701658065702570A06089464D
:107F9000804680F803610088FCF762FB80B1A0682E
:107FA0000088FCF7FBFDA0680088FCF79FFDA06837
:107FB000B0F8FA10C9B1703006F025FD18B114E020
:107FC00040F6C4316BE0A06890F878118DF800108D
:107FD000009900919DF8001039B190F8802001239C
:107FE0001946703005F0EEF980B1A068703006F0E7
:107FF0000AFD28B1A06890F8EC0000BF00F0B0FBCB
:10800000A06890F8051189B1A5801EE0A068A0F8CD
:10801000A85090F8791180F8EE100021022000F0AD
:1080200041FEA06880F802510220E7E790F8B811FD
:108030008DF80010009900919DF8001019B9818CFD
:10804000828A914200D8818AA18030F8FE1F491EA1
:108050008FB230F8021F394420F85C190188394486
:10806000018001F05BFD20B1A06850F8981F3944F1
:108070000160A168B1F8FA00012802D8401CA1F8FB
:10808000FA000FB181F80C5181F80251B1F8FE20CD
:1080900001F1700005F018FB20B140F608413120D5
:1080A000FBF7A0FEA06890F87E100B2901D00C29E8
:1080B00018D1B0F87420B0F89431D21A12B2002A54
:1080C00010DBD0F89611C0F8861090F89A1180F85D
:1080D0008A100321FDF7CCFDA06880F87E5080F85F
:1080E000BE6026E0242911D1B0F87410B0F89421B4
:1080F000891A09B2002909DB80F87E5000F082FE5F
:108100000028A06880F8AE5129D012E090F87D10C8
:10811000242901D025290CD1B0F87410B0F894218D
:10812000891A09B2002904DB80F87D5000F06AFE4C
:10813000A8B110480090104B104A41464846FCF741
:10814000E3FDA0680123052190F87E20703005F042
:1081500039F9002809D0BDE8F843FCF7CFBDBDE8E8
:10816000F8430021084600F0D5BBBDE8F8830000C5
:108170001C0100201589000019840000518D0000A9
:1081800070B50F4CA56895F87D10202902D02629DE
:1081900003D011E000F084FE08E095F87E20012372
:1081A0000B2105F1700005F00DF938B1A168002030
:1081B00081F87D0081F8AE00002070BD2A20E9E73B
:1081C0001C01002004480021806820F8B01F81783D
:1081D000491C8170704700001C010020074810B541
:1081E000816811F8B20F401E40B20870002804DA0E
:1081F0004FF4C9713120FBF7F5FD10BD1C010020C3
:108200001A4908B5896891F87E20B8B1102A06D0BD
:10821000142A07D0152A08D01B2A22D108E00121F0
:108220000B2007E001F0ACFA06E000F059FD03E096
:108230000121062000F036FD012008BD212A10D1C1
:1082400091F8AE0102280ED091F8AE01012808D1B4
:1082500091F8AF018DF80000009800909DF80000A3
:1082600008B1002008BD01211720E3E71C01002010
:1082700038B500286BD1374CA06890F87F10CA073A
:1082800002D0012109205BE08A070AD501210C20D8
:1082900000F008FDA06810F8B61F41F00101017060
:1082A00050E04A0702D50121132049E00A0705D50D
:1082B00010F8E91F41710121072041E011F0300F52
:1082C00045D090F8A5118DF80010009900919DF807
:1082D0000010C9BB90F8A4118DF80010009900910E
:1082E0009DF80010C9B190F87E1024292DD090F887
:1082F0007D10242929D0002300F5CB7200F5D2711E
:1083000005F057FCA06810F87F1F21F0200141F014
:1083100010010170002180F82511A06890F87F10ED
:10832000C90614D505F060FC00F010F9A16801F150
:108330002C00C28B21F8EE2F408C488001211520A3
:1083400000F0B0FC012038BD01E00123D4E700209B
:10835000F9E700001C01002070B50D46064605F047
:108360009FFA0446304605F0A7FA294600F01EF8A9
:10837000B8B1204605F0BFF801000DD00A4880686A
:1083800090F86B208A4207D090F8AE11012905D0F1
:1083900090F86700204204D0012070BD90F8B10130
:1083A000F8E7002070BD00001C01002070B50D46EC
:1083B000044605F0A0F850B31649896891F86A2080
:1083C000824224D091F8AE31012B05D091F866306D
:1083D000234213D01DB11AE091F8B031F8E791F8BB
:1083E0006310214213D15AB1042A0ED004280CD0B4
:1083F000082A0AD0082808D0824208D9002070BD77
:1084000040F255110620FBF7EDFC8242F6D3012025
:1084100070BD00001C0100200C490246487898B944
:108420000846806842B18978090703D590F8800032
:10843000082809D00120704700F12C018A8C818E18
:108440008A4201D8FEF7D4BF002070471C010020EB
:1084500038B53D4C0546A068703006F0D4FA0028C7
:1084600070D1002D6ED1A0680123194690F88020AC
:10847000703004F0A7FF002864D1A06890F878114C
:108480008DF80010009900919DF8001049B100216D
:10849000A0F8A81090F8791180F8EE1000210220C1
:1084A00045E090F87E2001230421703004F08AFF1B
:1084B0000546FFF7DDFE002844D12846FFF7A0FE61
:1084C00000283FD1A0680123002190F87D20703062
:1084D00004F078FF78B1A0680123042190F87E2091
:1084E000703004F06FFF30B9A06890F8A20010B1AE
:1084F000002112201BE0A06890F87D100A291AD0F4
:10850000002D1FD100F01AFB00281BD1A068012309
:10851000002190F87D20703004F054FF002811D025
:10852000A06890F88C0100280CD00021FF20BDE845
:10853000384000F0B7BB10F8EA1F01710021072096
:10854000F5E7FFE738BD00001C0100200A4810B520
:10855000816891F86000012809D0088801F5ED7262
:108560002C3105F002FBBDE8104001F005BC0220F3
:1085700081F8600010BD00001C01002070B5254C82
:1085800005002FD100F0A4F800F048F8050029D12B
:108590006088410706D5A16891F88010072901D1AC
:1085A00001212170800712D5E068C078192805D212
:1085B000194951F8201009B1884708E0FF2804D074
:1085C00040F24D713120FBF70DFC01F00BF9A07862
:1085D000C00607D5A06890F87E100B2902D10C21A7
:1085E00080F87E106078000711D5A068012305216E
:1085F00090F87E20703004F0E5FE28B1A1680825CF
:10860000002081F8C40102E00020FCF74DFC284660
:1086100070BD00001C0100209401002070B52A4CA0
:108620000020A178C90715D0206901230521C5784C
:10863000A06890F87E20703004F0C4FE58B1AD1EE2
:108640000A2D06D2DFE805F007070505070705052F
:108650000707082070BD2069FDF734FC38B1206998
:10866000C57845B1012D06D0162D18D103E0BDE81F
:10867000704000F03DBDA06890F87D0004F0F0FE71
:1086800068B1A16891F87D001F2808D0202803D088
:10869000162D0CD0022070BD262081F87D00192DEA
:1086A00007D20A4850F8250018B1804703E020207F
:1086B00070BD00F01DFDA268F2E93213491C43F1C0
:1086C0000003C2E9001370BD1C010020300100202E
:1086D00070B5224CA07800073ED5A068703006F037
:1086E00092F948B1A068FE21002580F8EC1090F8BE
:1086F0007E1019290CD104E040F257713120FBF7AC
:1087000071FB80F8B350FFF769FDA06880F87E50D8
:10871000A06890F87D101F2902D0272913D10BE003
:1087200090F87E0004F09CFE08B1262000E0202096
:10873000A16881F87D0006E0012180F88D1180F8A4
:108740007D5080F8AE50A06890F88010082903D1C1
:108750000221217080F8EC1070BD00001C01002087
:10876000FEB505466846FCF703FA18B3222200213D
:10877000009803F020FC0321009805F0F1F8009820
:10878000017821F0100101702946FDF7C7FB002197
:108790005F4C44F62F160E2D7ED00EDCA5F102059F
:1087A0000C2D1CD2DFE805F01E1B49AAAA1E1B5582
:1087B0001BAA343040F68211A6E0152D5CD008DCEF
:1087C000112D14D0122D1ED0132D1CD0142D06D116
:1087D00052E0162D27D0172D69D0FF2D72D040F60C
:1087E000F81191E0A168009891F8EE100EE0A068F1
:1087F00090F8EE10009805F08FF8A06890F8EF1050
:10880000009805F08BF879E000980621017175E079
:1088100000980B220271592242718171B021C171FD
:10882000122101726AE00098D4F8081091F8B02182
:10883000027191F8B111417160E0A168009801F5F1
:108840008C7105F07EF8A1680098E43105F076F8A7
:1088500054E00191029101F039FEA168304091F895
:10886000BC1001408DF80410000A8DF8050001A924
:10887000009805F070F841E0A068B0F84C1000983E
:1088800005F076F8A068B0F8F010009805F074F8DC
:10889000A068B0F8481000E015E0009805F070F806
:1088A000A068B0F8EE10009805F06EF826E0A16818
:1088B00091F8AE0101280098B8D011F8662F027126
:1088C0004978B8E712E00191029101F0FFFDA1683B
:1088D000304091F8BC1001408DF80410000A8DF86A
:1088E000050001A9009805F031F807E0A06890F8AC
:1088F0008F21D0F89011009805F012F8FCF712F9CA
:10890000002804D140F6FC113120FBF76BFAFEBDC4
:108910001C0100202DE9F047874C82468946A0685B
:108920000088FBF79DFE06000AD060884FF0000526
:10893000C005A06809D5A0F8A45080F80C5108E043
:1089400040F6A2513120FBF74DFA30F8A41F491C24
:10895000018001F0E3F84FF0010820B360880005C2
:1089600006D5A06890F8831011B1C0F898501AE0AD
:10897000A068D0F89810491CC0F89810D0F89C3026
:108980008B4201D35A1A00E00022A7887F1DBA4209
:1089900001D880F8A280994205D3C0F8985080F899
:1089A000FA8101F0E9F960884FF0020710F4407F86
:1089B0000ED0A06890F8811011B1032908D102E00F
:1089C00080F8818001E080F881700121FEF736FD9A
:1089D000A06890F88110012904D16188490501D56A
:1089E00080F88170BAF1000F76D1A178490602D5DE
:1089F000A0F8205104E0B0F82011491CA0F8201183
:108A00004846FFF7BBFD40EA09008146FFF720FD1D
:108A1000A768B7F80001401CA7F8000197F8040107
:108A200028B1FCF7AFFAB0B1A7F8005113E0FCF79A
:108A300021F908B1A7F80051FCF716F958B197F8D9
:108A40000C01401CC0B287F80C01022803D9A7F81A
:108A5000005187F80C51A0680123002190F87E2076
:108A6000703004F0AFFC20B9A06890F87E000C28AC
:108A70005ED1A0680123002190F87D20703004F0C1
:108A8000A1FC50B3A0680123002190F88020703031
:108A900004F098FC08B3A06890F88110022947D12F
:108AA00090F80C01C8B9304603F06DFFA8B1A0687A
:108AB000703005F0A8FF80B9A168B1F8FA0001286C
:108AC00036D981F80281B1F8A620B1F8A400931E2E
:108AD000984203DB012004E01CE029E0101A401E4C
:108AE00080B2B1F80021A3889A4201D3012202E0AA
:108AF0009A1A521C92B2904200D91046012801D114
:108B000081F80251A168B1F874201044A1F8FC006A
:108B100001F0CEF8A0784A46C0F38011504601F02B
:108B200011F8A06880F80351BDE8F047FBF7E4BFF7
:108B30000120A168E4E700001C0100207CB5584C2E
:108B400001230021A06890F87D20703004F03AFCE9
:108B500000287DD0A06890F8B511002539B100211A
:108B60000E2000F09FF8A06880F8B55195E090F8CD
:108B7000B41119B190F8B610890716D090F8A41165
:108B80008DF80410019901919DF8041041B190F8FD
:108B9000A5118DF80010009900919DF8001089B181
:108BA00090F8AE1101292FD071E000210C2000F0C7
:108BB00079F8A06810F8B61F41F00101017080F843
:108BC000FE506AE090F87E1024291BD090F87D10AA
:108BD000242917D05FF0000300F5CB7200F5D271A5
:108BE00004F0E7FFA06880F8A4510021142000F0F1
:108BF00059F8A16801F12C00C28B21F8EE2F408CAE
:108C000048804AE00123E7E790F8AF118DF80010A3
:108C1000009900919DF8001031BB90F87E2001234F
:108C20000B21703004F0CEFBF0B9A06890F86A0018
:108C300005F0F1FE0546A06890F86B0005F0EBFE2C
:108C40000646A06890F8B011284605F0EFFE00E057
:108C50001EE050B1A06890F8B111304605F0E6FE74
:108C600018B1002000F01CF911E0A06801230321D5
:108C700090F87E20703004F0A5FB40B9A068012375
:108C8000022190F87E20703004F09CFB08B1002097
:108C90007CBD0021162000F005F801207CBD0000FD
:108CA0001C01002070B50D4C06460D46A0687030C2
:108CB00005F0A9FE20B140F60F213120FBF792F814
:108CC000A268002082F8EC6015B1A2F8B00070BD77
:108CD00022F8AA0F0120107170BD00001C010020B5
:108CE00070B51A4D0026AC6894F87B0101280AD0B3
:108CF000022829D194F8B4000621A0B184F8EE101E
:108D0000012102201BE094F8C40100281CD100229C
:108D100004F5BE7004F5887104F1D00304F00AFB79
:108D2000012105200BE094F8BC00400705D5112077
:108D3000032204F8EE2F617000E00D200121FFF7FF
:108D4000B1FFA86880F87B6170BD00001C010020A5
:108D500070B52B4A03465088184350801046402B6C
:108D600080680DD09E074FF000054FF001044FEAD8
:108D7000C3760CD54EB140F60F513120FBF732F8D7
:108D8000BDE870400421FEF759BBD1601CE0C6B1BC
:108D90001161C978062902D00B2912D109E090F897
:108DA0007E1017290DD10021C0E9301180F88240D2
:108DB00007E090F87E10112903D180F8825080F8E6
:108DC000B440990716D5D168C978052902D00B2976
:108DD00010D109E090F87E1015290BD10021E0E9AF
:108DE000321100F8454C05E090F87E10102901D1B1
:108DF00080F88350980601D50820507070BD00009F
:108E00001C0100202DE9F041244C0125A26892F8B4
:108E1000960108B1012700E0002792F8971109B1E7
:108E2000012600E000260FB992F86A000EB992F808
:108E30006B1002F16203187259720120987292F855
:108E4000AE01012801D007B916B1002000F028F8C2
:108E5000A0682C3004F01CFF0646A06804F0C4FE95
:108E6000C0B1A0682C3004F013FFA168074601F5DB
:108E7000ED7208882C3104F078FEBE420AD2F8F771
:108E8000ABFB0146B81B642800D26420F8F7E2FA75
:108E900000B100252846BDE8F08100001C0100203B
:108EA00010B5104CA1680A88A1F8062281F80402C6
:108EB00091F86A0005F0AFFDA16881F8080291F809
:108EC0006B0005F0A8FDA26802F2022182F80902F7
:108ED00001200870002082F8AE01BDE8104000F0CB
:108EE0004BBF00001C01002010B5154C01230021D0
:108EF000A06890F87E20703004F064FA90B1206988
:108F000004F0A7FCA168A1F89401B1F8741005F071
:108F10009BFD48B1A068282180F89510763001218A
:108F200081770BE0012010BDA168206901F5CB71AC
:108F300004F08AFCA1680B2081F87E00002010BD9F
:108F40001C01002070B5294C01230021A06890F875
:108F50007E20703004F036FAB8B10021206904F0A8
:108F60004BFCA0B12069A168B0F80D00A1F89401F4
:108F7000B1F8741005F068FD68B1A068282180F888
:108F800095107630012181772EE0012070BDBDE87B
:108F9000704000F0ADB8206904F05EFC04F0F5F913
:108FA0000546A0682946C0F89C512069007904F064
:108FB00077FBA168A1F8960120692946B0F8050061
:108FC00004F06AFBA168C1F89801206904F047FC2D
:108FD000A168A1F8A001206904F044FCA168A1F8EF
:108FE000A2010D2081F87E00002070BD1C01002030
:108FF00038B5294C01230021A06890F87E207030FC
:1090000004F0E0F970B9A06890F87E20122A09D027
:1090100001230521703004F0D5F908B1082038BDCE
:10902000012038BDA06890F8B40008B9FFF7CAF86D
:10903000A168206901F5887104F023FCA16820690A
:10904000E03104F015FCA16891F8CC018DF8000026
:10905000009800909DF8000020B14FF42871312055
:10906000FAF7C0FE0888A1F8CE0101F5E871206981
:1090700004F002FCA168206901F5EC7104F0F5FB35
:10908000A0680146012280F8CC21142081F87E00DE
:1090900000F072FE002038BD1C0100201CB5134CEE
:1090A000A06890F87F00C00701D001201CBD694670
:1090B000206904F0ECFB01F009FA44F62F11084096
:1090C0009DF80020A168024001F8BC2F9DF8012006
:1090D00002EA10204870FFF775F8A06810F87F1FAB
:1090E00041F00101017000201CBD00001C010020A6
:1090F0000A4A10B5906890F87F100B0701D501203F
:1091000010BD41F0080180F87F101169C97880F81E
:10911000E910FFF757F8002010BD00001C010020E7
:109120002DE9FC41344CA06890F87F0010F0300F1E
:1091300002D00120BDE8FC81206904F0C3FB18B314
:10914000206904F0B1FB0746206904F0B1FB064634
:10915000206904F0A7FB0546206904F0A7FB01463F
:109160000097A06833462A462C3004F0CBFDA07847
:10917000800703D5E068C078142809D0A06890F86B
:109180007D001C2804D007E0BDE8FC41FFF7B0BF1C
:10919000A168012081F86000A16891F860000128B1
:1091A00011D091F8A5018DF80400019801909DF867
:1091B000040040B991F8A4018DF8000000980090D7
:1091C0009DF8000028B111F87F0F40F010000870E2
:1091D0000DE091F87F0001F5F47240F0200081F875
:1091E0007F0031F82C0B04F094FD00F0C5FDFEF774
:1091F000E9FF00209EE700001C010020F8B51A4C92
:1092000001230A21A06890F87D20703004F0DAF87C
:1092100038B3206904F056FBC8B1206904F044FB60
:109220000746206904F044FB0646206904F03AFB37
:109230000546206904F03AFB01460097A0683346D2
:109240002A462C3004F05EFDA06804F0CDFCA16835
:10925000002081F8AE0081F87D00FFF777F900204B
:10926000F8BD0120F8BD00001C01002010B5094C1C
:10927000A06890F87F00400701D5012010BDFEF7DF
:10928000A1FFA06810F87F1F41F0040101700020C9
:1092900010BD00001C01002010B5094C012309215C
:1092A000A06890F87D20703004F08CF8002806D07B
:1092B000A168002001F8A20F087301F8250C10BD69
:1092C0001C01002010B50F4C01230021A06890F86C
:1092D0007E20703004F076F838B1FEF773FFA16895
:1092E000102081F87E00002010BDA0680123052118
:1092F00090F87E20703004F065F808B1082010BDA9
:10930000012010BD1C0100200648806890F87E10E6
:10931000112901D002207047122180F87E10002010
:10932000704700001C010020F8B5344C01230B21CC
:10933000A06890F87E20703004F044F878BBA068F4
:109340000123002190F87E20703004F03BF820B318
:10935000A06890F87D00242822D0206904F0CEFA7D
:1093600000B3A06890F8BC1041F0040180F8BC1074
:1093700021694A7902F0070280F86320097901F037
:10938000070180F8621090F8AF318DF80030009B33
:1093900000939DF8003043BB08E00120F8BDFFE7D3
:1093A0002020FBE7BDE8F840FFF7A2BE90F8AE3101
:1093B000012B1AD000F16A0301255E788E4206D196
:1093C0001978914203D1022180F8AE110DE000F529
:1093D000FF71028821F8022990F862200A7190F842
:1093E000630048710D7000F0C7FCA168212081F86E
:1093F0007E00FEF7E7FE0020D0E700001C01002001
:109400002DE9F8434E4CA06890F87D10202909D032
:109410005FF0000790F87E10222905D087B300F195
:109420007D0503E00127F5E700F17E0510F8BC1F7C
:1094300041F0040101702069FCF754FD4FF0010870
:10944000002608B339462069FEF786FFE0B16A4678
:109450002169A06804F0DAF888B3206904F02AFAD8
:10946000A168A1F89401B1F8741005F0EDFA38B3D1
:10947000A068282180F89510763080F81E8053E08F
:10948000FFE70220BDE8F883A0684FF0000990F8DC
:10949000AE11012915D080F8AE61F7B12069A1683D
:1094A000C07881F8EA0008FA00F2C2F3006060B107
:1094B0000A2081F87D0091F8AE00A0B908E014E020
:1094C00027E01E20FFF7ECFCE7E740F2CB3101E09C
:1094D00040F2D3313120FAF785FC2E70FEF77EFE84
:1094E000FFF706FE81464846CCE7A06890F8AE112B
:1094F000012909D080F8AE61A06800F17E018D429B
:1095000012D180F87E600FE00020FFF7C9FC2E70BA
:10951000F2E7A0689DF8001080F896119DF8011000
:1095200080F8971124202870A06800F17E018D42F8
:1095300002D1FEF753FE01E080F8AE600020A1E703
:109540001C01002010B50A4CA06810F8BC1F41F0A7
:1095500004010170206904F0DBF9162801D0002015
:1095600010BD206904F0D6F9BDE81040FEF708BE32
:109570001C010020024800690079FEF701BE0000CE
:109580001C01002010B5084CA06890F87E00172838
:1095900001D0022010BDFEF721FEA1681B2081F83A
:1095A0007E00002010BD00001C01002010B50B4CF7
:1095B00001231946A06890F88020703003F002FF64
:1095C00008B1002010BD206904F078F9A16881F885
:1095D0007A01072081F88000F3E700001C010020D9
:1095E0002DE9F041374D00262846A968006901277A
:1095F00091F87D3000790E2B01D1122806D0314A26
:1096000000249268BC321C2B04D005E0FFF744FE16
:10961000064653E0142802D0042B0BD00CE081F84E
:109620007D4081F8AE400521104605F09EF9FEF719
:109630008DFF43E00E2802D0202B0FD010E081F8E0
:109640007D4081F8AE400888A1F80E021A2081F80A
:109650000C0281F80A7200F08FFB2FE0162806D06A
:10966000262B01D1162802D0172814D026E001F8A5
:109670007D4F81F83140487821281FD008211046BD
:1096800005F073F9A8680B21BC3005F06EF91A20BB
:10969000FFF706FC12E091F87E0022280ED181F837
:1096A0007E40FEF79BFDA86890F8AE01012802D12C
:1096B0000020FFF7F5FBA86880F8AE413046BDE812
:1096C000F08100001C01002070B52C4CA06890F8BF
:1096D0007F10890707D590F87D200123082170307D
:1096E00003F070FEE8B1A06890F8B600800712D4CD
:1096F000206904F0E5F8A16881F8B700206930F826
:10970000052FA1F8B8204088A1F8BA0011F8B60FCB
:1097100040F002000870A06890F8B610C90702D0A7
:1097200010E0012070BD90F87F108A0704D54FF437
:1097300037713120FAF756FB41F0020180F87F10B3
:10974000FEF740FDA068002590F87D10062905D1A0
:1097500080F87D5080F8AE5000F00EFBA06890F8C5
:10976000B41149B180F8B45100F006FBA06890F83C
:109770007D1009B980F8AE50002070BD1C0100209A
:1097800010B5174CA36893F8F20008280ED200F128
:109790000802C0F10800C1B2981800F58870FAF705
:1097A000ADFBA16811F8F22F10440870A36893F87C
:1097B000F2000838042811D2021DC0F10400C1B221
:1097C0009818E030FAF79AFBA068002180F8F210B0
:1097D0000121BDE810400420FFF764BA10BD00006D
:1097E0001C01002004482721806880F87D1000219A
:1097F00080F88C11704700001C010020094810B54A
:10980000806890F87E10142904D040F29A613120CB
:10981000FAF7E8FA012180F8B310152180F87E10DC
:1098200010BD00001C01002010B50A4CA06890F883
:109830007F00C00708D0FEF7D1FCA06810F87F1F9A
:1098400021F00101017010BD40F283613120FAF76F
:10985000C9FA00001C01002010B50A4C01230021A8
:10986000A06890F87D20703003F0ACFD20B1A168B5
:109870001C2081F87D0010BD4FF4E1613120FAF722
:10988000B1FA00001C0100200A4810B5806890F869
:109890007F10C1F30112012A04D040F20F71312070
:1098A000FAF7A0FA21F0100180F87F10BDE810400F
:1098B000FEF794BC1C01002010B50A4C01230021C6
:1098C000A06890F87D20703003F07CFD20B1A16885
:1098D0000E2081F87D0010BD40F2FB613120FAF7C7
:1098E00081FA00001C0100200448806810F87F1FE6
:1098F00021F004010170FEF771BC00001C01002082
:10990000094810B5806890F87E10102904D040F204
:1099100092613120FAF766FA012180F8B310112123
:1099200080F87E1010BD00001C01002010B50A4C0C
:1099300001230021A06890F87D20703003F042FDE3
:1099400020B1A1681F2081F87D0010BD40F21B717D
:109950003120FAF747FA00001C010020084810B532
:10996000806890F87E10212905D021B140F2227143
:109970003120FAF737FA222180F87E1010BD00005E
:109980001C010020074810B5806890F87E1015294A
:1099900004D040F2A7613120FAF724FA192180F8A7
:1099A0007E1010BD1C010020074810B5806890F89B
:1099B0007E10152904D040F2A1613120FAF712FA85
:1099C000172180F87E1010BD1C01002070B51B4DC2
:1099D000A86890F87E101B2902D040F2C16107E010
:1099E000002480F8B34090F8C41121B140F2C56161
:1099F0003120FAF7F7F990F8B41041B180F8B4408B
:109A00000188A0F8C81180F8C6410C2108E001883F
:109A1000A0F8C81180F8C641012180F8CA110B21B5
:109A200080F8C4110088FAF705FE03F045F900F04C
:109A3000A3F9A86880F87E4070BD00001C010020DA
:109A400010B5084C01231946A06890F880207030AA
:109A500003F0B8FC002803D1A168082081F8800039
:109A600010BD00001C010020144810B5C1688068BA
:109A7000097990F87D200A2A09D190F8EA208A42D3
:109A800005D1002180F87D1080F8AE1010BD90F84F
:109A90007F20130707D522F0080180F87F10BDE86A
:109AA0001040FEF79BBBFF2904D040F27D613120BE
:109AB000FAF798F9BDE81040FFF794BE1C010020AA
:109AC00010B5154CA06890F8B610890711D490F81D
:109AD0007D2001230021703003F074FC20B1A168C7
:109AE000062081F87D0009E040F2E7613120FAF7B5
:109AF00079F9002180F8AE1080F8B411A06890F8D0
:109B00007F00800707D5FEF769FBA06810F87F1F6C
:109B100021F00201017010BD1C010020084810B5A1
:109B2000806890F8831041B990F87E2001230621C7
:109B3000703003F047FC002800D0012010BD000069
:109B40001C010020F8B5594C06461546A06809B11D
:109B5000002104E0B0F80E11B0F8FE201144A0F886
:109B60000E1190F878118DF80010009900919DF871
:109B7000001039B990F8802001231946703003F0A5
:109B800021FC30B1A06830F8A81FB0F8562011446D
:109B90000180A06890F8AE2032B1B0F8AA10B0F8F9
:109BA000FE301944A0F8AA1090F9B230002B06DD5F
:109BB000B0F8B010B0F8FE703944A0F8B010012130
:109BC0003D2716B180F8957012E02478022C09D058
:109BD000012C11D03DB300F194021170E9060ED5AD
:109BE0001E2118E090F8EE20062A44D0162242E00A
:109BF00000F19402117047E090F87A213BE02907C8
:109C000002D580F895703FE0A90601D5232102E036
:109C1000A90703D02A2180F8951035E040F6BC4111
:109C20003120FAF7DFF82AB1B0F8AA20B0F8AC403A
:109C3000A24216D2002B05DDB0F8B020B0F8AC304F
:109C40009A420ED2B0F8A830B0F8A62093420AD3B8
:109C500090F878318DF80030009B00939DF800302B
:109C60000BB1222207E090F881303BB1B0F8A4306C
:109C7000934209D3082280F89520B9E7B0F8A420D0
:109C8000062A01D33E22F6E790F894108DF80010D2
:109C9000009900919DF8001019B1BDE8F84004F05A
:109CA000A3BEBDE8F8400021FDF7C8BB1C010020A1
:109CB00070B52D4DA86890F8811051B1012908D0D8
:109CC000022909D0032907D040F67A213120FAF77A
:109CD00089F8B0F8FC1035E090F88010082934D0ED
:109CE000B0F8A410B0F8A62000248B1C9A4206D32A
:109CF000511A891E0C04240C01D0641EA4B290F8E1
:109D0000A21039B190F87D2001230921703003F0B1
:109D100059FB30B3FFF702FF68B1A9680020983102
:109D200006C98B1C9A4203D3501A801E00D0401ED5
:109D3000A04200D284B20CB1641EA4B2A868B0F8EC
:109D4000FC102144A0F8F81070BDB0F8A41003294D
:109D5000BFD330F8741F428E1144491CA0F8841000
:109D600070BD0024EAE700001C01002001490870D2
:109D7000704700009B02002001480078F9F75ABEA6
:109D80009B02002003498A88028089788170002024
:109D900070470000200F00203EB50C4605460088A5
:109DA000694603F0E5FA01004FF0000005D0C4F861
:109DB0000200A071208002203EBD019911F17001C6
:109DC00081F84E00D1F81620C4F802208A7EA271D4
:109DD0002A88228091F84E208DF80820029A02925B
:109DE0009DF80820002AEBD100203EBD1CB500885C
:109DF000694603F0BDFA00280BD10B48007888B102
:109E0000019805F016FD28B1019890F8B50118B138
:109E10003A201CBD02201CBD0199012081F8B5012A
:109E200000201CBD11201CBDF801002010B5044607
:109E300005F0F6FC30B1044881882180C08860803C
:109E4000002010BD012010BD000200203EB50546D7
:109E500000F03CFBC0F3002010B3002402A88DF8F2
:109E600004408DF808400090AA786978287801AB02
:109E700005F030FD002812D19DF8040005F031FCFA
:109E800080B19DF8080005F02CFC58B106489DF8FB
:109E9000041081749DF80810C174848200203EBDB6
:109EA00001203EBD11203EBD200F0020017879B178
:109EB000417869B141881B290AD381881B2907D3BE
:109EC00004490268C1F802208088C88000207047D9
:109ED00012207047200F0020006840F2E2418842C3
:109EE00003D30349886000207047122070470000A8
:109EF000200F0020034AD2E90012016042600020D6
:109F0000704700006CA3000010B5052000F0D4FAE3
:109F1000FDF756FE02490148486010BDAD9F0000A4
:109F2000F801002010B503F077F9FBF773FC00F09F
:109F3000DDFA0F484FF6FF710E4BC18101820021FF
:109F4000C175018301801B221A804FF4A4745C80C8
:109F50009A80DC808174C174032383700223C370F0
:109F60008280C28040F6A66282608175017310BD56
:109F7000200F00200002002010B558B10A490A78CD
:109F80006AB10022427003230370012303710A7037
:109F9000184610BD41F646113920F9F723FFBDE8F8
:109FA0001040FBF7CFBF0000200F00202DE9FE4F2F
:109FB00092460F46814605F033FC002863D03349B2
:109FC000B9F85420B9F852600888904200D310467E
:109FD00080468888B04200D206464C8840F6480049
:109FE000844200D30446CD88854200D3054684428E
:109FF00000D304464FF4A4711B2E01D08D4204D12E
:10A00000B8F11B0F3FD08C423DD06A4651464846BE
:10A0100005F08AFBBDF806004146404500D90846D8
:10A02000F880BDF80810A14200D80C463C81BDF86C
:10A030000210B14200D80E467E80BDF80410A9423D
:10A0400000D92946B98001223A701B38E02802D98C
:10A0500040F6724114E01B3EE02E02D940F67441F6
:10A060000EE04FF4E060A4F5A474844202D940F6F7
:10A07000764105E0A1F5A471814204D940F678410A
:10A080003920F9F7AFFEBDE8FE8F00000002002086
:10A090002DE9F04188B00C46064603F04CFF98B11C
:10A0A000304603F03BFF30B1B4F801101220002914
:10A0B0000BD0802909D8304603F01FFF40B130464D
:10A0C00003F097FE30B109E0422008B0BDE8F0810E
:10A0D0000C20FAE7304603F01BFFA8B3304604F02B
:10A0E000F2F80028F4D1304603F09EFE0028EFD1AC
:10A0F0003046FCF77BF9B4F8010042F2107100FB26
:10A1000001F8E178304603F0EFFE304603F002FF3D
:10A11000E8B10022114601A8FAF7D0F804006AD08D
:10A120000021FBF7A5FDBDF8040020802146304644
:10A1300003F014FF05F074FB3A4D002804F12C00E5
:10A140000FD0AA88E9880EE0FFE71220BDE742465B
:10A1500000213046FDF79AF80028B6D041F23B4185
:10A1600053E01B221146C2840185A868E06241F6D3
:10A170004C57304603F0D6FE10B9304603F0ECFEE3
:10A18000E7602188ADF80810A97C8DF80A10E97CF9
:10A190008DF80B10A98AADF80C1005A900910120CB
:10A1A00004AB02AA214605F0FCFA40B10021BDF83B
:10A1B0000400FAF7ADF8F0B141F2874125E09DF8CF
:10A1C00010008DF818009DF814008DF81900BDF8E6
:10A1D0000C00ADF81A0006A9204603F088F9E878CB
:10A1E0000090AB78EA88A9882088FAF75DF920B159
:10A1F00041F2924109E0092067E742462146304694
:10A20000FDF744F820B141F294413920F9F7EAFD15
:10A210000548436823B1002204F5D27120469847CF
:10A22000002052E7200F0020F80100202DE9F04126
:10A2300088B00446008806A903F09AF8002847D1A0
:10A240000798002790F8E8118DF8081002990291FC
:10A250009DF808108DF80C1090F87F10703089066A
:10A2600002D59DF80C1049B15FF000018DF8041083
:10A2700005214C3004F0F4FB10B104E00121F5E7B6
:10A280009DF8040018B32189E08805F03FFA002802
:10A290001ED1A188608805F039FA002818D12189DB
:10A2A000E08805F029FA002812D1A188608805F01D
:10A2B00023FA06000CD1079800F5D2754FF001087B
:10A2C00085F801809DF80C1029B13A262FE01A205C
:10A2D00008B0BDE8F081394603AA05F025FA618887
:10A2E000BDF81200814200D20846E880A188BDF87E
:10A2F0001400814200D208462881E288BDF80E1081
:10A300008A4200D2114669802289BDF810108A4223
:10A3100000D2114640F64802A980914200D311466E
:10A32000A980904200D202462A8185F800806F7091
:10A330003046CDE710B50446C188808805F0E6F9BF
:10A3400000280FD16188208805F0E0F9002809D1A4
:10A350000548A188818021880180E188C1806188C9
:10A360004180002010BD0000000200200BB0120B45
:10A370005900B0120807060504030200FCF8F4F0C7
:10A38000ECD8040300FCF8F4F0ECD80010B5FFF7AB
:10A39000EDFC0448406805F015FBBDE8104005F0F1
:10A3A00051B800000802002010B5074CA06805F065
:10A3B00009FBE06805F006FB02F02EFFFBF72AFA26
:10A3C000BDE81040FFF7AEBD0802002000B505490A
:10A3D000054805F0D8FA04480449001D5DF804EB6F
:10A3E00005F0D1BA180200200C0200202002002043
:10A3F00000B50849084805F0C6FA07480749001D96
:10A4000005F0C1FA0448064908305DF804EB05F090
:10A41000BABA0000440200200C0200204C020020C6
:10A420003C0200200148007870470000080200202C
:10A4300010B5FCF753F9FCF7BDFF0548FCF734F9FC
:10A4400005490448086006490448086010BD00003A
:10A45000A9130020AD64000028020020E55F000081
:10A460002C0200200C4910B501200870FCF766F999
:10A47000FDF7FEFC02F0BEFE0848FAF72BFC0020B8
:10A48000F9F78CFE07490648086008490648086045
:10A4900008490748086010BD08020020A9130020E1
:10A4A000814C000038020020F17B000034020020C3
:10A4B00059600000300200200121814002480268FA
:10A4C00011430160704700005402002001480068F9
:10A4D000704700005402002003480088C0F30020A9
:10A4E0004000401C704700005402002010B5F9F7EE
:10A4F000EDF80022084B114633F82140844203D383
:10A5000003EB8100827803E0491CC9B20C29F3D324
:10A510000248027010BD000016FA00009C020020E4
:10A5200070B5054616460C46022000F0F9F90649BA
:10A530000120F61E087005480660044808380560CA
:10A54000001F046070BD00009D02002010F5004057
:10A5500010B50C4C207880B10B494FF40000086016
:10A5600000F06AF8002120B10120607007480068FF
:10A5700001E061701020A0702170BDE81040002043
:10A5800000F0CEB99D02002008F5014000F4004023
:10A5900010B5022000F0C4F904490120087000F051
:10A5A00059F803494FF40000086010BD9D020020D7
:10A5B00004F50140034800210170417010218170B1
:10A5C000704700009D020020074810B5017841B196
:10A5D00000F032F818B105480068C0B210BD102074
:10A5E00010BD807810BD00009D02002000F40040E6
:10A5F000084810B5017859B10748D0F8000128B1D2
:10A6000000F00CF8002800D0012010BD022010BD81
:10A61000407810BD9D02002000F000400548D0F8B1
:10A62000041111B1D0F8080108B1002070470120D1
:10A630007047000000F00040054810B5D0F8000158
:10A6400020B1FFF7EBFF08B1012010BD002010BDC5
:10A6500000F0004004480021C0F80011C0F80411C7
:10A66000C0F808117047000000F00040084A10B51B
:10A67000C2E9020107491046F9F788FA002805D017
:10A68000401C03D07D214020F9F7ACFB10BD000039
:10A6900058020020C4A60000084A10B5C2E9020111
:10A6A00007491046F9F77EFA002805D0401C03D070
:10A6B00072214020F9F796FB10BD000058020020DF
:10A6C000C4A60000010000001011004000000000BE
:10A6D000000000000000000000000000074A10B564
:10A6E000537833B1064B1960191D08600120907032
:10A6F00010BDBA213C20F9F775FB0000A002002034
:10A700000CF50040094810B5017851B1807840B18E
:10A7100007490020C1F8040106494FF000700860A5
:10A7200010BDE1213C20F9F75DFB0000A0020020F4
:10A7300000F0004004F5014070B50B4C0025207876
:10A7400058B100F0E5F80948D0F8040118B10848FC
:10A750000068E07000E0E5702570002000F0E0F88F
:10A760006570A57070BD0000A002002000F00040E0
:10A7700000F400400D4810B5017891B1807880B1A7
:10A780000B490020C1F804010A4A4FF40030106060
:10A79000D1F80021012A03D14A600649091D086049
:10A7A00010BDD1213C20F9F71DFB0000A0020020C4
:10A7B00000F0004004F501400348002101704170A1
:10A7C0008170C17070470000A00200202DE9F041A7
:10A7D00005461C4690460F46012000F0A1F8124E97
:10A7E000124834710760114945EA0440091F40F0DE
:10A7F0008070086001F013FB38B90C481030016814
:10A8000021F0FF0141EA0801016000F081F83DB943
:10A810000848074A0649FC3AC0F81015C0F8142544
:10A8200001207070BDE8F081A002002008F5004012
:10A8300000F1004088F00140084810B5417849B166
:10A840000121017006480022C0F80021C0F8002252
:10A85000016010BDC5213C20F9F7C4FAA002002018
:10A8600000F000400648017841B10648D0F80401E4
:10A87000002802D004480068C0B27047C078704712
:10A88000A002002000F0004000F400400149012037
:10A890008860704700F000402DE9F04700282ED076
:10A8A00018480078B0B1184DD5F80401002826D119
:10A8B0000227C5F80473154C2068C04340F3001606
:10A8C000206840F0100020604FF400484FF0E0296D
:10A8D000761C09E040F253113C20F9F783FA00BFDF
:10A8E000C9F88082F9F7FCF8D5F804010028F7D000
:10A8F0001EB9206820F010002060C5F80873BDE87C
:10A90000F0870000A002002000F0004010ED00E001
:10A9100002490148086070470000020208F5014042
:10A9200010B5044600F022F8002C17D00C4A0C4851
:10A930000C4914320C4B012C05D0022C08D0832179
:10A940003D20F9F74FFA022404601160200604E06C
:10A950000324046011604FF40000186010BD000073
:10A9600000F50040AB14002004F50140044800212C
:10A970000160016003494FF02070086070470000DB
:10A9800000F5004008F501400548D0F8001221F01C
:10A990004001C0F800120349002008607047000021
:10A9A0000010004060150040044908600448D0F8D9
:10A9B000001241F04001C0F80012704760150040DD
:10A9C00000100040014890F822007047640F0020FA
:10A9D000F8B51E4CD4F804031027C0F30016C4F8D1
:10A9E00008730220C4F80002194800251A4980F8AB
:10A9F0002C501848086019480068B0B1FF208DF845
:10AA00000000C4F810510120206104E09DF800000E
:10AA1000401E8DF800009DF8000018B1D4F8100118
:10AA20000028F3D09DF8000050B100F0B1FCC4F84C
:10AA3000105100F029FE002E01D0C4F80473F8BDB7
:10AA400040F2A3713E20F9F7CDF90000001000405C
:10AA5000640F002000000E0C08F501405015004066
:10AA60002DE9F0411F4C0746884694F82C00C10799
:10AA700018D01D4A4FF0406111601C4DD5F80012EE
:10AA800041F00101C5F8001240F0020084F82C00EA
:10AA9000404600F05DFE00F029FC01263FB1012F89
:10AAA0000ED016E040F22D613E20F9F79BF94046AA
:10AAB00000F03CFC404600F0FDFB66722E6008E0B2
:10AAC00000F05CFC00F0AAFD0220607200F0D2FCF5
:10AAD0006E600748C664074801683846BDE8F04123
:10AAE00005F050B8640F002004F50140001000404C
:10AAF000008000404C8500402DE9F047354D06466A
:10AB00004FF0406089462860334C94F82C0040F0A8
:10AB1000020084F82C00084600F01AFE00F0E6FB64
:10AB2000DFF8B880002716B1012E27D03FE0484655
:10AB300000F0FCFBE079012805D1D8F8001241F0C3
:10AB40000801C8F80012484600F0B4FB012060720A
:10AB5000A06A40F48010A0624FF4801028604FF487
:10AB60007A71B9F1020F07D040F6340049F6EC7261
:10AB70001044B0FBF1F71AE00846F7E700F0FEFBDF
:10AB800000F04CFDE079012805D1D8F8001241F021
:10AB90000401C8F8001202206072A06A40F400109C
:10ABA000A0624FF400102860292700F063FC00F039
:10ABB0004DFC01F00BF80068012806D0002130465A
:10ABC00004F0E0FF3846BDE8F087FFF701FF002002
:10ABD000F9E7000004F50140640F00200010004078
:10ABE000024A136B0360506B08607047640F0020CB
:10ABF00010B51DC8014981E81D0010BD540F00208B
:10AC00000E4910B5CA69824202D34FF402610AE0CC
:10AC100001220A7308610A494A640A4A1368834296
:10AC200004D340F629013E20F9F7DCF80023C1F8EF
:10AC300044311060BDE8104000F0FEBC640F0020FD
:10AC4000008000404485004070B5104C064602204C
:10AC50002073962500F066F8024694F8210094F8D7
:10AC6000201001280DD0284604F0A4FF08492061D7
:10AC70000020C1F844012169E069084405490860E1
:10AC800070BD3346284604F0B1FFEFE7640F0020A3
:10AC9000008000404485004010B501F0DCF8002839
:10ACA00006D00448016821F0010141F08071016083
:10ACB00010BD0000741700402DE9F041382200213A
:10ACC000134801F078F900F0DFFC01F07DF8114D38
:10ACD000104E00240F4F0835103628B901F08BF8BC
:10ACE00010B901F092F808B1242206E001F0CDF885
:10ACF00010B901F0C0F840B14022FF21384601F000
:10AD00005AF92C603460BDE8F0813822F5E7000084
:10AD1000640F0020000E00400148C0697047000029
:10AD2000640F0020144810B590F82110407A41B10A
:10AD300002290BD0022809D001290BD0012809D003
:10AD400015E00028F6D14FF4D9710DE0BDE81040B0
:10AD500000F016BC0948006800F00F00032806D078
:10AD6000042806D040F2E7113E20F9F73BF8012015
:10AD700010BD022010BD0000640F0020101500401F
:10AD80000148806970470000640F002010B500F092
:10AD900061FCFFF71DFE04F08BFE0F480F4A816A2D
:10ADA00041F480011160002484620473C4618461F1
:10ADB00000F050FC0A48C0F84841C0F84441C0F8CF
:10ADC0004041C0F84C41012004F0ABFEBDE810400A
:10ADD000012004F099BE0000640F002008F5014036
:10ADE000008000402DE9F041012004F09AFE38482F
:10ADF000002404600126066001F01DF8354D18B1ED
:10AE0000286840F48060286001F009F828B12868BB
:10AE1000314920F069000843286001F01CF838B17E
:10AE20002C48001D016821F47F4141F4B0510160BC
:10AE300028492A483C310860F8F7C0FE40B14FF07D
:10AE40008050D0F83003411C02D0224910310860F4
:10AE50004FF01020006E411C04D021490A6860F3B5
:10AE600017420A601E4940F25B6054390860091FAE
:10AE700040F203100860081F0660012000F068FC23
:10AE8000174940F20110C4310860164E0225C6F879
:10AE900000521649144808601548164F06F500760A
:10AEA00004861030C46180F82C403C70012004F00E
:10AEB0002BFE1020C6F804014FF0E020C0F800512E
:10AEC0007868002802D0BDE8F0410047BDE8F08175
:10AED000FC1F00403C170040960000802C000089B9
:10AEE0008C1500400010004000000E0C08F50140D9
:10AEF000540F0020700200200149087570470000BF
:10AF0000640F002004490860044810F82C1F41F029
:10AF10000101017000F062BA04150040640F0020C6
:10AF20002DE9F047354E07464FF040608A461446FB
:10AF30003060104600F00CFC00F0D8F9DFF8C0904B
:10AF4000304D4FF0010827B1012F1DD040F2227182
:10AF50004AE0204600F0EAF9204600F0ABF9022C66
:10AF60000FD040F6340000BF49F6F8510144504676
:10AF700000F092FB0446484600F07AFB85F8098011
:10AF800014E04FF47A70EFE700F0F8F900F046FBB8
:10AF900000F070FA49F6BA71504600F07DFB0446A5
:10AFA0001748001D00F064FB022068721648046018
:10AFB00017491648C1F81005A86A40F40020A86295
:10AFC0004FF0006030601021C9F8041300123060A7
:10AFD00000F03CFA0F49C1F84C800B480C30006877
:10AFE000A04204D340F249713E20F8F7FBFE21460F
:10AFF0003846BDE8F04704F0C5BD000004F5014047
:10B0000000100040640F0020408500404081004057
:10B0100098F00140008000400D4B10B5D8719A7235
:10B0200051B102201872012808D002280FD040F632
:10B030002A113E20F8F7D6FE0120F3E7587A0228BD
:10B0400005D100F09BF9BDE8104000F0E7BA10BD53
:10B05000640F0020014900200860704740850040CF
:10B060000A4908B5D1F81C21012A01D0002008BDE9
:10B07000074A126802F07F02524202700020C1F8B3
:10B080001C01044800680090012008BD0010004029
:10B09000481500401C110040034A010E116002498E
:10B0A0000002083908607047241500400068024912
:10B0B00020F07F40086070473C15004010B500F05C
:10B0C00023FB06480068032801D00B2804D140F276
:10B0D0008A213E20F8F786FE10BD00005015004082
:10B0E0000149487570470000640F00202DE9F047C2
:10B0F000514D0127EF645148D0F800905048006846
:10B10000504CC4E90C0900F043F94F49A06A0860AB
:10B11000DFF838A10026A662DAF8001240F21D120C
:10B120009143CAF8001284F82C60DAF80C0100B9D7
:10B13000AF6400F0B1F905464048001F0068E061C7
:10B14000FFF7F0FD84F82000607A84F82100A66102
:10B150003F4EA80701D53068A061280701D53068A7
:10B16000A0614FF000084946284600F01DFA18B9C2
:10B17000CAF810704FF00108324FE807A7F1100726
:10B1800002D03868804731E0A80726D568071ED46A
:10B1900000F061FED8B900F04EFEC0B92D4800683D
:10B1A000C0F3425CC0F3006300F00F02C0F3031170
:10B1B000C0F303205BB10AB101B140B92548001DBD
:10B1C000006820B1BCF1030F01D245F0040545F33E
:10B1D00080004146401C7A6807E015F0280F05D032
:10B1E00045F34011BA684046491C9047E80601D52E
:10B1F000F8688047607A02281BD1207B002818D08D
:10B20000022804D0012806D040F6033109E0216964
:10B21000E069084408E0E1692069884204D840F602
:10B2200004313E20F8F7DEFD3060BDE8F04700F065
:10B2300003BABDE8F0870000008000404C85004064
:10B2400004B50040640F002008F5014000100040E4
:10B25000448500405014004070B5114B8C8803EBBE
:10B260008003C3F820460C78D1F8011044EA01218C
:10B27000C3F800160B4D296800F10806012404FAF2
:10B2800006F332B1012A06D040F2C1413E20F8F760
:10B29000A9FD994300E0194384400C432C6070BD24
:10B2A000001000404016004001490120087070471E
:10B2B0007002002010B5044600F0CDFD00280ED02D
:10B2C000094A11685006022CD0F8200308D0C0F3B8
:10B2D000062000BF21F4FE4141EA0020106010BDAD
:10B2E000C0F30660F6E70000881500400D48407D79
:10B2F000252807D0262807D0272807D00A2807D8CE
:10B30000042206E0022107E01A2105E0502103E0B3
:10B31000062202EB4001C9B2034A116002494C31D6
:10B3200008607047640F002008150040124908B5F6
:10B3300091F91420497D01280AD002280AD0042856
:10B340000AD008280AD040F2DA310620F8F74AFD80
:10B35000002004E0012002E0032000E002206B4610
:10B36000F5F748F818B140F2F3413E20EEE79DF9B9
:10B37000000000F0E7F908BD640F00200348017ADF
:10B38000012902D1807AFFF7D1BF7047640F0020F6
:10B390000548407A012803D0022803D104F070BB8D
:10B3A00004F07ABB70470000640F0020094808B51C
:10B3B0000021C0F80011C0F80C11C0F81011C0F83D
:10B3C0000411C0F81411C0F8181103480068009067
:10B3D00008BD00000010004018110040164810B5CC
:10B3E00090F82C00C10726D0810713D51348D0F858
:10B3F000001241F00101C0F80012114800680B284A
:10B4000005D00A2803D0032801D0022813D140F226
:10B4100023510DE040070ED508480A490830C1F80D
:10B4200014050948D0F84001012804D140F22A51FE
:10B430003E20F8F7D7FC10BD640F0020001000403C
:10B440005015004098F00140008000400848014637
:10B45000C27991F82C1012B1012A03D006E041F014
:10B46000020101E041F0040180F82C10FFF7B6BFA3
:10B47000640F002010B500F0EEFC002808D100F0A9
:10B48000DAFC002804D10348016841F4C0210160BE
:10B4900010BD00006815004038B5324D0024287BEF
:10B4A00020B13148D0F84401012807D00022697A40
:10B4B0002E48012904D002290AD019E00122F6E71A
:10B4C000D0F80C11012901D0002411E008240FE06C
:10B4D000D0F80C11012906D00021254B1B68012B47
:10B4E00003D0042402E00221F7E700240C431443B4
:10B4F00014F00B0F05D1D0F81011012929D000212B
:10B500000C431C490978D1B11B49096811F0FF0FA0
:10B5100003D0D0F81421012A00D0002285F822207F
:10B5200011F0FF0F03D0D0F81801012800D000203F
:10B5300085F823000E481030006885F82400FFF7D6
:10B5400035FFE00609D5200707D4687A012802D024
:10B5500003E01021D4E744F020040848006800907C
:10B56000204638BD640F00200080004000100040DD
:10B57000001400407002002040160040448100404A
:10B58000084810B5006800F00F00032806D0042812
:10B5900006D040F212213E20F8F724FC012010BD15
:10B5A000022010BD101500402DE9F041194C0D4648
:10B5B000217A29B110F0110F0BD0FFF709FA27E01B
:10B5C00015494FF04060086000F05EF800202073DD
:10B5D0001EE0012901D0012600E00026E0790128C3
:10B5E0000ED0002700F050F89621304600F062F8A7
:10B5F00001464FB13B358D4204D90020BDE8F081B2
:10B600000127EFE70120E071A27A3046FFF788FCBE
:10B610000120F3E7640F002008F5014005480021F0
:10B62000C0F81C11D0F8001241F48871C0F8001263
:10B6300070470000001000400448816A41F4800116
:10B64000816203494FF4800008607047640F002056
:10B6500004F50140054900200860091F0860091F22
:10B6600008600249091D08607047000048850040D5
:10B670000349C979002902D10249C1F8140570476C
:10B68000640F002098F0014002480021C17101724E
:10B6900041727047640F0020054AD279012A06D012
:10B6A0004FF47A7201F5FA71B1FBF2F1401A70476A
:10B6B000640F002070B5134C03460D4694F821200A
:10B6C00000205AB1214691F8201063B1012B11D10D
:10B6D000012A284612D004F0ADFA09E040F2667162
:10B6E0003E20F8F77FFB012A284604D004F0B0FA88
:10B6F000E169084470BD04F0C5FAF9E704F0B3FA53
:10B70000F6E70000640F002010B50022012908D0E0
:10B71000022904D040F269213E20F8F763FB4FF084
:10B72000807205490A4305490A60054908430349EF
:10B73000091D086010BD000008011000141500402C
:10B74000000003020149C0B2086070470C150040B8
:10B7500010B50749012805D0022805D08B213F20CC
:10B76000F8F740FB032000E00420086010BD000053
:10B770001015004070472DE9F0410D0004464FF0D0
:10B7800002064FF0010708D02878D0B1012807D071
:10B79000022814D003283BD116E080F820700EE078
:10B7A0006868C82803D30421F5F754FE08B10026C1
:10B7B00007E02046696800F02AF9012601E0F4F765
:10B7C00061FE3046BDE8F08120780028F7D1686836
:10B7D000F4F72AFEE0B16968087828B1A078052856
:10B7E00007D040F27B1110E0204600F018F9677096
:10B7F000E5E7204600F027F9E07804F10C0100F0BD
:10B800000AF80028DBD140F27D116A20F8F742F8EF
:10B8100084F82070D3E7F6F769B82DE9F0410D46BA
:10B8200004000BD0267900270220092D7BD2DFE807
:10B8300005F008102E2E5B647C97860040F295116F
:10B84000E2E0A07804286FD00328FCD04FF4D07138
:10B85000DAE0A078042804D0032802D04FF4D27193
:10B86000D2E00520A07084F82070207880BB0021F1
:10B87000204600F0CCF8207B012804D0A069E061CC
:10B880000021A26841E0E078F5F70CFFF7E7A17826
:10B89000042904D0032902D04FF4E171B4E02278E6
:10B8A00022B12146304600F0E6F8A4E0042900D099
:10B8B0000120A070A268022D0BD0062130469047CF
:10B8C00000286BD00078002868D04FF4EE719BE020
:10B8D00031E0052130469047002871D000780028DB
:10B8E0006ED040F2D7118FE0A078052802D040F248
:10B8F000E31189E00221A26807E0A078052802D0C0
:10B9000040F2E91180E0A2680121304690470146EB
:10B910002046FFF730FF02286DD0F0B3012864D035
:10B9200040F2292170E05DE067E0A078052802D0B0
:10B9300040F2EF1168E0BDE8F041F4F7A3BDA07854
:10B94000052802D04FF4FA715EE0A2680A21304661
:10B95000904701462046FFF70EFF40F2F71153E0F3
:10B96000A178052906D062780AB1032902D040F2F5
:10B97000FB1149E0217829B121463046BDE8F0416C
:10B9800000F079B894F8201089B184F82070A07084
:10B99000A26808213046904701E029E02BE000280A
:10B9A0000ED0007800280BD040F207212CE06178FF
:10B9B00059B1E07804F10C01FFF72DFF10B1677069
:10B9C000BDE8F08140F20B211EE0A070A2680721C3
:10B9D000304690470028F3D000780028F0D040F29D
:10B9E000132111E04FF406710EE00421A2688CE7E8
:10B9F0000321A26889E7002DE2D100F0EAF800688F
:10BA00000028DDD040F233216A20F7F743FF0246D9
:10BA1000037B0069084410615938F6F7FBBD012229
:10BA200002730022C2752B2282824A794AB1042213
:10BA300082758A686A320261C968816103218170F6
:10BA400070470322F4E710B5044600202073E07528
:10BA50002B20A082487960B10420A075C8686A30A4
:10BA600020618968E069F5F7C7FDA0610420A07036
:10BA700010BD0320F1E770B505460C46C878F6F70F
:10BA800091FB78B1204600F010F8A2680921284601
:10BA90009047002808D00078002805D0DB216A20D4
:10BAA000F7F7F8FED721FAE770BD00218170017029
:10BAB0004170704770B5F4F73FFD0546002406E07D
:10BAC0002046F4F73FFDFFF7F0FF641CE4B2AC4200
:10BAD000F6D370BD2DE9F0410D46F4F733FD0400B7
:10BAE00007D0A0786FF02206012806D0022810D1D6
:10BAF00003E06FF00100BDE8F0816FF0150755B16C
:10BB00002846F4F791FC30B1287830B1A0780228AB
:10BB100008D03046EFE73846EDE729462046FFF7E4
:10BB20007EFF03E029462046FFF78DFFE07804F111
:10BB30000C01FFF770FE08B10020DCE740F2AE21F7
:10BB40006A20F7F7A7FE10B50446F4F7FBFC0100E6
:10BB500004D008786FF0220268B902E06FF00100AB
:10BB600010BD887838B1022807D0012805D00120FF
:10BB70000870002010BD104610BD2046FFF77BFF67
:10BB8000F7E72DE9F0410E460746F4F7D5FC0546E8
:10BB900000240AE02046F4F7D5FC807818B14FF075
:10BBA000FF30BDE8F081641CE4B2AC42F2D3082E51
:10BBB00002D96FF01500F4E717B13146384601E0BD
:10BBC00000210846BDE8F041F4F7A2BC0020F7F7D9
:10BBD0009FBA0020F7F782BA10B5F6F76BFFBDE801
:10BBE000104000F000B8410A43F609525143C0F337
:10BBF000080010FB02F000F5807001EB5020704748
:10BC0000F5F764BD002809DB00F01F020121914017
:10BC10004009800000F1E020C0F880127047002841
:10BC20000DDB00F01F02012191404009800000F16E
:10BC3000E020C0F88011BFF34F8FBFF36F8F7047C4
:10BC400070B50246002000291DD0A2FB0101400A68
:10BC500040EAC150490A401C41F1000140F2A17282
:10BC6000831841F100015B1C41F100040021D3F174
:10BC7000FF33A14103D271216D20F7F70BFE00F5D0
:10BC8000F460B0FBF2F070BD4058002800D00120F5
:10BC90007047D0F80C24D0F80C0402F00102C00365
:10BCA00003D58A4201D1012070470020704710B5AA
:10BCB00001218807F7F7ACFD002800D0012010BD56
:10BCC0004FF080400121016070474FF08041D1F872
:10BCD0001824D1F8181402F00302C90303D58242D4
:10BCE00001D1012070470020704710B500214FF0AE
:10BCF0008040F7F78DFD002800D0012010BD0028FE
:10BD000009DB00F01F02012191404009800000F191
:10BD1000E020C0F88012704700280DDB00F01F0201
:10BD2000012191404009800000F1E020C0F880111D
:10BD3000BFF34F8FBFF36F8F704700100200FA0000
:10BD40000000FE53A0711BEB951033CF46C96395DD
:10BD5000BE5E29386E73002809DB00F01F02012146
:10BD600091404009800000F1E020C0F88012704747
:10BD7000EFF3108172B60278012A01D0012200E0AF
:10BD800000220123037001B962B60AB10020704796
:10BD90006FF0220070470021017008467047EFF3F2
:10BDA000108172B60022027001B962B6002070479D
:10BDB000F7F75CBE4FF08050D0F830010F2801D06B
:10BDC00000207047012070474FF08050D0F83001BC
:10BDD0000A2801D0002070470120704700B5FFF706
:10BDE000F3FF20B14FF08050D0F8340108B10020AB
:10BDF00000BD012000BD4FF08050D0F830010E286A
:10BE000001D000207047012070474FF08050D0F8DB
:10BE10003001102801D000207047012070474FF0FA
:10BE20008050D0F83001062803D0401C01D00020FB
:10BE300070470120704700B5FFF7F1FF48B14FF0A0
:10BE40008050D0F83401062803D3401C01D00120D3
:10BE500000BD002000BD00B5FFF7E1FF38B14FF095
:10BE60008050D0F83401062803D3401C01D00020B4
:10BE700000BD012000BD4FF08050D0F830010D28EA
:10BE800001D000207047012070474FF08050D0F85B
:10BE90003001082801D00020704701207047002A97
:10BEA00004BF00207047521E07D0037891F800C0ED
:10BEB000634504BF401C491CF5D000780978401A3E
:10BEC0007047F0B480EA010C03461CF0030F3CD12C
:10BED00013F0030F0BD0002A04BFF0BC704711F819
:10BEE00001CB03F801CB521E13F0030FF3D1032A49
:10BEF0004FD9B2F1004F4CD2C2F1000C4FEAEC74B2
:10BF00000CEB947C4FEAAC0CCCF1000CBCF1000FB4
:10BF10001BDD0D1F1C1F1CF0010F03D055F8046F13
:10BF200044F8046F5FEA6C0607D06F68676055F8E5
:10BF3000087F44F8087F761EF7D101EB8C0103EBF4
:10BF40008C03CCF1000C02EB8C02002A04BFF0BC85
:10BF50007047B2F1004F26D2002ADCBFF0BC704718
:10BF6000491E5B1E12F0010F03D011F801CF03F838
:10BF700001CF521004BFF0BC704791F801C083F8A4
:10BF800001C011F802CF03F802CF521EF5D1F0BC68
:10BF90007047042AD9D351F804CB121F43F804CBBD
:10BFA000042AF8D2D1E711F801CB03F801CB521ED5
:10BFB000F9D1F0BC704770B4034601F0FF0C10F0EB
:10BFC000030F09D0002A04BF70BC704703F801CBEF
:10BFD000521E13F0030FF5D1C9B241EA012141EA23
:10BFE0000145032A39D9B2F1004F36D25142CC175C
:10BFF00001EB947189104E42002E11DD191F16F0CD
:10C00000010F18BF41F8045F741004D04D6041F86F
:10C01000085F641EFAD1714203EB860302EB8102D2
:10C02000002A04BF70BC7047B2F1004F1DD2002A35
:10C03000DCBF70BC7047591E12F0010F18BF01F829
:10C0400001CF521004BF70BC704781F801C001F8E5
:10C0500002CF521EF9D170BC7047042AE0D3121FE0
:10C0600043F8045B042AFAD2DAE703F801CB521E44
:10C07000FBD170BC70474FF0FF3070470020704715
:10C08000002070474FF0FF30704770477047002026
:10C0900070474FF0FF3070474FF0FF30704700217E
:10C0A000017070474FF0FF3070474FF0FF3070471E
:10C0B000002070472DE9FC41054600F1030020F007
:10C0C00003000C46009049788DF80410A178160002
:10C0D0008DF8051000D0002001A9F8F789F8009923
:10C0E00008440090A17841B1638AE27806B100204B
:10C0F000F8F70EFB00990844009032462146684646
:10C1000000F008F80098C01D20F007000090401BC8
:10C11000BDE8FC812DE9F04706460C4608784978D1
:10C1200000270844914600F0FF083D460EE0237AC0
:10C13000022B00D20223E279032A00D20322A17942
:10C14000607900F0F8FE6D1C0744EDB24545EED372
:10C150003068C01C20F003003060B9F1000F00D03F
:10C1600000203A464146F8F71DFA3168084430602D
:10C17000BDE8F08730B50D468DB01446014610225B
:10C180006846FFF79EFE1022294604A8FFF799FE95
:10C190006846F8F7D3FB18B16FF015000DB030BD4D
:10C1A0001022204608A9FFF78CFE0020F6E70020A9
:10C1B00070473EB50446011D6846F9F7EBFF0028BD
:10C1C00004D06946204600F048F801203EBD0EB577
:10C1D0000146684600F027F86846FAF705F80EBDF4
:10C1E00010B504462046F7F7F1FE002806D0A178E6
:10C1F000207800F004F80028F4D0012010BD70B5BC
:10C200000C460546F7F754FF002802D03E2D01D01A
:10C21000012070BD122C04D02046BDE87040F7F715
:10C2200063BF002070BD0A88C2F30B0202804A88F7
:10C2300042804A789309002242714B78C3F301137C
:10C240001BB1012B05D0022B05D00271091D8160A5
:10C2500070470122F9E70222F7E710B50C4609788A
:10C260000170417821F00F0141702288C2F303224E
:10C2700011434170A2788270628821F03001120A65
:10C28000C2704170227902F0030241EA021121F0EA
:10C29000C0014170627941EA82114170A168021DBA
:10C2A000914206D06288FB2A00D3FB22001DFFF7D3
:10C2B00008FEA078001DC0B210BD2DE9F041044673
:10C2C0000F7800200C2505263E22FF231B2F7DD250
:10C2D000DFE807F0EA0E25272D636D819BAFB1BC27
:10C2E000C7E2F4EAEA31D2D5FDF1F0EFEEEDEC0071
:10C2F00025700879A0704879E070B1F80500000A4F
:10C300002071C8796071087AA0710889000AE0710B
:10C31000887A20724889000A60720820C2E01020E2
:10C3200000E01A2020700879A0700120BAE02046B1
:10C3300000F046F9B4E022700A20A07011F8040F52
:10C34000E070887820714888000A60710879A071CF
:10C350004879E071D1F80600A0604889A081C868DA
:10C36000C4F80E00088A6082D1F812006061C88AA1
:10C370002083087EA076088B000AE076887E2077EE
:10C38000488B000A6077087FA077888B000AE077E7
:10C39000887F84F820001F2084E022701420A07081
:10C3A0000879E0708888000A20718879A7E02270F7
:10C3B0000420A0700879E07088792071C888000A8C
:10C3C00060718868C4F80600C86800E06CE0C4F8D2
:10C3D0000A000C2066E022700320A0700879E0704B
:10C3E00088792071C888000A6071087AA07108896C
:10C3F000000AE071887A20724889000A6072087B1E
:10C40000A0728889000AE072D8E02270A6700879CC
:10C41000E0708888000A2071D1F80600C4F8050091
:10C42000D1F80A00C4F80900C889A4F80D000D204D
:10C4300038E0112043E026700879A0704879E07058
:10C44000B1F80500000A2071C87958E00820207072
:10C450000879A0708879E070C888000A2071087A8D
:10C460004DE0302020700879A0708879E070C8888D
:10C47000000A2071032015E02270072044E022709A
:10C48000A5700879E07088792071C888000A607109
:10C49000087AA071487A27E02046091DF7F7DAFDEF
:10C4A000002801D06070801CBDE8F08173E047E097
:10C4B00028E053E061E01AE009E0FFE75720207030
:10C4C0000879A0708888000AE0700220EAE72270EC
:10C4D0001220A0700879E070487920718879607125
:10C4E000C888000AA071087AE0710620DAE7237094
:10C4F000A120A0700879E070487920710020607157
:10C500000420CFE72370A220A0700879E07088880B
:10C51000000A207188796071C888000AA071087AC1
:10C52000E0710889000A2072887A60724889000ADE
:10C53000A072087BE0728889000A20730B20B1E7A3
:10C540002370A320A0700879E0708888000A207109
:10C5500088796071C879A0710520A3E72270132043
:10C56000A0700879E07048792071D1F80600C4F80D
:10C5700005004889A4F8090020E02370A420A070D9
:10C580000879E0708888000A207188796071C8791C
:10C59000A071072086E723708020A0708A88A4F805
:10C5A0000320CA88A4F805200A7AE2714A7A228117
:10C5B0008A7AA272C97A01F00101E1720A2071E758
:10C5C0003E220270012282700A79C2708A79027159
:10C5D000CA88120A42710A7A82714A7AC271D1F803
:10C5E0000A208260CA8982810A7C82730A8A120ABE
:10C5F000C2738A7C02744A8A120A42740A7D827467
:10C600008A8A120AC274897D0175132070473E22FE
:10C6100002700122827011F8042FC2708A780271B0
:10C620004A88120A42710A7982714A79C271D1F834
:10C63000062082604A8982810A7E82730A8B120AEE
:10C64000C2738A7E02744A8B120A42740A7F827411
:10C650008A8B120AC274897F0175132141700846C2
:10C66000704710B520B1FFF7A4FD20B1002010BD28
:10C670006FF0150010BD6FF0220010BD10B56FF007
:10C68000150420B1FFF7A3FD08B1002010BD20461E
:10C6900010BD10B520B1FFF7A3FD20B1002010BDE3
:10C6A0006FF0150010BD6FF0220010BD02F04ABE01
:10C6B00002F08CBE10B5F7F72BFD002010BD10B5B1
:10C6C000F7F734FD002010BD02F09CBE08B50078DD
:10C6D0008DF80000684602F04CFD08BD012070474F
:10C6E000FDF7FABB01207047007800B1012002F08D
:10C6F000C5BC70B5054610220021FFF75CFC102276
:10C70000002105F11000FFF756FC4FF08054D4F8DB
:10C710008000401C0BD1D4F88400401C07D1D4F811
:10C720008800401C03D1D4F88C00401C0BD0D4F8F6
:10C7300080002861D4F884006861D4F88800A8617A
:10C74000D4F88C00E8610020F8F778FA18B9D4F82A
:10C75000A000C00718D1D4F89000401C0BD1D4F829
:10C760009400401C07D1D4F89800401C03D1D4F8A1
:10C770009C00401C08D054F8900F286060686860E6
:10C78000A068A860E068E860002070BD70B54FF058
:10C7900080550446D5F8A400401C05D1D5F8A80062
:10C7A000C0430004000C3AD0D5F8A000C00736D032
:10C7B000D5F8A400C4F80100D5F8A800A4F8050035
:10C7C000A07940F0C000A071D5F89000401C0FD0B7
:10C7D000D5F89400401C0BD0D5F89800401C07D029
:10C7E000D5F89C00401C03D00020F8F727FA40B190
:10C7F00010220021E01DFFF7DEFB01202070002049
:10C8000070BD55F8900FC4F807006868C4F80B00B5
:10C81000A868C4F80F00E868C4F81300EDE700202A
:10C82000ECE702F098BC02F09EBDFDF763BB02F09E
:10C830007CB902F095B902F0AAB902F0B5B902F0DC
:10C84000BDB902880A8002F0C2B902880A8002F0EB
:10C85000D7B902F0FFB902F003BAFDF793BAFDF7BA
:10C860009BBA02F006BA02F014BAFDF7BFBA02F0A2
:10C870003BBAFDF7DBBA02F03BBA02F042BA02F073
:10C8800044BA02F05BBA02F06EBA02F07ABA02F071
:10C890008DBA02F0BEBA02F051BBFDF7D7BA10B59F
:10C8A000F7F730FC002010BD02F06FBB02F08DBB2B
:10C8B00002F0A1BB02F0ADBB02F0B4BB02F0C7BBFB
:10C8C00002F0DFB802F05BBD70B50B88047F00F1A9
:10C8D000240523F4004602883544A41D2D882244F3
:10C8E00092B22544541E2C4494FBF2F402FB0462E1
:10C8F000408892B2904203D903F40040104302E012
:10C900004FF400409843088070BD20F4004221F4A9
:10C9100000439A4207D100F4004001F400418842EC
:10C9200001D0012070470020704770B5007F1C4681
:10C93000801D084413460988049AC91C89B2151938
:10C94000C01E8D4205D8811822461846FFF7B9FA55
:10C9500000E00024204670BD70B5007F1C46801D9D
:10C96000084413460988049AC91C89B21519C01EC7
:10C970008D4205D8104422461946FFF7A2FA00E07E
:10C980000024204670BD8188C088884201D10120E2
:10C9900070470020704781880089884201D10120BA
:10C9A00070470020704770B5044600F1240180886C
:10C9B00020F400400144208A00281AD0A2890025D2
:10C9C000104480B2A0810A88904205D940F26311D8
:10C9D0004FF01400F7F706FA09D1A06908B1407FBB
:10C9E000887004F104012046FFF76EFFA5812582BF
:10C9F000012070BDF8B5044600F12403C0880E463E
:10CA000020F40047608AD91908B1B04201D2002051
:10CA1000F8BDE089002540B1B1F800C0604508D0FC
:10CA200040F24B211420F7F7DDF9607F88700D800C
:10CA30000EE094F81CC018440CF1060CBC44604491
:10CA4000B4F81EC020F803CC94F820C000F801CC44
:10CA5000E0893044E0810888304408809AB1A11D03
:10CA60002046FFF731FFE581607F401C6077A07DA5
:10CA70008DF80000009800909DF8000078B1E088E3
:10CA8000A082A5750BE0207FE189801D3844194400
:10CA9000084430F8031DE183807884F82000658223
:10CAA0000120F8BD10B50446C088A188814207D096
:10CAB000A08928B9208A18B9A088A18A884201D102
:10CAC000002010BD211D2046FFF7FEFE0020208221
:10CAD000012010BD10B5044600F12402C08820F4E6
:10CAE000004002442088452800D24520884204D2D4
:10CAF00040F219111420F7F775F9E07D002803D0F2
:10CB00001088884201D2002010BD1180A11D20464E
:10CB1000FFF7DAFE0020E075012010BD2DE9F0419D
:10CB2000418986880446002500F10A0706E0394657
:10CB30002046FFF7C9FE6D1C6189ADB2B142F6D146
:10CB40002846BDE8F08130B5C488818800F1240210
:10CB500021F4004313448288858AAA4212D0A1425C
:10CB600010D0818971B9826972B11046FFF713FF45
:10CB700050B91089243220F400401044997880780C
:10CB8000884201D1002030BD184630BD007F801D95
:10CB90000844C01E1060088870472DE9F0410E4619
:10CBA000C1880289044600F12408008821F4004568
:10CBB00022F40047452800D24520B04203D2DB21B1
:10CBC0001420F7F70FF91046FFF79FFE10B1002071
:10CBD000BDE8F081AF4208D9217F781B401A801F41
:10CBE000864202DD0020E075F1E708EB0500012137
:10CBF0000680E175ECE738B5C488818800F124022D
:10CC000021F400431A44A14210D08389058A128876
:10CC10002B44934208D3ADF800106946FFF754FE49
:10CC2000BDF80000A04201D0012038BD002038BD71
:10CC300070B5C6888588034600F1240425F40040B9
:10CC40002044B54202D10020188270BD04889D891D
:10CC50001E7F641B354428440D88A4B2C01CA54225
:10CC600000D90C809C8924B1002414700988198291
:10CC700070BD0124F9E708B5818AA1F57F42FF3A2A
:10CC800008D0827D8DF80020009A00929DF8002047
:10CC900052B904E04FF462711420F7F7A3F88088CA
:10CCA000814201D1002008BD012008BD4FF6FF716F
:10CCB000818200218175704710B5818AA1F57F427C
:10CCC000FF3A04D04FF459711420F7F78BF8C1885C
:10CCD0008182C18909B1012100E00021817510BD67
:10CCE0002DE9F0411D461646069F0B4604463A467E
:10CCF0002946304600F04FF8834201D2A82118E0BF
:10CD0000E01C20F003012046A14201D0A92110E03F
:10CD100024220021FFF74FF94FF6FF70A082A819D7
:10CD2000801D784380B225776080B0F5004F03D92D
:10CD3000AF211420F7F756F8268000206077BDE871
:10CD4000F0818161886170472DE9F0410B4604460E
:10CD500000F1240105894689808825F4004739447B
:10CD60000F46854202D10020BDE8F0810AB1C81CFF
:10CD7000106023B1227FF91C1846FFF7A2F83F8804
:10CD800004F108012046FFF79FFDB54201D120893B
:10CD900060813846E8E70144891D51438AB2002189
:10CDA000452801D2C0F145012432501880B27047A5
:10CDB0002DE9F0478846C1880446008921F40046E1
:10CDC00004F1240520F4004705EB0609FFF79DFD5B
:10CDD000002298B92088452800D24520B74206D9BC
:10CDE000237FB91BC91A891F814200DA0846E189ED
:10CDF00011B1B9F80030C01A404503DA6282002050
:10CE0000BDE8F087207F2944801D30440844A4F801
:10CE10001280C01EF4E70021C181418281757047F4
:10CE200070B50023082904D240F2CB111520F6F783
:10CE3000D9FF02680AB91EE01046026893888B4247
:10CE400002D01368002BF7D1948813468C4201D18D
:10CE500011680DE001F10805AEB20025B44209D316
:10CE6000641A11440D608C800268126802600A60C6
:10CE7000016000E00023184670BD10B50C0006D01C
:10CE8000082C09D240F295111520F6F7ABFF08B136
:10CE900000210160002010BD18B1A1B2006800F0AF
:10CEA00014F8201D10BD0021026803E09388126869
:10CEB000194489B2002AF9D100F007B800230B60A9
:10CEC0008A8002680A600160704700234360021D87
:10CED000018102607047A0F57F43FF3B01D002292A
:10CEE00001D300207047F7F745BAA0F57F42FF3A1B
:10CEF00001D0022901D300207047F7F775BA70B549
:10CF000005460C46084600F06EF908B1102070BDC9
:10CF1000022D01D3072070BD25700020608070BDF8
:10CF200010B50446F7F7ACFAA04201D9012010BDB4
:10CF3000002010BD704770B50E461D46114600F02A
:10CF400011F804462946304600F003F82044001D3D
:10CF500070BD10B50A460121FFF71DFFC01C20F06F
:10CF6000030010BD10B50A460121FFF714FFC01CD5
:10CF700020F0030010BD09B1002100E00221431898
:10CF80001A7D022A08D05B7D022B09D0032A03D028
:10CF9000032B05D00020704700EB4100008B704749
:10CFA00000EB4100408B704709B1002100E00221F5
:10CFB00000EB4100018B11B9408B002800D001200B
:10CFC000704738B583788DF80030009B00939DF84A
:10CFD000003053B90AB1002300E00223C218147DC7
:10CFE000022C04D0527D022A04D0002038BD1A46FB
:10CFF0005B1C00E05A1C81B1C518002400EB430300
:10D000002C751C8303238418237500EB820300EB2B
:10D0100042005B680B60008B8880012038BD10B532
:10D0200009B1002100E0022143181C7D944203D184
:10D0300000EB4100008B10BD5B7D934203D100EB00
:10D040004100408B10BD002010BDB0F5FF7F01D224
:10D05000410800E0FF21401A40F27261884200DB83
:10D06000084680B270470121FFF785BF2DE9F041E6
:10D07000064642F3800748780C4622F004057F1CE0
:10D0800000B10DB9284304D145B100212046F7F77E
:10D09000FFFA0121A1701FB1002002E00121F5E794
:10D0A00002202218127D032A02D1022D00D0401C3A
:10D0B0002218117504EB4001002204EB80000A8362
:10D0C0004068A270314662F30F01C6E90001BDE875
:10D0D000F0812DE9F0411E461346044609B10020B7
:10D0E00000E002200121A17021180A7D012A03D04D
:10D0F000497D01290CD1401C04EB40050027298BF8
:10D10000B5F820C08A19624505D920442F830775D8
:10D110000020BDE8F08104EB8000324640680844FE
:10D120001946FEF7CEFE288B30442883A7700120D5
:10D13000EFE702220021FFF772BF10B50121FFF7D0
:10D1400033FF002800D0012010BD0122FFF739BFB6
:10D150000022FFF736BF70B509B1002300E00223BB
:10D1600001218170C11802240D7D012D07D04D7D54
:10D17000012D09D04FF48B710920F6F733FE00EB37
:10D1800043031A830C7503E000EB43035A834C7589
:10D190000021817070BD012101707047012211468C
:10D1A000FFF73DBF01220021FFF739BF0021FFF744
:10D1B000E2BE002809DB00F01F0201219140400976
:10D1C000800000F1E020C0F880127047F7F7B6BB8E
:10D1D0004FF080410020C1F808014FF0E02101200C
:10D1E000C1F80001704708B1002070470120704766
:10D1F000F7F7EABCF7F7D8BC10B5002904464FF0A2
:10D20000060102D0F6F77AFE01E0F6F793FE6079A8
:10D2100020F0C000607110BD704730B50C46054667
:10D220008DB04FF0030104F1030012B1F6F766FE72
:10D2300001E0F6F77FFE60790D2220F0C00040F09B
:10D2400040006071002104A8FEF7B5FEE0788DF87B
:10D250001F0020798DF81E0060798DF81D001022C6
:10D2600029466846FEF72DFE6846FFF7AFFF9DF89A
:10D270002F0020709DF82E0060709DF82D00A0708A
:10D280000DB030BDF8F77EB8C10701D0012070475E
:10D29000800701D5022070470020704710B5012893
:10D2A00008D0022804D040F29A310620F6F79AFD01
:10D2B000012010BD002010BD002904D0012803D09A
:10D2C000012901D00220704701207047FFF7B0BC50
:10D2D0000121F8F7E7BB10B502F0C0FB18B1BDE8BB
:10D2E0001040FDF771B9FF2010BD10B5F8F722FC12
:10D2F000102803D0F8F7EEFB102800D1082010BD4D
:10D3000010B5F8F717FC102807D0F8F7E3FB102842
:10D3100003D0F8F757FC012010BD002010BD10B558
:10D32000F8F708FC102803D0F8F794FC012010BD92
:10D33000002010BD70B50E468CB0144601461D4647
:10D340001022684600F01AF91022314604A800F0B5
:10D3500015F96846FFF73AFF08A94FF01002284672
:10D360001CB100F00BF90CB070BDFEF7AAFDFAE796
:10D3700010B50C460021FFF7B8FD606018B1012020
:10D380002070002010BD022010BD40F2E241484351
:10D39000704740F2E241B0FBF1F080B2704770B5E7
:10D3A000044690420BD2101B642800D2642025183A
:10D3B0008D4203D80421F4F74DF808B1204670BD22
:10D3C000284670BD10B5A2F10F030C2944D2DFE846
:10D3D00001F006080D1215181C2427412A31C2B38A
:10D3E0003AE0072A3AD0082A38D035E00C2A35D05E
:10D3F0000B2A33D030E00D2A30D02DE00C2B2DD964
:10D400002AE0103A0B2A29D926E0032B26D990F8D6
:10D41000440008B31B2A21D91EE0042A1ED01BE0B9
:10D42000062A1BD018E01C2A18D01D2A16D01E2A46
:10D4300014D011E01F2A11D0202A0FD0212A0DD09C
:10D44000222A0BD0232A09D0242A07D0262A05D045
:10D4500002E003E00E2A01D0002010BD012010BD23
:10D460000C2813D00B2811D00D280FD01F280DD059
:10D4700020280BD0212809D0222807D0232805D026
:10D48000242803D0262801D00020704701207047AF
:10D4900011F00C0F16D04A074FF41671002A02DA69
:10D4A0004FF0100201E04FF0400201DA4FF0960118
:10D4B00001F5BC71A0EB0103884210D993FBF2F097
:10D4C00080B27047022902D070280AD807E03C28B1
:10D4D00005D93C38C11700EB91708010F0E70020AF
:10D4E000EEE77038C11700EB5170C010E8E709682B
:10D4F000C0F866107047C10701D00120704781074E
:10D5000001D502207047400701D508207047002050
:10D51000704710B540F6C412012906D0022905D083
:10D5200040F2C6312920F6F75DFC08B1104610BD67
:10D5300040F2E24010BD2DE9F0410C460546C668B8
:10D54000F4F7A2FB98B1BCB13046E968F4F786F86D
:10D55000002811DD2044401EB0FBF4F707FB04F166
:10D560003046F4F749F8E8603846BDE8F08140F20B
:10D570004B212920F6F736FC0020F6E730B513469C
:10D5800006E0CC18D51A14F8014C5B1E4455DBB2EA
:10D59000002BF6D130BD38B505460C466846FDF780
:10D5A0005FFD10B39DF90000607294F82310A17222
:10D5B00094F90B100022411A00D5494295F8273002
:10D5C0008B4210DCFF2B0ED0217B491CC9B221738A
:10D5D00095F82830994202D8E17A7F2903D1E07288
:10D5E000002020730122104638BD7F206072002089
:10D5F00038BD00238362028640F271235A4301EB57
:10D600000212521EB2FBF1F1C16270472DE9F05FC8
:10D61000074690468B460126084600F041F98246AF
:10D62000584600F049F98146FFF765FF0446504629
:10D63000FFF761FF054654EA050000D10026FCF71C
:10D640004BFF10EA090F00D10024FCF745FF10EA58
:10D650000A0F00D1002597F86A00A04200D10024EB
:10D6600088F8004097F86B00A84200D1002588F8A0
:10D67000015074B96DB9584600F01CF9B7F8741030
:10D68000401A00B247F6FE71884201DC002800DC37
:10D6900000263046BDE8F09F40F2E2414843704723
:10D6A00040F2E24110FB01F0704710B500231A462A
:10D6B00003E0845C2343521CD2B28A42F9D30BB1FB
:10D6C000002010BD012010BD10B5044690F82000C8
:10D6D00008B1252801D9122010BD2AB1607D28B1DA
:10D6E000012809D01F2010BD002010BD2046BDE834
:10D6F00010401146F8F7A2BBA288096904F1150091
:10D70000F8F748FB84F82300EEE730B5421C8A4264
:10D7100004D00A68C0F8012009794171417901F00B
:10D720001F0141710021C1724318491C5C78C9B2C4
:10D7300004F00102640804F001051544620802F0D7
:10D7400001042C44520802F001052C44520802F056
:10D7500001052C44520802F001052C44520802F045
:10D7600001052C4404EB52029A71C37A05291A442C
:10D77000C272D9D330BD70B5D0F81F2090F82330D5
:10D7800012F0FF0F23F01F0308D1C2F307242CB9B6
:10D79000C2F3074414B9120E00D15BB3B0F81920DC
:10D7A000B0F81B50B0F81740837D41B1B2F5506F0F
:10D7B00005D940F607518A4201D8012100E0002135
:10D7C0004678222E16D159B9911F40F67A46B142B9
:10D7D00010D87BB1082B0DD893420BD2944209D8B4
:10D7E000B5F5FA7F06D2B0F81D00B0F5486F01D844
:10D7F000012070BD002070BD70B5B0F80720B0F8F2
:10D80000095030F8054F10F8013CC08831B1B2F52D
:10D81000506F03D940F607518A420BD9911F40F649
:10D820007A46B1420ED86BB1082B0BD8934209D27D
:10D83000944207D8B5F5FA7F04D2B0F5486F01D805
:10D84000012070BD002070BD42680A60007A087136
:10D850007047B0F809007047B0F807007047B0F89B
:10D8600009007047B0F80B00704780890880704746
:10D87000D0F816000860704742680A608068486007
:10D88000704750F80E2F0A60406848607047426841
:10D890000A60806848607047007800F003007047B5
:10D8A0000079704780887047C0887047008970474A
:10D8B00040897047C0887047407970470079704749
:10D8C0000079704701891B290CD341894FF4A47258
:10D8D000914207D381881B2904D3C088904201D389
:10D8E000012070470020704710B5FB2904D94FF480
:10D8F000AF612A20F6F776FA417010BD0179490729
:10D9000004D04079400701D00120704700207047C3
:10D9100000797047407970470171704741717047D5
:10D9200010B51B2A04D940F2DF312A20F6F75AFA43
:10D930004270BDE81040C01CFEF7C3BA0968C16060
:10D9400070470A6842604968816070470A684260AF
:10D950004968816070470A68426049688160704721
:10D96000027801F0030122F003020A4302707047BB
:10D970000171090A417170478171090AC1717047CB
:10D980000172090A417270478172090AC1727047B7
:10D99000027802F00F02032A03D0052A04D1FFF710
:10D9A000EABE40780C2801D0002070470120704763
:10D9B00070B5144605461F2A03D9B2212A20F6F76E
:10D9C00011FA05F10900FEF77CFAA41D6C7070BD18
:10D9D00010B5027801F00F0322F00F021A43027013
:10D9E00007290CD2DFE801F004060406040804004D
:10D9F000062102E00C2100E02221417010BD6E21C1
:10DA00002A20F6F7EFF90A6840F8092F8988818003
:10DA10007047027822F0800242EAC1120270704719
:10DA20000A6840F8032F8988818070470278402374
:10DA300022F0400203EA81110A430270704770B578
:10DA4000144605461F2A03D9D4212A20F6F7CAF91D
:10DA500005F10900FEF735FAA41D6C7070BD0121B7
:10DA600000F053B84168002291F80231002B04D035
:10DA700081F80221406800F040BC70472DE9FC416C
:10DA80000E46A0F57F411746FF3914D030800021A3
:10DA90007171F6F7CFFD0446FFF755F805000AD07F
:10DAA0002046294601AAFFF771F8708030B1FB28A3
:10DAB00006D9C92126E00020BDE8FC81C82121E06B
:10DAC0000198FFF7E9FE012803D0022801D0D821F0
:10DAD00018E0307129467388032520463A460095A0
:10DAE000FEF723FF2046B760FEF7DCFF38B10021C8
:10DAF00020460A46FFF728F918B10120DCE7E821A3
:10DB000000E0ED212B20F6F76DF92DE9FC410446EC
:10DB10000E460020F6F75EFB0546002016B90120F0
:10DB2000F6F758FB0026B0462F1817E02088401C57
:10DB300080B22080B84202D34046A4F8008080B270
:10DB4000A84204D3B84202D20020BDE8FC81694655
:10DB5000FFF70EFC0028F8D0761CF6B2B742E5D8E5
:10DB60004FF6FF7020801220EFE770B550800C89CF
:10DB700094808B89D38048891081CD895581CE8D41
:10DB8000AE4208D14D8D854205D10D8E9D4202D108
:10DB90008B8DA34201D0012300E00023137348853D
:10DBA0005089C88590888885D088088601201070A3
:10DBB00070BD10B58C880A894B88C988A0F8483098
:10DBC000A0F84C10A0F84A40A0F84E2010BD70B547
:10DBD00015460C4600F0C7F896302844A04201D8FC
:10DBE000201A70BD002070BD2DE9F0470446C78E95
:10DBF000468FB0F84C50B0F84000854200D305463F
:10DC0000204694F86B1000F09EF80146E586618787
:10DC1000A28F04F12C00E38F8046AA4200D22A464C
:10DC20008B4200D20B460282A8F81230BD4201D1CD
:10DC3000B14201D0012000E000208146B4F84850F4
:10DC4000B4F84200A78E268F854200D3054694F88B
:10DC50006A10204600F07FF894F86010022908D17D
:10DC6000AF4200D23D46864200D23046002184F8C1
:10DC70006010A8F80850A8F80C00BD4201D1B042CD
:10DC800001D0012000E0002040EA0900BDE8F08753
:10DC9000406870472DE9F04116460F46044600F0F3
:10DCA00062F805463A46E168E06A00F047F8A919CB
:10DCB000814200D308462063BDE8F0811B22028424
:10DCC0008283C2828282428102820281428582856F
:10DCD000828400290AD14FF4A4714184C183418315
:10DCE0000183C18141828181C185018670470068BD
:10DCF00001F19C02904203D9401A9C3840087047B9
:10DD00000020704710B5029C8182C2820383448345
:10DD100010BD5080888A9080C88AD080088B10817E
:10DD2000488B5081012010707047022903D0C00039
:10DD3000703080B2704780003C30FAE7884200D3F0
:10DD40000846801A7047B0F84E10B0F8440081427F
:10DD500000D208467047B0F84A10B0F84600814239
:10DD600000D208467047962190F86B3090F86A20F0
:10DD700000F000B82DE9F0410D46064698461746DA
:10DD8000808E1146FFF7D1FF044639463046FFF733
:10DD9000E2FFA04200D20446B08F4146FFF7C5FF24
:10DDA000074641463046FFF7CEFFB84200D338461B
:10DDB00020442844801DBDE8F081012802D1487923
:10DDC000800901D00020704701207047012806D14A
:10DDD00048790121B1EB901F01D10120704700204B
:10DDE0007047022803D0032801D00020704701208B
:10DDF000704710B50446007CFFF7F3FF48B194F874
:10DE00004F0004F15001FFF770FA082801D00120FB
:10DE100010BD207C18B1022801D0E07D10BDBDE806
:10DE200010400020F6F70ABF08B590F864108DF88E
:10DE30000010009900919DF8001009B1012008BD63
:10DE400090F886008DF80000009800909DF8000082
:10DE5000002008BDFF200870C86AFFF79CB91CB5F8
:10DE60000446D4220021FEF7A6F8FF2020707F2070
:10DE700084F8260013206080F6F79CFC0146E062DF
:10DE800000226846FFF7F2F800220121E06AFFF75E
:10DE900062F904226846E16AFFF7E8F800221146B9
:10DEA000E06AFFF758F90020A07304F12000BDE8F4
:10DEB0001C4000F062B98078C0F3800008B10020F7
:10DEC00070471F207047F8F7B7BF80687047012080
:10DED000704710B50446203000F00FF96188BDE8A6
:10DEE00010402822F9F786B90022826243881D2B50
:10DEF00001D0417370474273704710B50024C06A67
:10DF0000FFF717F900B10120844384F0010010BD30
:10DF100000207047807800F0010070478078C0F3DF
:10DF2000C0007047012070478078C0F34000704700
:10DF300090F90E0070470078FF2801D0012070474B
:10DF4000002070470A6840F8112F898881800121DC
:10DF500081717047007B704701207047C161704735
:10DF600080F86010704770B5044680780125C0F3D2
:10DF7000C00038B13C23FF222046E169F8F788FF52
:10DF800084F86450A078C007FBF7F6FE84F861506F
:10DF900070BDC07B002800D00120704710B5FFF78E
:10DFA000A4F90446F7F7F2FC38B12046F7F726FC4F
:10DFB00018B11021FFF779FB08B1002010BD012036
:10DFC00010BD0121F8F7C2BB0121F8F7BFBB2DE955
:10DFD000F041044600274F7011200D4608702022A2
:10DFE00004F16601281DFDF76CFF01262E7284F8EE
:10DFF00064702879002811D1E888A4F89000E069BD
:10E0000090F8851084F8921084F88E600088F6F7F6
:10E0100011FBFEF74BFEE06980F87060BDE8F0810F
:10E020002DE9F04104460F46407EF7F7A7FB064670
:10E03000207E04F1490520B11EB1607EF7F792FB06
:10E04000A0B194F86200002824D0A07E002821D03E
:10E0500094F848002946FFF7B9FEA8B1F7F77EFB10
:10E060003A462946BDE8F041FFF7D7B8012084F8C9
:10E0700048003A4629463046FFF7CFF8617E2846E9
:10E08000BDE8F041F7F786BB39462846BDE8F041C8
:10E09000FFF7B2B8BDE8F08110B504460846FDF7B9
:10E0A0001FF82179BDE81040252001F069BD10B5A9
:10E0B00004462630FCF7D4FF002802D17F2084F8E4
:10E0C000260010BD0278202322F0200203EA41112D
:10E0D0000A430270704770B50170427014460D46D5
:10E0E000807800F07FF810FB05F06043FF2803D331
:10E0F0005C212E20F5F776FE70BD10B504468078C1
:10E1000000F070F86178227811FB02F14843C0B248
:10E1100010BD10B5044600F04DF86179491CC9B234
:10E120006171627891420BD100226271E178014302
:10E13000E170A378994203D1E2702179491C2171E1
:10E14000BDE8104000F025B88170704770B50446F6
:10E15000807800F047F8617811FB00F5E07800F076
:10E1600041F86178627910FB012021782279891ABF
:10E1700011FB05F1081AC0B270BD00210160818059
:10E1800001214170017070470021C170417101711E
:10E19000704710B5012807D0022807D0042807D0FF
:10E1A00039212E20F5F71EFE252010BD262010BD9A
:10E1B000272010BD014600208A78D30702D0CB78F3
:10E1C000DB0706D0930706D5CB789B0703D4022044
:10E1D0007047012070475207FCD5C9784907F9D428
:10E1E00004207047C0F38001C0F34002114400F0E6
:10E1F00001000844704740F25A314843704740F2EA
:10E20000EF2070470E021C043006600C5A03B4065F
:10E21000C505F50B2512A301B103BF05EF024906A1
:10E22000A30910B590F8D01009B1002010BDD0F8A6
:10E23000CC1049B990F8A81031B1D0E92B128A421C
:10E2400002D9FFF790FEF0E7012010BD10B531B103
:10E25000012908D040F28A713020F5F7C3FDBDE8EE
:10E26000104000F0D4B9002180F8A810BDE810409B
:10E2700000F03BB910B5044690F8B400002819D05E
:10E28000012084F8D00001462046FFF769FE94F88B
:10E29000B40070B114F8A00FF3F758FE2078F3F72C
:10E2A000A3FF14F8A009F3F77DFF20B1002084F844
:10E2B000B400002010BD40F20F213020F5F792FD90
:10E2C000D0F8A400704790F8B40070470EB56946C6
:10E2D0000120FEF714FE38B14FF4A1713020F5F79C
:10E2E00081FD0298FFF7C6FF6846F5F7C1FF0028D9
:10E2F000F7D0F9F7FBF800200EBD7CB5044690F886
:10E300000301002853D194F8340103284FD1FDF7BD
:10E3100063FC0146D4F85C01F3F7A0F9002846DD60
:10E32000E16811B1B0FBF1F000E00020B4F8741026
:10E33000401C0844A4F84401B4F84401B4F8FC10AB
:10E34000081A00B2002832DD94F86801F3F7FEFDE8
:10E3500000282CD0012084F84901B4F8A600B4F8B4
:10E36000A41001AE401AB4F87410401E084485B2DF
:10E3700017E00096B4F84411002301222046F9F773
:10E3800085F9002813D0012804D040F20C61302018
:10E39000F5F728FDB4F84401BDF804100844A4F8CA
:10E3A0004401B4F84401281A00B20028E1DA7CBD27
:10E3B0000020704770B50446012600F00CF9A4F85F
:10E3C000C000002084F8B800012084F8C30094F84D
:10E3D000A80004F1B80560B14FF47A71D4F8C40014
:10E3E000F3F70AF9C4F8C40000212846FFF7A3F8A0
:10E3F0000FE02046FFF769FD06463146D4F8C40019
:10E40000F3F7FAF8C4F8C40031462846FFF793F84A
:10E41000461CB4F8C800411C0A2902D23044A4F8B2
:10E42000C800D4F8A40030B1B4F8C800401C0A28D1
:10E4300001D3022000E0032084F8C200002120461E
:10E4400000F022F820B12046BDE8704000F00DB881
:10E4500094F8A000294600F0BCF8002804D140F24E
:10E46000AD613020F5F7BEFC70BD10B5044614F860
:10E47000A00FF3F797FE0020207510BD10B5FFF731
:10E4800028FD00F5847010BD70B5044690F8D000EA
:10E490000D4608B1012070BDD4F8CC00A8B12046CB
:10E4A000FFF713FD05442046FFF7E8FF4119D4F8B4
:10E4B000CC00884206D20120C4F8CC002046FFF7E9
:10E4C00052FDE7E7401BC4F8CC00002070BD10B53A
:10E4D000044690F86B0000F0A3F902462046BDE820
:10E4E000104040F21711FFF7D5BB10B5FCF74EFCFA
:10E4F000BDE81040F3F7ACBF2DE9F047044690F8B3
:10E500004A01002851D094F8340103284DD194F8E1
:10E510006B9001F07EFA054694F87501F8F7D8FF84
:10E52000284486B294F87501F8F7D2FF00F5C86068
:10E530001FFA80F8484601F005FBD4F870110D1A57
:10E54000484601F00DFB4FF47A7A00F2E730B0FB59
:10E55000FAF02D1A484601F0F5FAD4F808110F1A0E
:10E56000484601F0FDFA4AF2A1310144B1FBFAF04C
:10E57000391AA1F160007043B0FBF8F2292000EBDA
:10E5800051006032A0EB520100EB5200A94201D8C9
:10E59000854201D9F5F7A0F83146E068FDF750FB58
:10E5A0000021C4F83C0184F84A11BDE8F08770B539
:10E5B0000C46054601F0D4FA4AF2A13108444FF462
:10E5C0007A71B0FBF1F6284601F0BCFA30442044E1
:10E5D00070BDF3F78BB910B50446FFF7A3FCA0B1EB
:10E5E0002046FFF797FC18B92046FFF79DFC20B1A5
:10E5F000492401F073FA28B901E04224F9E701F057
:10E6000063FA00B1E41D204610BD6B2010BD70B54B
:10E61000044690F8A100002518B1012000F087F809
:10E6200005462046FFF751FC4119D4F8C400B83420
:10E63000F2F7E2FF0026E06004F80B6B012004F81B
:10E640000109032004F8C2092046FFF7C4FFA4F81B
:10E65000C00029462046FFF717FF30B994F8A00004
:10E6600004F1B801FFF7B5FF28B1A4F8C860BDE810
:10E670007040FFF73ABF40F2F6613020F5F7B2FB89
:10E6800010B50446002084F8340194F86801F3F7CB
:10E6900089FD202084F8680110BD2DE9F84300258C
:10E6A00080F8A850D0F8C4608846044680F8B4507A
:10E6B000012780F8B570D0F8A4003946A034F7F7E8
:10E6C000D7FA6068C0F85C616168207881F86801F9
:10E6D0006168C1F86C816068C0F86061646884F842
:10E6E00034510023A4F864511A4619462046009577
:10E6F000F8F7CCFF20B140F223213020F5F772FB70
:10E70000C4F83051C4F8285184F83471A4F8465143
:10E71000A4F8445104F59874657634F8BC0C401E96
:10E7200024F8BC0CE586BDE8F843FFF7DEBE08B56B
:10E7300000284FF00101684602D0F5F7DFFB01E049
:10E74000F5F7EAFB9DF8000042F210710002B0FB01
:10E75000F1F201FB120008BD10B5040008D0092930
:10E760005CD2DFE801F007363E3E3A5B434A570091
:10E770009C2150E00021C4F8701194F84811204603
:10E7800089B1B0F84621B0F874108A4206D1B0F8C9
:10E79000FC20511AA0F8FE1011460DE0511AA0F805
:10E7A000FE1091B208E0B0F84411B0F87420891A54
:10E7B000A0F8FE10B0F84411A0F87410D0F8581169
:10E7C000C0F85C11F9F7D8FB2046BDE81040F9F716
:10E7D000C1B9BDE8104000F005B9BDE81040FCF734
:10E7E00085BC2046BDE8104000F027B80120F2F7B4
:10E7F00021FEBDE81040FEF745BD94F83401042821
:10E8000001D0BE2107E02046FFF73AFFBDE81040E7
:10E81000FBF7B2BAC7213020F5F7E4FACB21FAE7CB
:10E8200010B501F09DF94DF6417108444FF47A712D
:10E83000B0FBF1F000F2751010BD7CB50446FDF799
:10E84000CBF90146D4F85C01F2F708FFE16811B199
:10E85000B0FBF1F000E0002094F87E100D290CD000
:10E86000B4F87420B4F846111318CB1A1BB2002B5D
:10E8700006DB491CA4F8461106E0B4F8460112E094
:10E88000401C1044A4F8460194F849018DF800009A
:10E89000009800909DF8000040B9B4F84601B4F823
:10E8A000FC10884202D1401CA4F84601B4F866016D
:10E8B000401CA4F86601B4F8A600B4F8A410401AED
:10E8C000B4F87410401E084485B226E001A8002365
:10E8D00000901A462046F8F7D9FE002838D00128C3
:10E8E00004D040F259613020F5F77CFAB4F84601C3
:10E8F000B4F8F810421A12B2002A09DABDF804205E
:10E900000244AA1A12B2002A02DAA4F8461104E05C
:10E91000BDF804100844A4F84601B4F84611681A7A
:10E9200000B20028D2DA94F8810078B1082084F887
:10E930009500012084F89400204600F055F8204608
:10E94000FFF79EFEBDE87C40FBF716BA3E20EEE7DF
:10E950007CBDF401FA00960064004B0032001E00FA
:10E9600014000A0005000200010000EBD10001F0D4
:10E9700007030278012199408A430270704710B55D
:10E980000446D0F89C01E168884209D1B4F8A0118E
:10E99000A28A914204D1B4F8A211E28A914213D022
:10E9A0002188A4F8BC11FEF7F4FCA4F8BE01B4F869
:10E9B000A001A4F8C001B4F8A201A4F8C20101208A
:10E9C00084F8B801FBF7D8F902212046F7F750F98F
:10E9D000002004F87E0F0320E07010BDF5F7B6BDEF
:10E9E00000207047F6F7E4BA002180F87D1080F827
:10E9F0007E1080F8811090F8031109B1022100E027
:10EA00000321F8F71BBD90F87C00FE2801D00120FF
:10EA100070470020704710B5012806D0022804D0A6
:10EA200040F263210620F5F7DDF910BD012802D080
:10EA3000022805D102E0012904D001E0022901D019
:10EA40000020704701207047401A00B247F6FE715F
:10EA5000884201DC002801DC01207047002070475B
:10EA600000EBD10001F00701007801228A4010403C
:10EA7000C840704718B1022801D00120704700201B
:10EA80007047FEB5817804461A2925D00EDC162978
:10EA90002DD2DFE801F02C2C2C2C2C212C2C2C2C12
:10EAA0002C2C2C2C2C2C2C2C2C2121212A291ED036
:10EAB0000BDCA1F11E010C2919D2DFE801F01818B6
:10EAC0001818181818181818180D3A3904290ED2E1
:10EAD000DFE801F00D020D022088B0F5706F06D25C
:10EAE00001276946FEF744FC18B10220FEBD122042
:10EAF000FEBD019D68462E4605F5BC7506F27916E9
:10EB000000F094FE38B128788DF808000298029041
:10EB10009DF8080008B10C20FEBD2F70A078307061
:10EB20006846FEF79FFF0020FEBD10B50446007842
:10EB300018B1012801D0122010BD00F02BFE20B129
:10EB4000F6F788FE08B10C2010BD2078FFF792FF81
:10EB5000E21D04F11703611CBDE81040F6F7ACBEDE
:10EB600010B5044600F0F2FE08B10C2010BD20786C
:10EB700018B1012801D0122010BDFFF77BFF611CE6
:10EB8000F6F712FF08B1002010BD072010BD10B528
:10EB900000F000FE20B1F6F75DFE08B10C2010BDBC
:10EBA000F6F7D0FE002010BD10B500F0CFFE08B182
:10EBB0000C2010BDF6F720FF002010BD10B50B464D
:10EBC000012200F11001FEF7B5FB002010BD10B5C9
:10EBD00000880021FEF789F918B190F87B1111B176
:10EBE00007E0022010BD90F87E10142903D01529EB
:10EBF00001D00C2010BD022180F87B11002010BD37
:10EC000038B5054600880021FEF76FF9040003D0EF
:10EC100094F87B0110B110E0022038BD94F87E001A
:10EC2000142801D0152808D194F8CC018DF80000E3
:10EC3000009800909DF8000008B10C2038BD10220B
:10EC4000A91C04F5BE70FDF73CF9012084F87B0196
:10EC5000002038BD10B50821F5F76CF9002010BD73
:10EC600010B5044600F0F9FDFFF762F920700020AE
:10EC700010BD10B5044600F0D3FD40B1FB2020804C
:10EC800040F648016180A080E180002010BD012095
:10EC900010BDFEB50D460646FBF718FCC0F300207C
:10ECA00000B330886946FEF763FB002819D1019C48
:10ECB000002784F86C7014F86A0F00F046FCA87006
:10ECC000607800F042FCE870A0788DF808000298A7
:10ECD00002909DF808006A3C0028EAD1308828801C
:10ECE0000020FEBD0120FEBD0821017000207047FC
:10ECF00010B50446D820207000F073FD607000202D
:10ED000010BD082101700020704710B5044600783E
:10ED100008B1012810D100F03DFD20B1F6F79AFDB1
:10ED200008B10C2010BD2078FFF7A4FE611CFEF78F
:10ED3000E7FA08B1002010BD122010BD10B504463E
:10ED400000F004FE08B10C2010BD207808B10128A5
:10ED500007D1FFF78FFE611CFEF7E1FA08B1002032
:10ED600010BD122010BD10B5044600F013FD08B10F
:10ED70000C2010BD207800F00100F6F765FD0020A2
:10ED800010BD1CB5044600F068FD00208DF802009F
:10ED900003218DF8011014F8011B8DF803108DF874
:10EDA00000006846019400F0F8F91CBD7FB50546E7
:10EDB00000F053FD06462878002460B18DF800402D
:10EDC00001200DF10101F5F70DFF20B1684600F0BB
:10EDD00097F8002812D18DF80C403046FFF79EF8C6
:10EDE00018B18020ADF80D0001E0ADF80D408DF8B0
:10EDF0000F402878012803D038B1122004B070BD2C
:10EE000003A93046FBF744F9F8E7304600F03CFD33
:10EE1000F4E730B58BB0044600F01FFD02462079C0
:10EE2000042803D86088B0F5804F02D912200BB0B7
:10EE300030BD00258DF80450217900959DF8000023
:10EE4000052940F010008DF8000054D2DFE801F0F1
:10EE5000030805110B0040F0010040F0020006E03D
:10EE600040F0090001E040F0010040F004008DF89E
:10EE70000000BDF800000090BDF80000ADF80500EE
:10EE80002188DDF8060061F31F20CDF806006188B7
:10EE9000DDF8090061F31F20CDF80900607B8DF8D3
:10EEA0000D0060798DF80E00A0798DF80F00D4F870
:10EEB00007000490B4F80B00ADF81400A07B8DF8A7
:10EEC00016007F208DF8170001208DF818008DF8AE
:10EED00019508DF81A008DF81B501046FFF73AF8BC
:10EEE0008DF81C008DF81D508DF81E5009A901A841
:10EEF00000F0DEF89BE741F293013920F4F772FF4E
:10EF000070B5044600780121FDF7EFFF050007D03A
:10EF1000FFF7D9F960B12846FFF706F810B105E010
:10EF2000422070BD2846FEF7F5FF08B10C2070BDE9
:10EF3000611C2846FFF706F8002070BD3EB50D465F
:10EF4000044600F06DFC30B1A28844F29020824269
:10EF500003D912203EBD01203EBD40F6480082424A
:10EF600000D302462088ADF800006088ADF80200AA
:10EF7000ADF804206088ADF80600ADF808202088C0
:10EF800028806846FBF752F93EBD3EB50446FBF7C4
:10EF90009DFAC0F30020B0B10DF107000090227976
:10EFA000E178A0780DF1060300F094FC002809D167
:10EFB0002088ADF80400B4F80500ADF8080001A8F9
:10EFC00000F0A6F93EBD01203EBD10B5044600F09C
:10EFD000E1FB20B1F6F73EFC08B10C2010BD207813
:10EFE000FFF748FDE279611CF6F7E2FB08B100206B
:10EFF00010BD022010BD10B50446012000F0C8FA73
:10F0000028B121460120F5F705FE002010BD0C2097
:10F0100010BD10B50088F6F7ABFC08B1002010BD9C
:10F02000302010BD1CB5044600F017FC00208DF800
:10F0300000008DF8020003208DF8010014F8010B88
:10F040008DF803006846019400F010F91CBD1CB552
:10F05000044600F0E5FB78B12088ADF80000608838
:10F06000ADF802002088ADF804006088ADF8060015
:10F070006846FBF75FF91CBD01201CBD10B5F5F714
:10F08000EDFD002010BD7CB50C46054600F0C8FB28
:10F0900060B169462846FEF76BF9002805D10021CA
:10F0A0002246019800F040FB00207CBD01207CBD81
:10F0B0002DE9FC410F460546067800F0C5FA002808
:10F0C0000AD1284600F09AFA002805D10120F5F768
:10F0D00081F8864202D30720BDE8FC810121304639
:10F0E000FDF703FF040004D0FFF7EDF850B10C204A
:10F0F000F2E7002201213046FDF7EDFE04000FD0BB
:10F10000FEF7ADFE2046FEF713FF3870E87429467F
:10F110002046F7F723FA0646687ED0B12EB118E0F4
:10F120004FF491513920F4F75DFE00226846E16A00
:10F13000FDF79CFF00220121E06AFEF70CF8042293
:10F140006846E16AFDF792FF00221146E06AFEF789
:10F1500002F83046C0E710B50446002000F018FA67
:10F1600028B121460020F5F755FD002010BD0C20E8
:10F1700010BD10B5007800F00100F8F725F9002067
:10F1800010BD10B5044600F04BFB20B12046BDE891
:10F190001040FBF74BB8012010BD2DE9FC4106469D
:10F1A000457800780121FDF7A0FE04001ED0FEF78F
:10F1B00082FEF178814200D808460746042D18D017
:10F1C000E06AFDF7EBFF384481B22046012200F0EF
:10F1D000F1F900280BD1032D00D0DFB12046FEF756
:10F1E000A1FE7178032910D0A0B904E04220BDE847
:10F1F000FC817FB9F2E7042907D12046FFF763F8C5
:10F2000040B1E06AFDF799FF20B1012D04D0032D34
:10F2100002D00EE01220EAE72046FEF783FE08B196
:10F22000002202E0012D13D001226846E16AFDF7B9
:10F230001DFF042D18D072683B460121E06AFDF7DE
:10F2400048FF38B17078022806D0032804D00BE0BC
:10F250000222EAE70720CAE7E06AFDF79FFF0246BD
:10F260000121E06AFDF777FF0020C0E72DE9FC41AE
:10F2700007464578C67800780121FDF736FE040080
:10F2800003D0FEF751FE18B103E04220BDE8FC8137
:10F290000026E06AFDF786FF304481B288462046AA
:10F2A000012200F087F90028F0D1042D08D0032DA9
:10F2B0000AD02EB12046FFF706F818B10C20E5E77A
:10F2C0001220E3E7012D0CD12046FEF72BFE08B1FA
:10F2D000042202E0012D10D005226846E16AFDF704
:10F2E000C5FE7A6833460021E06AFDF7F2FE30B1D0
:10F2F000022D06D0032D04D008E00622EDE70720FA
:10F30000C4E742460021E06AFDF725FF0020BDE783
:10F3100010B50446808828B1012803D0022801D006
:10F32000122010BDE07800F0DCF948B1A07800F0C0
:10F33000D8F928B12046BDE81040012100F084B87A
:10F34000112010BD7CB50C46054600886946FEF7C5
:10F350000FF8002806D1019829882180B0F8A00074
:10F36000608000207CBD10B5044601460020F5F702
:10F3700039FC10B900202060A080002010BD7CB5B1
:10F3800000886946FDF7F4FF58B9684600F04EFA68
:10F3900038B1019C94F8B41104F5DA70703429B9CD
:10F3A00001E002207CBD94F8451009B13A207CBDF3
:10F3B00094F846104FF00105890703D1057068469F
:10F3C000FEF750FB84F8455000207CBD7CB50C4610
:10F3D000054600886946FDF7CBFF08B102207CBDD9
:10F3E000A87830B100F0FDF9A070288820800020B6
:10F3F0007CBD019890F86E00F6E710B5FAF7D4FFDF
:10F40000002010BD2DE9FC41044640880D46B8B1EE
:10F4100020886946FDF7ACFF00280FD1208828809E
:10F42000019E06F10C0570362F6862883946304619
:10F43000FEF7DFF82868B842F6D10020BDE8FC816D
:10F440001220FBE7FAF76EBD2DE9F04786B08A4639
:10F450000646008801A9FDF78BFF002838D10298E5
:10F460004FF000080146894690F8FC118DF8001015
:10F47000009900919DF8005090F87E10703021297D
:10F4800000D13DB100244C3008210746FFF7E8FACF
:10F4900010B107E00124F6E70B213846FFF7E0FA48
:10F4A00000B9A4B104A800909DF8040003AB324653
:10F4B000494600F076F907000AD19DF80400029C45
:10F4C00048B104F5D774012060704DB906E01A20E8
:10F4D00006B0BDE8F08704F59774F4E7207808B12A
:10F4E0003A2712E084F800A09DF80C00A0709DF867
:10F4F0001010E1708DF800008DF80110B088ADF8A3
:10F50000020069464846FDF7F2FF84F8018038465C
:10F51000DEE710B50820FAF7CFFFBDE81040F8F796
:10F5200013BD4FF4A471884203D340F648018842CA
:10F5300000D308467047C10701D0012070478007FB
:10F5400001D5022070470020704710B5012806D071
:10F55000022804D040F263210620F4F743FC10BDDA
:10F560000EB569460120FDF7CAFC50B140F24111C9
:10F570003920F4F737FC0298FEF7A5FE08B1012008
:10F580000EBD6846F4F774FE0028F4D000200EBDCE
:10F5900010B5FFF7E5FF58B100F05FF90446FEF73C
:10F5A000C3FC18B92046FEF7B5FC08B1002010BD19
:10F5B000012010BD70B50C46054612B11F290CD8AC
:10F5C00016E0F5F71BF9A04201D2072070BD2846CE
:10F5D000FEF7A8FC18B11F2C01D9122070BD2846D7
:10F5E000FEF7A9FC30B121462846FEF770FC18B1A1
:10F5F000002070BD422070BD452070BD10B504468E
:10F600004078C1061CD5C0070BD0FAF70BFFB8B184
:10F610006078C10605D4000703D5207D02280FD1EC
:10F6200010E0207D022801D0A07E48B96078000754
:10F6300008D4D4F805004FF48041B1EB102F01D26B
:10F64000112010BD002010BD38B504460078EF2809
:10F6500043D8B4F80100ADF80000009800F051F96B
:10F66000A0B3617808070BD4D4F80200D4F80530B1
:10F67000020AB2EB132F30D82022B2EB102F2CD875
:10F68000607A18B3072828D8A07A28B1012803D0B7
:10F69000022801D0032820D14A0703D4022801D030
:10F6A000032805D1E07A08B1012816D1480707D40C
:10F6B000A07C28B1012803D0022801D003280CD156
:10F6C000C806207D03D5012807D102E005E0022805
:10F6D00003D0207E18B1012801D0122038BD0020AF
:10F6E00038BD10B5040005D0FAF7F6FE844301D00A
:10F6F000002010BD012010BDFB2803D840F64800B3
:10F70000814201D911207047002070471B38E12841
:10F7100006D2B1F5A47F03D344F29020814201D9EF
:10F7200012207047002070472DE9F0410646B0F8DE
:10F730005270B0F8544015462C30F7F74BFE804617
:10F740000221FDF7A5FE874200D238460746022176
:10F750004046FDF79DFE844200D220463188298034
:10F760001B2F13D9FB2F00D3FB276F801B280FD92A
:10F77000FB2800D3FB20E8804046FFF7D2FEA8809C
:10F780004046FFF7CEFE2881BDE8F0811B27ECE75D
:10F790001B20F0E710B5FFF7E3FE002800D00120A2
:10F7A00010BD2DE9F0419078069E1D46144608B91B
:10F7B000FAF792FEE478074614B9FAF78DFE04468C
:10F7C0006FB164B13846FFF7B6FE2046FFF7B3FECF
:10F7D0002FB124B12F7034700020BDE8F0810920D2
:10F7E000FBE710B5FCF711FB28B9FCF744FB10B997
:10F7F000FCF74BFB08B1082010BDFCF7DBFA40B961
:10F80000FCF7E2FA28B9FCF7F6FA10B9FCF707FBA7
:10F8100008B1042010BD4FF4B1613920F4F7E2FAC9
:10F8200010B5FAF753FEC0F3401010BD406800F069
:10F8300000B808B590F8341190F894008DF80000E5
:10F84000009800909DF80000401E084203D0042953
:10F8500001D0012008BD002008BD10B50121002005
:10F86000FDF743FB040008D1002201211046FDF7FB
:10F8700032FB040003D0FEF7F2FA204610BD4FF42D
:10F8800008713920F4F7AEFA70B50546FEF753FB60
:10F8900070B12846FEF717FD002808D02846FEF76D
:10F8A0000FFD04462846FEF7E5FC18B10C2070BD9C
:10F8B000422070BD64B12088FDF79AFC20880021A9
:10F8C000F4F726FD20B141F2B9413920F4F78AFA64
:10F8D000002070BD30B540F3000440F34000401CF0
:10F8E000039D641C00D019B100B10AB11CB901E03C
:10F8F000112030BD0021197000B900222A700020AB
:10F9000030BDC0B2C1060CD481064FEAC07103D528
:10F91000D1B9810718D401E00029FAD1000713D426
:10F9200010E0410610D481060ED4C1074FEA807161
:10F9300004D0002902DB400704D405E0010703D40A
:10F94000400701D401207047002070473EB569464A
:10F950000120FDF7D4FA78B140F25F113920F4F7B5
:10F9600041FA029C2046FEF7AEFC28B12046FEF785
:10F9700010FB08B101203EBD6846F4F779FC002871
:10F98000EFD000203EBD026812B901607047024608
:10F99000506808B18A42FAD18A42F7D05160704764
:10F9A00010B5FEF793FC08B1F32103E0F6F7A6FECD
:10F9B00018B1F8210120F4F715FABDE81040012034
:10F9C000F4F7ECBB10B5044602E020688047646899
:10F9D000002CFAD110BD10B50020F4F7DFFBF4F7CE
:10F9E00015FEF5F7E1F8F5F7D5FA002803D0D02198
:10F9F0000120F4F7F7F910BD10B5FFF7D1FFFEF7BE
:10FA0000EFFF002804D040F211110120F4F7EAF9C9
:10FA100010BDF3F75BBE01000B0002000A000500F9
:10FA200009000A000800140007001E00060032004A
:10FA300005004B0004006400030096000200FA0079
:10FA40000100F401000010B5FBF736F900F050F8A2
:10FA5000FAF7B0FDBDE81040FAF7AEBE10B5C82405
:10FA6000641EE4B2FAF7C4FD022803D0012800D0D6
:10FA7000002010BD002CF3D193213B20F4F7B2F904
:10FA800010B5F4F77DF8002805D0401C03D05021B4
:10FA90004020F4F7A7F910BD10B5F4F77DF8002861
:10FAA00005D0401C03D049214020F4F79BF910BD3C
:10FAB00010B5F4F75FF8002805D0401C03D057219B
:10FAC0004020F4F78FF910BD10B500210846F4F777
:10FAD0005DF808B1002010BD012010BD08B56846D2
:10FAE000F4F766F89DF80000002800D0012008BD5A
:10FAF0004FF0E0214FF40040C1F88001BFF34F8F79
:10FB0000BFF36F8FFAF732BF002809DB00F01F0246
:10FB1000012191404009800000F1E020C0F88012EE
:10FB2000704700280DDB00F01F02012191404009C1
:10FB3000800000F1E020C0F88011BFF34F8FBFF3C9
:10FB40006F8F704710B5012806D0022806D040F606
:10FB500064313E20F4F746F9282010BD182010BD6E
:10FB600010B5012806D0022807D040F678313E2093
:10FB7000F4F738F941F6146010BD41F2301010BDB1
:10FB8000FBF7C2BD10B50A4630B101280BD040F2D8
:10FB900027613E20F4F726F9BDE8104002F1280164
:10FBA0001046FAF779BDBDE8104002F12901104670
:10FBB000FAF75CBD70B5054614460846FFF7D0FF5E
:10FBC00005EB4501C1EBC511C0EBC1052046FFF7B0
:10FBD000C7FF28444FF47A7100F6B730B0FBF1F557
:10FBE0002046FFF7AFFF2844401D70BD2DE9F041CE
:10FBF00007461D460E4614461046FFF7B1FF07EBB9
:10FC00004701C1EBC71100EBC1014FF47A70022E1E
:10FC10000ED040F2DC52114401F6B731B1FBF0F6E0
:10FC20002046FFF78FFF30442844401DBDE8F08197
:10FC30000246F0E710B504460846FFF791FF4FF47F
:10FC40007A7100F2E730B0FBF1F0201A801E10BD8F
:10FC500010B504460846FFF783FF4FF47A71B0FBF6
:10FC6000F1F0201A10BD4FF47A72022908D040F248
:10FC7000DC5101F2E731B1FBF2F10844801E70471C
:10FC80001146F6E74FF47A72022907D040F2DC51B0
:10FC900001F57A71B1FBF2F1084470471146F7E7BC
:10FCA0000C0802170D0101020909010106020918D9
:10FCB000180301010909030305000000000000000A
:10FCC00073B5414DD5F87431996811F0010121D116
:10FCD00001AA40F6034004F0A1FC0446002870D1BC
:10FCE000019B9B681B7893B9BFF35B8F2B4653F83E
:10FCF000CC2FBFF35B8F02F00502BFF35B8F53E89D
:10FD0000001F43E800200028F9D1BFF35B8F019862
:10FD10000AF0BCFF01AA002141F2030004F07EFCBE
:10FD2000044600284DD1019B2848996808220131DA
:10FD300016F018FA01980AF0A9FF214601AA41F22B
:10FD4000010004F06BFC044600283AD10198836856
:10FD50005A7885F86820D9789A7842EA0122A5F87D
:10FD60006A201A7985F86920197ADA7942EA01223B
:10FD7000A5F86C205A799B7942EA0323A5F86E30E6
:10FD80000AF084FF214601AA41F2020004F046FC79
:10FD90000446B0B9019B0E4899684022013116F023
:10FDA000E1F90B4816F067FA01980AF06FFF95F831
:10FDB00074305A0610D40748452114F044FD6FF002
:10FDC0001204204602B070BDA802002018030020D3
:10FDD0002003002097AB0200214601AA42F2030053
:10FDE00004F01CFC04460028EBD1019BBE48996836
:10FDF0000822013116F0B6F901980AF047FF2146B2
:10FE000001AA42F2020004F009FC04460028D8D1FD
:10FE1000019B9B68B3F80120A5F8FC2091B221B1A9
:10FE2000DA78B248114618F0A0FC01980AF02EFFCB
:10FE300095F8746016F0200600F0F78095F894307D
:10FE40001B0711D501AA002142F21C0004F0E6FBB9
:10FE500004460028B5D10198836853F8012F5B68E8
:10FE6000C5E936230AF012FF95F8D0309E0623D557
:10FE70000DF10201684604F033FC04460028A0D1CD
:10FE8000042142F2240004F08DFA0646002800F016
:10FE9000D380042108300BF00FF8BDF80030038048
:10FEA000BDF8023043802246314642F2240004F07D
:10FEB000B5FB0446002884D195F8D0305C0610D5F7
:10FEC00001AA002142F22A0004F0A8FB04460028FF
:10FED0007FF477AF019883685B7885F818310AF072
:10FEE000D5FE082142F2010004F05CFA0446002825
:10FEF00000F0A280082108440AF0DEFF95F8D01037
:10FF000011F0400F024640F2022308BF0323880786
:10FF10004CBF43F02C0043F00C008B0695F8D13019
:10FF200048BF40F0400013F0090F95F89A3018BF11
:10FF300040F4006003F00603CE0748BF40F0100015
:10FF4000062B08BF40F4C070002116F065FA214668
:10FF5000002242F2010004F061FB044600287FF415
:10FF600030AF95F8743098061ED4B5F8FC10D9B9A6
:10FF700001AA41F2050004F051FB044600287FF479
:10FF800020AFB5F8FC3063B9019B9B685A7899782B
:10FF900042EA0122A5F8FC209A885448114618F03C
:10FFA000E4FB01980AF072FE082140F6014004F0DB
:10FFB000F9F9044600283FD0082108440AF07CFFE4
:10FFC00095F8D030D90702464BD545A1D1E90001BB
:10FFD00016F022FA2146002240F6014004F01EFBF2
:10FFE000044600287FF4EDAE014601AA4FF6014019
:10FFF00004F014FB0446002837D03D48572114F084
:020000021000EC
:1000000022FC16F08DFB044600287FF4DAAE06F0E1
:1000100099FC044600287FF4D4AEEB79002B55D12F
:100020003448492114F00FFCCBE6022140F66D4024
:1000300004F0B8F9044610B96FF06804C1E6022173
:1000400008300AF039FF012303704670214632461A
:1000500040F66D4004F0E2FA044600283FF4EEAEAC
:10006000AFE625484FF00051B2E701980AF00EFEC6
:10007000214601AA4FF6024004F0D0FA044610B11E
:100080001E485721BBE7019B1D4899680222013198
:1000900016F068F801980AF0F9FD95F8B9305B0799
:1000A000AFD501AA21464FF6034004F0B7FA10B1CC
:1000B00014485721A3E7019B134899680122114472
:1000C00016F050F801980AF0E1FD9AE704210F4874
:1000D00016F093F904F06AFD73E600BFAFF30080F9
:1000E000908800020080002078030020A8030020F0
:1000F000C0AB020045AC020010880002E9AB020070
:100100006103002017AC020060030020740300208C
:10011000014B1878704700BF0832002008B504482A
:1001200014F0E4F8BDE80840012018F0BEB900BFA3
:100130005F980200CB0710B506D500F001042046F9
:1001400002F012F9014B1C7010BD00BF08320020F4
:1001500008B521B1BDE80840054814F0C7B8054806
:1001600014F0C4F8BDE80840012018F09BB900BFA6
:10017000799802009598020070B503788AB0044619
:100180000E4607AD032B20D8DFE803F002191B1D34
:100190001149284615F08AFF63780493A3780393E6
:1001A000E378029323790193637900930B4AA3794F
:1001B00005951E21304614F0A6F80AB070BD084916
:1001C000E7E70849E5E70849E3E7084A0A2128463E
:1001D00014F099F8E0E700BFA0980200C998020067
:1001E000A7980200AE980200B8980200C2980200D8
:1001F00030B589B00C46154616F06EFC6946FFF71F
:10020000BBFF35B906482246694614F06FF809B0BD
:1002100030BD04482B462246694614F067F8F6E7DD
:10022000EC9802000B99020010B588B00C4616F04D
:1002300053FC6946FFF7A0FF03482246694614F0C5
:1002400055F808B010BD00BF3099020000B589B064
:1002500016F042FC6946FFF78FFF0348694614F029
:1002600045F809B05DF804FB4699020010B588B066
:100270000C4616F031FC6946FFF77EFF0348224624
:10028000694614F033F808B010BD00BF5D99020054
:1002900010B588B00C4616F01FFC6946FFF76CFFDE
:1002A00003482246694614F021F808B010BD00BF8B
:1002B0008099020030B52C4889B014F017F80CF082
:1002C000E3FC014620B1294814F010F809B030BD14
:1002D00027480CF01DFD0446002836D0014625486D
:1002E00014F004F824482146EEE7244813F0FEFFFA
:1002F00014F091FC224802F02DF8014608B1214883
:10030000E2E7214D0FCD03AC0FC42B68236001231E
:1003100000931E491E4B022203A805F045FA04462D
:1003200010B101461B48CFE71B4813F0DFFF013433
:1003300004F0010148BF494200200CF083FD002178
:100340004FF4004010F06EFBF1E7144806F012F98C
:10035000134806F0DBFA204604F03AFC0146002878
:10036000C3D01048B0E700BFA4990200CF990200A3
:1003700035010100EA990200099A0200469A02003A
:10038000600400205D9A0200808E0200288F020027
:10039000388F02007A9A0200A09A020044040020DA
:1003A00020040020269A020030B50A4C0A449142EB
:1003B00000D130BD11F8013B58400309E35C83EAEA
:1003C0000013DDB2C3F30313E05C80EA0510C0B292
:1003D000EDE700BFCD9A0200436803F00303022B50
:1003E00070B504460E46816010D0032B04D0012B5B
:1003F0000FD10025284601E0056800200023636036
:1004000010B1314611F008FA284670BD0068002589
:10041000F4E705490548452213F068FF02484521E5
:1004200014F009FA0025E8E7DD9A0200009B0200BB
:100430000B6801330B60014B1B68184768040020F0
:10044000014B1860704700BF6804002007B50B46D9
:10045000002102460191034801A900F0D5FB03B039
:100460005DF804FB3104010030B585B0CDE9010130
:100470000446002501A90548039500F0C5FBDDE908
:1004800002309842B8BF255405B030BDC7420200C3
:100490002DE9F74FB0F81CA01AF0080F0446934658
:1004A0001CD001290CBF4AF0100A4AF0200AA0F81B
:1004B0001CA004F114000EF0B3FB40B9BA49BB48CC
:1004C000AC2213F013FFB848AC2114F0B4F98BF34D
:1004D0001188BFF36F8F03B0BDE8F08FB44FDFF822
:1004E000CC820AF0070A022906D1204613F018FF31
:1004F0000028DED0012865D1D4F81890A38BB9F17B
:10050000000F19DA0026256823F00703C4E9006606
:1005100043F00103A383A38B03F00702524500922B
:1005200003D0A268002A40F0F18015B9002E00F037
:100530002B814FF0000AEBE003F00702511F012965
:1005400022D8002123F00703062A25689BB2C4E9BC
:1005500000110CD18D422A4638BF0A462AB1E18BE0
:1005600012680131E183002AF8D143F00203A3832A
:10057000204613F0D5FE06460028CCD0A38B43F0CE
:100580002003A3830026C6E7042A0DD123F0070326
:100590009AB2A283204613F0C3FE054680B142F012
:1005A0002002A2830025EDE740F21B1239464046A7
:1005B00013F09CFE40F21B11384614F03CF9002564
:1005C0002E46A8E7032831D1BAF1000F0AD03946E8
:1005D00040464FF4AB7213F089FE4FF4AB713846CE
:1005E00014F029F9236853B93946404640F25712AE
:1005F00013F07CFE40F25711384614F01CF92369C1
:100600001E6856B9394640464FF4AD7213F06EFE7F
:100610004FF4AD71384614F00EF9A38B23F00703A5
:1006200043F00603A3830025A94674E704282ED1CE
:10063000BAF1020F0AD03946404640F25D1213F07B
:1006400055FE40F25D11384614F0F5F8E38B53B1D6
:10065000394640464FF4AF7213F048FE4FF4AF7185
:10066000384614F0E8F823695E6856B939464046C2
:1006700040F2611213F03AFE40F26111384614F074
:10068000DAF8A38B23F0070343F00403CAE7052835
:100690002ED1BAF1010F0AD0394640464FF4B2725A
:1006A00013F024FE4FF4B271384614F0C4F82368F6
:1006B00053B93946404640F2651213F017FE40F236
:1006C0006511384614F0B7F823699E6856B9394663
:1006D00040464FF4B47213F009FE4FF4B47138463B
:1006E00014F0A9F8A38B23F0070343F0050399E75F
:1006F00040F26B123946404613F0F8FD002540F2F7
:100700006B11384614F097F82E468DE74FF0010A2A
:1007100043F00803A38304F11403184601930EF079
:100720007FFA40B920494046AC2213F0DFFD1E4855
:10073000AC2114F080F88BF31188BFF36F8FBAF1FE
:10074000000F39D1002D4CD116B11A492046B047BF
:100750004FF04003EFF3118B83F31288BFF36F8FD9
:1007600001980EF04FFA40B90F494046812213F02C
:10077000BDFD0D48812114F05EF801980EF060FA7D
:10078000A38B23F00803A383A38BDA0631D523F0D0
:100790001003A3830121B4F81CA00AF0070A002962
:1007A0007FF4A1AE85E600BF3A9B0200009B0200E9
:1007B000189B020005080100A1680029C2D00B683F
:1007C000D1F804B0009A002B38BF00239A46204687
:1007D0004B46D847BAF1000FB4D0DAF80030514692
:1007E000EEE72946009A2D684B46204613F0B4FDEB
:1007F000A8E713F020011EBF23F02003A3830221EA
:10080000C9E700BFF8B504460D4600F114064FF0E5
:100810004003EFF3118783F31288BFF36F8F3046E5
:100820000EF0F0F940B90A490A48812213F05EFD42
:100830000748812113F0FFFF30460EF001FAA56151
:100840003A4620460121BDE8F840FFF721BE00BF2F
:100850003A9B0200009B02002DE9F04704460F4638
:1008600013F090FD051E54DB04F114094FF0400312
:10087000EFF3118A83F31288BFF36F8F48460EF0AF
:10088000C1F940B933493448812213F02FFD314872
:10089000812113F0D0FF48460EF0D2F9E38BA28BF2
:1008A0004FF6FF718B4202F007064AD0022E1FD18D
:1008B0000133E38335464FF0010848460EF0B0F9A6
:1008C00040B924492448AC2213F010FD2148AC2142
:1008D00013F0B1FF8AF31188BFF36F8FB8F1000FE7
:1008E00017D0002332463946204613F035FD10E07C
:1008F000930701D0062E0FD100233B606368EBB94C
:10090000C4E900773546F6B9524602212046FFF782
:10091000BFFD2846BDE8F087052E17D0012E0AD06E
:100920000E490D4840F2C91213F0E0FC0B4840F2AA
:10093000C91113F080FF6FF0040504E01F606760C9
:10094000E0E76FF00A054FF00008B6E76FF08505A5
:10095000F9E700BF3A9B0200009B0200189B0200CF
:1009600070B5002939D00568AB68B3F5004F2CBFCE
:10097000082404240C1B641BE40801222146284699
:1009800013F02CFDC30708D4144915489A2213F01C
:10099000ADFC12489A2113F04EFF2146284613F071
:1009A00033FD261831460022284613F017FD361A6B
:1009B000B44208D009490A48A22213F097FC07481C
:1009C000A22113F038FF21462846002213F022FD11
:1009D0002146BDE8704013F058BE70BD609B020018
:1009E000009B02002DE9F0470668B3681446B3F592
:1009F000004FC1F1000202EA01072CBF08250425BF
:100A000031EA02021AD0BD4228BF3D46B946CF1B8B
:100A100007F1FF3A1AEA070F0AD03449344840F286
:100A20000D1213F063FC314840F20D1113F003FF77
:100A300074B94FF000094846BDE8F087A94204D8D0
:100A40002146BDE8F04713F062BE4FF00009DFE732
:100A5000B368B3EBD40FECD93919491B304613F006
:100A6000F5FC0146304613F07BFD80460028E0D0BF
:100A7000B368B3F5004F2CBF0823042309EBC0056E
:100A80001D44354455447F422F40A7EB09094C448F
:100A9000A9EB030307349B1B24F00704A41BB0EB52
:100AA000D30F4FEAD3074FEAE40408D201463A468F
:100AB000304613F0FFFC4146304613F08AFD3946BC
:100AC000304613F0A1FC3844844208D239463046FF
:100AD000224613F0EFFC2146304613F07AFD012246
:100AE0003946304613F096FCA5E700BF609B020034
:100AF000009B0200B2F5802FF8B507460D4616465A
:100B00000ED2042A0AD83E493E484FF4C17213F06F
:100B1000EDFB3B484FF4C17113F08DFE042200E061
:100B20000822B61AEC1D354424F0070425F0070509
:100B30002D1B172D4FEAD5060AD83149314840F20E
:100B40008B1213F0D3FB2E4840F28B1113F073FE7F
:100B500000233C603146E360A660204613F080FC31
:100B600001218500471C204613F070FC1B35ED0861
:100B70002844B0420AD9224922484FF4CB7213F0DC
:100B8000B5FB1F484FF4CB7113F055FE002304F161
:100B900010021946BB422FDB2A462046002113F0E3
:100BA00051FC00231A461946204613F022FC771BFD
:100BB00020460122002113F02DFC3A46294613F06D
:100BC00041FC2B4629462046002213F012FC3146F8
:100BD0002046002213F036FC3B46314620460022D8
:100BE00013F007FC31462046012213F013FC29467E
:100BF000BDE8F84013F0EDBC42F8041B0133C9E72F
:100C0000609B0200009B02002DE9F04F91B08B46E3
:100C1000029092461C4600259AF8000008B9284622
:100C20005EE325280AF1010707D0029B5946984741
:100C30000028C0F25583013510E2182200210AA8CD
:100C400015F09BFA9AF80130252B78D000229446B3
:100C5000164696461046394617F8013B2B2B00F0F6
:100C60009D8000F29480202B00F09B80232B00F0CD
:100C70009A8028B19DF8300040F004008DF83000D3
:100C8000BEF1000F05D09DF8300040F008008DF84F
:100C900030002EB19DF8300040F010008DF830008B
:100CA000BCF1000F05D09DF8300040F020008DF819
:100CB00030002AB19DF8302042F040028DF83020FB
:100CC0009DF8302002F04400442803D16FF38612CF
:100CD0008DF830209DF830202A2B42F080028DF8CC
:100CE00030207BD19DF8312042F001024B1C8DF861
:100CF00031201A782E2A9DF831200CBF01210021C5
:100D000061F341028DF8312074D15A782A2A6AD0D1
:100D1000013300210A26184610F8012BA2F13007F2
:100D2000092F40F28E809DF830200E91C2F34000D2
:100D300040EAD17161F341028DF830205AE00AF1A6
:100D400002078DF833309DF83130D90740F14981E1
:100D500054F8049BB9F1000F07DA9DF8302042F0F7
:100D600004028DF83020C9F100095A0740F1428190
:100D700054F8048BB8F1000F80F241819DF83130B6
:100D80006FF341038DF831304FF0FF3837E12D2BF1
:100D90000CD0302B7FF46DAF01225CE74FF0010ED9
:100DA00059E7012657E74FF0010C54E7012052E7BD
:100DB0000CFB0202303A33461E4616F8010BA0F136
:100DC0003007092FF4D9994293D09DF830100D9235
:100DD000D20F62F341018DF830108AE70B460022F2
:100DE0004FF00A0CE8E79DF8312042F004028DF83C
:100DF000312002331F4617F8012B6C2A41D025D829
:100E0000682A2BD06A2A46D04C2A4CD01F4617F8A5
:100E1000012B9DF831308DF83320782A00F2D980EB
:100E2000572A4DD8412A03D0453A022A00F2D180F0
:100E30009DF83230042262F302038DF83230012330
:100E40009EE006FB01213039034664E7742A26D070
:100E50007A2ADBD19DF8313006220DE05A78682AD3
:100E60009DF8312006D1012161F3C6028DF83120B1
:100E70009F1CCCE71346022262F3C6038DF8313083
:100E8000C5E75A786C2A9DF8312001D10421EBE79F
:100E900013460322F0E79DF831300522ECE79DF878
:100EA00031300722E8E7BDF8303023F4F04323F077
:100EB000020343F4804343F00203ADF83030A6E769
:100EC000A2F15801202900F2848001A050F821F0FD
:100ED000950F0100D30F0100D30F0100D30F0100C4
:100EE000D30F0100D30F0100D30F0100D30F010076
:100EF000D30F0100310E0100D30F0100950F010047
:100F0000550F0100310E0100310E0100310E0100BC
:100F1000D30F0100550F0100D30F0100D30F0100C3
:100F2000D30F0100D30F01009D0F0100950F0100A9
:100F3000B90F0100D30F0100D30F0100B90F010059
:100F4000D30F0100950F0100D30F0100D30F010053
:100F5000950F01009DF83210012003F0780360F333
:100F60000201402B8DF8321002BF9DF8301041F085
:100F700001018DF83010632A31D1003B18BF0123E5
:100F80009DF83020C2F340010B4363F341028DF81A
:100F90003020D8E69DF832100220DEE79DF832209E
:100FA00003F07803A3F14000032161F302024342FE
:100FB0008DF832204341E3E79DF83220032113F0FE
:100FC000780F61F302028DF8322014BF0123002351
:100FD000D6E79DF8303043F001038DF83030002320
:100FE000CEE79DF93020002AB4BFDDF834904FF0F1
:100FF000FF39BAE69B077FF5C7AEDDF838809DF86C
:1010000031200023CDE90D339DF8323003F0070382
:10101000012BC2F3C30236D1D31E042B20D8DFE844
:1010200003F00307071F1F0054F8040BC11704E067
:10103000073424F00704F4E80201CDE90A019DF821
:10104000303013F0030654D002983B4652465946BE
:1010500013F0DBFB0028C0F243810544BA46DBE510
:1010600054F8040B012A4FEAE071CDE90A0105D1D9
:101070009DF828300A9300230B93E0E7022ADED183
:10108000BDF92800D2E7022B23D1D31E042B13D89D
:10109000DFE803F0030A0A12120020680A90002118
:1010A000231D0B911C46CAE7073424F00703F3E81D
:1010B0000201CDE90A01F5E754F8043B0A93012A3D
:1010C0004FF000030B93D3D0022AB8D1BDF82830DB
:1010D000D0E7042B07D1073424F00704F4E8020119
:1010E000CDE90A01ABE7032B04BF54F8043B0A9394
:1010F000A5E79DF833007828B0D8622822D82528A3
:101100003FF493AD5828A9D10DF126030093DDE9F2
:101110000A0104AB0CAA13F02DFB8246B8F1000FB4
:101120000DF126000CDB9DF83020A0EB0A036FF3D5
:10113000861298458DF8302002D9A8EB03030D9351
:1011400080463DE06338152888D801A151F820F089
:10115000D1110100351201005D1001005D10010088
:101160005D1001005D100100351201005D100100ED
:101170005D1001005D1001005D100100931201007F
:1011800061120100651201005D1001005D10010097
:10119000A91101005D100100611201005D10010044
:1011A0005D10010061120100B8F1000FDDF828A008
:1011B0000ADB4146504614F08AFF0AEB000800267D
:1011C000BAF1000F0CD149E7504614F079FFF4E76B
:1011D0000A9B8DF8103000260DF111080DF1100A50
:1011E000A8EB0A0306B101339DF83220D0066BD577
:1011F000023352060D9948BF0E9A0B4448BF9B1804
:10120000B9F1000F79DD9DF83020A9EB0309C2F395
:1012100080030393530770D4500664D546B1029BF4
:1012200059463046984700285ADB039B01351E4635
:10123000302359E01E0711D413F0100618BF2026E2
:10124000DDE90A23002A73F10001BFF65DAF5242C7
:1012500063EB4303CDE90A232D2655E72B26EFE761
:10126000002651E70A9848B30DF1260300930CAA13
:1012700004AB002113F07EFABDF8323003F0EF0327
:1012800043F4F04343F010038246ADF832300026B9
:1012900044E70A9B072A3FF6E1AEDFE802F00D04BF
:1012A000060D08080D0D1D70D8E61D80D6E62846EF
:1012B000E917C3E90001D1E61D60CFE6DFF8C4807D
:1012C0000646A8F1050A8BE7110748BF013390E7EE
:1012D000184603935946029B98470028039B04DA5B
:1012E00011B0BDE8F08F20234D444A46002AA5EBFB
:1012F000090109F1FF39EBDC0D4636B1029B594675
:10130000304698470028EBDB01359DF83230D9068E
:1013100001D41A0706D5029B594630209847002869
:10132000DEDB01359DF83230DB0607D59DF8330052
:10133000029B594698470028D2DB01350D9E2E446A
:10134000731B002B16DC029843465246594613F095
:101350005CFA0028C4DB0544A944A9EB0503002B73
:101360007FF77CAE029B5946202098470028B7DBC8
:101370000135F2E7029B5946302098470028AFDB41
:101380000135DDE7869B020008B504464FF04002B8
:10139000EFF3118382F31288BFF36F8F17F081F898
:1013A000204601F0E9FF034812F0A0FF01F060FAC7
:1013B000FCE700BF879B02002DE9F74FCDE9000154
:1013C000DFF8A480DFF8A49016461446019B9D190F
:1013D0002D1B14B903B0BDE8F08F009B1E4F013BDD
:1013E000032B96BF1D4A3F21D15C404612F07EFF81
:1013F0004FF0000B5C4526D915F80B10384612F05B
:1014000075FF0BF1010BBBF1080FF3D11448DFF8A6
:1014100060A0DFF860B012F069FF0027BC4216D967
:10142000E95DA1F120025F2A28BF2E21584612F063
:101430005DFF0137082FF1D10A4812F057FF072C42
:10144000C8D9083CC2E7484612F050FFD9E75046D9
:1014500012F04CFFEDE700BFB59B0200C49B0200F9
:10146000BF9B020001C70200B09B0200BB9B0200B1
:10147000BD9B0200C19B02002DE9F7430F460646C3
:101480000821C06A13F0A8FA3C68134B241A80465E
:101490003C6004EA03059946AC4203D8002003B03F
:1014A000BDE8F08308236A462146304613F0F7F979
:1014B0000028F4D16946304613F098FA40B1BDF8DF
:1014C0000230BDF804203C6005EA090513441D44C0
:1014D000A4EB0804E0E700BF0000FFFF2DE9F04F98
:1014E000044695B0C06A082113F076FA63681B0CB5
:1014F0001B04054603A9E089039313F091FA039BAB
:10150000A18906AE1944491B32460823204604919E
:1015100013F0C5F9021EC0F2AB80E36A1A7900230A
:10152000F15C914240F092800133082BF8D1A06821
:1015300063682844834280F081800399204613F039
:101540000BFA024694E0049BBDF81A201B0C1B0406
:1015500013440493DFF820B1DDF810A008AA04A911
:10156000204613F0E1FA0246002840F0818008A9E5
:10157000204613F03BFA002836D0636805930AAA88
:1015800005A92046059E13F0CFFA024600286FD128
:10159000BDF82820BDF820309A4228D06268059B0B
:1015A0009A42ECD156451FD1BDF82430E3B1BDF8C5
:1015B00022300AEA0B071F4408A8A368ADF82230BE
:1015C00013F001FAE36ABDF824801E68764206F043
:1015D00020030193B8F1000F10D108A9204613F0A1
:1015E0007DFA0246002843D1CA45B5D19FE70AA932
:1015F000204613F0FBF90028D0D0D3E7019B4345E8
:1016000028BF43460CAA394620461E4613F047F928
:10161000024668BB36B10CAAA1683346204613F0D7
:1016200028FA02463146E06A13F0D6F9A16801446F
:10163000A160EAB9A8EB06083744CBE7204613F0CF
:101640005EFA024600283FF478AF11E0049B314671
:101650002046A3EB050913F0EEF900287FF473AFE1
:1016600004A92046FFF708FF024600283FF472AFA6
:10167000104615B0BDE8F08F0000FFFF2DE9F047E0
:10168000044688B00D4600F11407384617F038F8C4
:1016900028460CF073FEA06248B9AD48452113F00E
:1016A000D2F86FF00505284608B0BDE8F0878368DA
:1016B0001B699847E06230B9A648452113F0C3F88A
:1016C0006FF01505EFE7A06A83681B699847036808
:1016D000013B1F2B02D9A0484521EFE7A06A2168F2
:1016E00005AA16F018FE10B19C484521E6E7A3892B
:1016F0002BB1069AB3FBF2F502FB153515B19848EC
:101700004521DBE7E389012B02D896484521D5E73F
:10171000E36A009593F804804FF0FF324FF0FF33F7
:1017200038460DF0BDFAE06A082113F055F9A946D4
:101730000646E3891FFA85FA534544D8E3894B45A9
:1017400000F0D68053450BD1009908234246891BEF
:10175000204613F0DCF818B9E089694613F060F907
:1017600069462046FFF788FE0546002840F0C28003
:10177000009B7D4A63601340A3609146D4E9011346
:1017800099420ED3082301AA204613F088F8C0B965
:1017900001AB13F8012B904540F0F280013008288E
:1017A000F7D16368E0891B0C1B046946009313F0B2
:1017B00037F9A38900994246204613F0A8F800287B
:1017C00025DA054696E0A1892B04891B13FA81F1DD
:1017D000424608232046009113F099F878B1E08939
:1017E000694613F01DF909F10109009908234246E1
:1017F00020461FFA89F913F08AF800289ED0013597
:1018000097E7002A00F0D4806FF01C0572E04AD000
:101810006368334400934FF6FF780099A3898AB236
:101820009B1B9A421AD35148492113F00CF8616866
:10183000204613F091F80028C3D162684A4902EAB1
:101840000103A2891344A3EB460363600B40A3602A
:101850002046FFF743FE002840D0B2E7082303AA42
:10186000204613F01CF80028ABD103A9204613F042
:10187000BDF838B1BDF80C30434503D1BDF8103088
:10188000002B54D0009B33440093C6E75B1A4246BA
:10189000204613F03CF8002893DB08D0E26AA368E6
:1018A00012681344A360D4E901318B42EED8616819
:1018B000A38901EB46029A42CDD1DFF8AC80A36840
:1018C00001EA08029342C6D0204613F045F80028EA
:1018D0007FF477AF636803EA0803A360A089A38855
:1018E000A0EB4606B34205D1204613F008F968E79D
:1018F0006FF02C0538460DF0ABFA002D7FF4D3AE17
:101900000123E28923741A48A389492112F09BFF1D
:101910006268184893B24921120C12F094FFA26831
:10192000154893B24921120C12F08DFFBBE6134803
:10193000492112F088FF6368E0891B0C1B0469468B
:10194000009313F06DF80099204613F005F882E734
:10195000E19B0200029C0200299C02004B9C0200B9
:10196000689C0200819C02000000FFFF0C9D0200A9
:10197000A99C0200C59C0200DC9C0200F29C0200B3
:1019800001A9204613F032F8D4F804A080B1009BDE
:10199000BDF80820BDF80610E06A03EA0903A36059
:1019A000114413F019F803445345A3603FF429AFE1
:1019B000AAEB06036360E1E62DE9F04F1E46037CC7
:1019C00089B00446894690464BB96548452112F0D6
:1019D0003AFF6FF00C05284609B0BDE8F08FC36AE6
:1019E0000821184612F0F8FF31468246184612F0D8
:1019F000F3FFA389A3EB8A039E42074600F2AB8064
:101A000016B1002A00F0A7806368039304AA03A913
:101A10002046DDF80CB013F087F805460028DAD12F
:101A2000BDF810304B4505D06268039B9A42EDD15A
:101A3000E6B9D0E704A9204612F0D8FF0028F3D079
:101A4000BDF8143086B19E4210D1BDF812004FEAA5
:101A50001B410904014433464246204612F02DFF43
:101A6000002803DC0546B6E7002BB4D0002F3FD199
:101A700004F1140A4FF0FF324FF0FF335046DFF805
:101A8000E4B00DF00DF90022E3899A4260D0D4E968
:101A90000131781883422ED3FF2306A8ADF81890A1
:101AA000ADF81A10ADF81C608DF81E3012F08BFFE7
:101AB00036B1A16833464246204612F0DAFF0546A9
:101AC000E06A314612F088FFA3680344A360002D4A
:101AD00044D106A9204613F001F8054600283DD15F
:101AE0003346019350460DF0B3F9019B1D4672E752
:101AF0005744BFB2BCE7E06A0192082112F06CFFC4
:101B00004FF6FF71ADF818100021ADF81C10191830
:101B1000ADF81A10A18903EA0B030B44181A606090
:101B200006A812F050FF06A9204612F0D7FFE08960
:101B3000211D12F075FF636803EA0B03A3602046C2
:101B4000FFF7CCFC03460028CBD1019A01329BE77A
:101B50006FF01B03C5E76FF015053CE72B46C0E7A8
:101B6000C89B02000000FFFF2DE9FF471E46037CD3
:101B7000BDF8309004460F46904643B928484521A9
:101B800012F061FE6FF00C0004B0BDE8F087C06A8F
:101B9000082112F021FFA389A3EB40039E423CD809
:101BA000636801934FF0000A02AA01A92046019D33
:101BB00012F0BAFF0028E7D1BDF80830BB4208D1C7
:101BC00002A9204612F012FF18B10AF1010A1FFA09
:101BD0008AFA6268019B9A4218D0D145E4D2BDF8D6
:101BE0000C30BBB1D14515D8BDF80A102D0CB3424D
:101BF0004FEA054528BF334642462944204612F0A5
:101C00004EFE0028C0D1BDF80C00BDE7BDF808307D
